:020000040000FA
:20000000C0070000D1060000D1000000B106000000000000000000000000000000000000BA
:20002000000000000000000000000000510700000000000000000000DB000000E5000000A8
:20004000EF000000F9000000030100000D01000017010000210100002B010000350100000A
:200060003F01000049010000530100005D01000067010000710100007B0100008501000068
:200080008F01000099010000A3010000AD010000B7010000C1010000CB010000D5010000C8
:2000A000DF010000E9010000F3010000FD01000007020000110200001B0200002502000024
:2000C0001FB5C046C04600F0EFFA04B00FB41FBD08205A49096809580847382057490968BF
:2000E000095808473C2055490968095808474020524909680958084744205049096809584A
:20010000084748204D490968095808474C204B49096809580847502048490968095808472E
:2001200054204649096809580847582043490968095808475C2041490968095808476020CF
:200140003E4909680958084764203C49096809580847682039490968095808476C20374996
:20016000096809580847702034490968095808477420324909680958084778202F4909687F
:20018000095808477C202D4909680958084780202A49096809580847842028490968095861
:2001A0000847882025490968095808478C2023490968095808479020204909680958084746
:2001C00094201E4909680958084798201B490968095808479C201949096809580847A020A7
:2001E0001649096809580847A4201449096809580847A8201149096809580847AC200F49D6
:20020000096809580847B0200C49096809580847B4200A49096809580847B8200749096896
:2002200009580847BC200549096809580847000003480449024A034B7047000000000020BA
:20024000C0070000C00700000122D84B5A6000BFD74A1268002AFBD0016000BFD44A126809
:20026000002AFBD00022D14B5A6000BFD04A1268002AFBD07047F0B505460E4617460024CD
:2002800006E0A200B158A2005019FFF7DDFF641CBC42F6D30020F0BD0120C043C549086042
:2002A0004010486070470146012292040868904201D9102070470020FCE7F0B505460C4647
:2002C0001646002706E028462168FFF7BDFF2D1D241D7F1CB742F6D3F0BD70B505460C46B5
:2002E0002E460BE0304600F075F9FF2C01D8002401E0FF3C013C012080023618002CF1D16B
:2003000070BD0146012292044868904201D909207047A9484069401C01D10F20F8E700207E
:20032000F6E7FEB504462068030000F037FA05042B4249598B00201DFFF7E3FF0546002D07
:2003400001D02846FEBDFFF7A7FF0120C00200F041F9042221469948FFF78DFF002801D011
:200360000320EFE708222146944800F06DF9002806D1002192480068FFF766FF00F00CF90F
:200380000320DFE7A768E6686068019031463846FFF7A3FF324638460199FFF78EFFB2006C
:2003A0003846019900F050F9002800D1CAE70320C8E700F0E3F9834800688349086041E01C
:2003C00060680190E668A0680090B2000099019800F03AF90746002F00D1B3E70E20B1E72A
:2003E000201DFFF760FF0546002D01D02846A9E76068002807D1FFF74FFF0320800200F083
:20040000E9F800F0C9F8FFF747FF0120C00200F0E1F8042221466948FFF72DFF002801D009
:2004200003208FE708222146644800F00DF9002806D1002162480068FFF706FF00F0ACF82F
:2004400003207FE700BF00207CE770B505460C46182D04D12068FFF764FF206002E0012091
:20046000206000BF00BF70BDF0B589B05248406903905248806881000398081802900398B2
:20048000000B01900121090302984018401E000B00900124002520462946019A00F0C4F841
:2004A0000022401E9141079106900126002730463946009A00F0B8F80022401E9141059157
:2004C0000490049BDB43059AD243069818430799114307910690374906980860079848602F
:2004E00009B0F0BD70B534484469344885684668AA003146204600F0A7F8002801D0002002
:2005000070BD0120FCE72D484068002801D0012000E000200546FFF7E5FF002807D0FFF759
:20052000BBFE0320800200F055F800F035F8FFF79BFF002D0ED0204846692048846847684E
:2005400021463046FFF7C9FE224639463046FFF7B4FE00BF00F020F810B5184844681A4802
:200560000460204600F0DCF810BD154800680068401C01D100BFFEE710480068002802D067
:20058000042806D101E0FFF7BEFFFFF7E5FF00BFFEE700BF00BFFEE7BFF34F8F0B480C49AB
:2005A000C860BFF34F8F00BFFEE7000000E5014000E4014000060040001000100008000026
:2005C000B8070000BC070000000000200400FA0500ED00E010B50146104B1A68084602234D
:2005E0000F4C636000BF0F4B1B68002BFBD0531C04D0904202D20A4B186101E0084B986068
:2006000000BF084B1B68002BFBD00023044C636000BF044B1B68002BFBD010BD00100010A5
:2006200000E5014000E4014010B5202A04DB0146203A9140002010BD914020239C1A03460F
:20064000E3401943904010BD034610B50B439B070FD1042A0DD308C810C9121FA342F8D00B
:2006600018BA21BA884201D9012010BD0020C04310BD002A03D0D30703D0521C07E000202C
:2006800010BD03780C78401C491C1B1B07D103780C78401C491C1B1B01D1921EF1D1184627
:2006A00010BD70477047704710B500F007F810BD014B1B68DB6818470000002019481A4972
:2006C0007047FFF7FBFFFFF7FBFC00BD20BFFDE71649174C24688C420BD1164B1B6899424F
:2006E0000CD1154B154A1360186810498842EDD00AE0134880F30888124B18470F4A1360BB
:2007000018680A498842E1D080F308880E49884204DD0E48026802210A4302605B681847D2
:200720000346DFE7C0070000C0070000FFFFFFFF000C0000141000100010000000000020B0
:20074000000400206B05000000200020240500400D48704502D1EFF3098101E0EFF30881C7
:20076000886902380078182802D1C046074A1047074A12682C3212681047000000B5054B16
:20078000054A9B58984700BDFDFFFFFF4B04000000000020001000000400000030B4744660
:2007A000641E2578641CAB4204D3635D5B00E31830BC18471D46F8E7000C00000010000017
:20100000881D0020E14F0100993D0000474F0100000000000000000000000000000000006D
:20102000000000000000000000000000515001000000000000000000993D0000993D000062
:20104000BD500100C3500100993D0000993D0000993D0000993D0000993D0000993D00006A
:20106000C9500100993D0000993D0000CF500100993D0000D5500100DB500100E150010030
:20108000993D0000993D0000993D0000993D0000993D0000993D0000993D0000993D0000A0
:2010A000E7500100ED500100993D0000993D0000993D0000993D0000993D0000993D0000B6
:2010C00000F002F813F06DFF0CA030C8083824182D18A246671EAB4654465D46AC4201D1F7
:2010E00013F05FFF7E460F3E0FCCB6460126334200D0FB1AA246AB4633431847AC4001008B
:20110000DC400100103A02D378C878C1FAD8520701D330C830C101D504680C6070470000CD
:201120000023002400250026103A01D378C1FBD8520700D330C100D50B6070471FB5C04605
:20114000C04613F0CFFE04B00FB41FBD826902498161024810447047611100000100000086
:2011600001B41EB400B510F0E7FB01B40198864601BC01B01EBD0000F0B44046494652469D
:201180005B460FB402A0013001B50648004700BF01BC86460FBC8046894692469B46F0BCC0
:2011A00070470000C1100000401E00BF00BF00BF00BF00BF00BF00BF00BF00BF00BF00BF14
:2011C00000BFF1D17047000070B505460C46164602E00FCC0FC5103E102EFAD2082E02D3C5
:2011E00003CC03C5083E042E07D301CC01C5361F03E021782970641C6D1C761EF9D270BD74
:201200008307FF22DB0E9A408907090E994000280BDA0007000F0838830828489B001B18B4
:20122000D86990430843D8617047830824489B001B181868904308431860704710B50446BE
:2012400000210120FFF7DCFF00211820FFF7D8FF00210B20FFF7D4FF02211920FFF7D0FF1F
:2012600002210D20FFF7CCFF02210E20FFF7C8FF02210F20FFF7C4FF0221C81FFFF7C0FF85
:2012800003211620FFF7BCFF03211520FFF7B8FF204600F019F8002010BD5A210180704736
:2012A00010B500F03AF810BD0648704710B500F035F810BD704770477047000000ED00E0D4
:2012C00000E400E003F900C330B50446374D95B007202870A81CFFF7E0FF5920A88034481E
:2012E00001F01CFC0546072000F0DCF929462F4800F08CFA641E072C0AD83021684601704B
:20130000847001F0E0FA002802D009A800F0DDFC284601F083FE15B030BD7047F8B5234E33
:201320000446B61E307801270D46002807D0204660380B2808D8204601F09AFB2BE0602CD9
:20134000F9D01C480860F8BD20466C38032803D8204601F0CFFB1EE0204670381F2803D8E4
:20136000204600F037F816E0204690380F2803D8204600F0BBF80EE02046A0380F2803D86B
:20138000204600F023F906E02046B0380F2804D8204600F000F9286000E02F60602CD2D11F
:2013A00028680028CFD13770F8BD00001A000020C53300000130000070477047704770473A
:2013C000704770477047704710B5012801D100F042FA10BD10B57038030013F09FFE150C47
:2013E00012161E22252C33383D41454950555C646C747B8085004A680878114603F093FFEA
:2014000010BD086803F0F7FF10BD0C790B7B8A680868214603F0FFFF10BD086804F075F876
:2014200010BD03F03DFC10BD08884A6880B2114604F03AFA10BD0A790888114680B204F096
:2014400086FA10BD087840B204F091FA10BD088880B204F0ADFA10BD086804F0BCFA10BD70
:20146000086804F0CFFA10BD086804F0F8FA10BD088982B209C9194604F020FB10BD05C9AF
:20148000114604F074FB10BD08884A6880B2114604F08DFB10BD0B7908888A6880B219461A
:2014A00004F0E1FB10BD0B7908888A6880B2194604F09AFC10BD08884B688A6880B21946DB
:2014C00004F0D8FC10BD08884A6880B2114604F023FD10BD088880B204F042FD10BD088879
:2014E00080B204F062FD10BD012010BD10B59038030013F013FE09060F161D242C363F46AC
:201500004E0088888A6883B20888194680B205F07DF910BD08884A6880B2114605F0D3F961
:2015200010BD08884A6880B2114605F017FA10BD08884A6880B2114605F04DFA10BD0888DC
:201540004B688A6880B2194605F07EFA10BD088982B2888883B20888194680B205F0B3FA4E
:2015600010BD08894B6882B20888194680B205F0E8FA10BD08884A6880B2114605F018FB8E
:2015800010BD888882B20888114680B205F0ACFB10BD012010BD10B5B02805D0B12808D0A7
:2015A000B2280BD0012010BD088880B205F08AFE10BD088880B205F0B5FE10BD08884B6802
:2015C0008A6880B2194605F0BEFE10BD10B5A038030013F0A3FD0B070E172028323C434D4A
:2015E000545D65004B6808788A68194607F0EFF910BD88888A6883B20888194680B207F056
:20160000FBF910BD08884C68CB688A6880B2214607F002FA10BD08884B688A6880B2194681
:2016200007F01CFA10BD8888CB6884B208888A6880B2214607F03CFA10BD8888CB6884B2C9
:2016400008888A6880B2214607F05CFA10BD08884A6880B2114607F090FA10BD088982B277
:20166000888883B20888194680B207F090FA10BD08884A6880B2114607F0ADFA10BD0889EF
:201680004B6882B20888194680B207F02AFB10BD08884B688A6880B2194607F0E7FB10BDED
:2016A000012010BD10B507F0CEFC0FF05FFF00F007F810F0ADF808F0C9F908F055F910BDF8
:2016C00001202B49C00308602A490020087003202949800288607047F8B5264D044628787F
:2016E000A04207D0002C05D0002803D023A14D2013F023FC2878A04213D02C700325002396
:201700002349AD021C48002C27D01B4A214E4032214F012C06D0022C13D018A16E2013F013
:201720000CFCF8BD0B6002230B604E6185601B4911625762091D91621749091DD162456056
:20174000F8BD0B6003230B604E610121C9028160134B9362D7624160F8BD0B600B608560BE
:20176000F8BD10B505A1772013F0E7FB10BD000080E100E02000002000F501407372635CA5
:2017800068616C5F63636D5F6161722E6300000000F500407C01002000F00040001100400B
:2017A000488100401CB50446002069460870204609F0CAF86946204608F088FF002803D10D
:2017C000FBA1B62013F0B9FB01A9204608F0DDFE002803D1F6A1BB2013F0AFFB68460078BC
:2017E0001CBD70B5F74D002428462C7620308471C47113F0A1FC28464038047020308473B8
:20180000847484762C74AC7070BDEAE710B50C46ED4982888A8042884A80007808700846E9
:201820000A38847008F087FEFFF7DBFF20460AF0EFF9E44AE0321146383908461446813874
:2018400009F0F0F82146E0480BF084FC09F073F813F072FC10BD10B50120FFF7ADFD10BDA8
:20186000F8B509F049FDD84DD64C0A3D022802D0207C00287CD0207E0026102819D1A078E4
:20188000002803D0CAA1D14813F057FBCD48E838817A89070DD50146267160398989E180E8
:2018A000C17A217281896181C089A0810120A0702676C44F203FB87C002859D1C448694684
:2018C000808908F003FF002805D06946687809784018687004E0BD48B5A11D3013F02DFB11
:2018E000207C002838D0BA488189FF300930406D8089814204D0B548ADA1223013F01DFBA3
:20190000B348808908F088FF002804D1AF48A8A1283013F012FB08F0F6FF00281CD0AC48AA
:201920008089FFF73FFF697840186870A5484038416D20318A7C012A0DD1A54A3E77928927
:20194000C287C87C20700120B876207E102801D0282800D1267626746978002908D09C4857
:201960008289FF300930C28601870120B8746E7009F092FC002805D1207C002802D0A878BE
:2019800001F0F0F8F8BDF8B50F460446FFF768FF8C4D403D28788B4E002813D0002F10D126
:2019A000307E002804D0FF2081A1C63013F0C5FA2C22A91C204613F024F90E20207000200D
:2019C00028708FE07F4D203DA87B002818D0002FF7D1307E102808D0282806D0002804D0CD
:2019E000FF2073A1D23013F0A8FA0120E070E87BA070287C60700F2020700020A87371E06A
:201A00000121204608F0B8FF002807D0307C002851D13946204608F0AFFFF8BDA97C694884
:201A20000C38009068480A38002913D00178052910D2002F56D1491C0170002666700D20F6
:201A40002070012028750622A01C009913F0D9F8AE7447E05C4800210A380170B0780028D6
:201A600014D0002F3ED1307E002803D050A1594813F063FA002565700120524920700A2237
:201A8000091DA01C13F0BDF8B5702BE0394620460BF0CAFA002825D1A87C002805D0002F6A
:201AA00020D149480A380178C5E7A87E002802D0307C002801D00020F8BD002F12D1307EE3
:201AC000002804D08F203AA1800013F036FA002666700A203B4920700622091FA01C13F084
:201AE00090F8AE760120F8BD10B53648017E002908D1007C012805D001210020FFF743FFAC
:201B0000002801D0072010BD012010BD10B501240AF0C6F80443FFF7E7FF044308F00CFFDB
:201B200001462143084610BDF8B51D4614460E4608F04BFD002807D0684608F051FD0028C6
:201B400003D0002C07D101E00120F8BD9B2018A1800013F0F2F908F0EFFCA04204D21D4815
:201B600013A1583013F0E9F9009808F05DF93146009808F06BF9E2B22946009808F022FB43
:201B800008F040FD002804D19F2009A1800013F0D4F908F0D3FE0E4800244030417C0029C1
:201BA00002D044740AF067F90948C480CCE700007372635C6C6C5F6374726C2E73302E6307
:201BC00000000000200300202C00002084060000D80100201502000010B50179002908D09C
:201BE00001290BD0FF20FE49043013F0A6F9002010BD831D42880488022103E04288048865
:201C0000831D01212046FFF78FFF10BDF8B51F4615460E46044609F06FFB022803D0F148A7
:201C2000007C00281FD0F0488089208008F0F4FD002803D1EA49ED4813F07FF90524684691
:201C400008F0F5FD00280ED0009808F037F93070022809D0012807D008F029FE641E240666
:201C6000240EECD10020F8BD3946009808F0C2FA2880002804D1AF20D949800013F05DF966
:201C800008F015FE002804D1D848D549193013F054F90120F8BD38B50446831D821C69466B
:201CA000FFF7B4FF00280DD00020607168460078012808D0022806D0FF20C949253013F0D5
:201CC0003CF9012038BD2071FBE700215BE670B5C44C0546403C2078002803D1C148007ECD
:201CE000002803D0BE49C24813F027F9287808F054FF28780BF079FB002020710120607118
:201D00003921E170207070BD70B5B64D0446403D2878002803D1B348007E002804D0B4485F
:201D2000AF49183813F009F9AF4E2188B089884203D109F0E1FA022807D002202871012028
:201D400068713821E970287070BD7F207076A648E17820304174A17801740020EEE710B51A
:201D6000A04C403C207800280BD19E48007E002807D109F0C1FA032803D009F0C1FA03286A
:201D800004D19A489649653013F0D7F8954900202031C8712071012060713A21E1702070FF
:201DA00010BD70B58F4C0646403C207800280BD18C48007E002807D109F09EFA032803D011
:201DC00009F09EFA032804D1884885497B3013F0B4F8844D2035E87908280CD2E879102252
:201DE000000100196830314600F029FEE879401CE871002000E007202071012060713B2187
:201E0000E170207070BDF8B5764D0446403D2878002803D17348007E002804D0B72070491C
:201E2000C00013F08AF8704F2188B889884203D109F062FA022801D0022022E03E8C6488EC
:201E40007200788CF98B521C944217D3694A51439200504312F04FFF401EFF2180B2F531C8
:201E6000884200D90846844200D22046711C401C12F041FF761C7043401E86B2FE85EE807C
:201E800000202871012068713C21E9702870F8BDF8B5544C0546403C2078002803D151484B
:201EA000007E002804D052484D497E3813F045F8A878002801D0012804D1A888FF21F531F5
:201EC000884204D94A484649783813F036F8464E2988B089884203D109F00EFA022807D03B
:201EE00002202071012060713621E1702070F8BD3D48002720308772A988B185012131762B
:201F0000A978012900D00021817237484030407C002801D009F0AFFF2771E3E770B5314C43
:201F20000546403C2078002807D12E48007E002803D109F0E1F9002804D02D482849A538C0
:201F400012F0FBFF287809F0AEFE00202071012060713021E170207070BD70B5214C054661
:201F6000403C2078002803D11E48007E002804D01F481B490D3012F0E0FF287800280BD0E5
:201F8000012809D0022807D06878402804D318481349143012F0D1FF284609F0A4F9002821
:201FA00001D0002000E00C202071012060713421E170207070BD70B50A4C0546403C207864
:201FC000002807D10748007E002803D109F094F9002804D006480249983812F0AEFF0BE0B3
:201FE000B01B000020030020D8010020AA0200000A060000C40900002978002914D00A2970
:2020000012D0142910D01E290ED028290CD032290AD04B2908D0642906D0FF2904D00B2064
:20202000FD49C00112F089FF284609F0BBFE00202071012060713321E170207070BD70B5C5
:20204000F64C06462078251D002804D120464030007E002803D0F049F14812F06EFF314674
:20206000002008F06FFD2870002804D106223146EC4812F0C6FD012060713221E170207089
:2020800070BD70B5E54C05462078002804D120464030007E002804D0E148DF49183812F0EA
:2020A0004CFF00216956042914D0002912D0081D10D0001D0ED0001D0CD0001D0AD0001DCC
:2020C00008D00A3006D0283104D0D548D249163812F033FFD44829780170012060713121BF
:2020E000E170207070BD10B5CC4C2078002804D120464030007E002803D0C749CB4812F0EC
:202100001CFF08F019FAE08008F0DEFA207200202071012060710521E170207010BDF8B5B3
:20212000BE4C07462034A07B25462035002805D1287E002802D1A878002804D05120B649EE
:20214000000112F0FAFE09F0D7F81026022822D1B7483988808988421DD1B0494839084620
:202160000A7F6038807A002A03D080070CD40C200CE0800708D406200877AD484030407C9F
:20218000002801D009F077FE2E760020E07326740120A073F8BD0220F8E710B59F4C2078F5
:2021A000002804D120464030007E002804D09C489949543812F0C1FE002020710E20A070D0
:2021C0000F20E070FF20A0710020C04320819548C01D0178A1728188A1814088E0810120D1
:2021E0006071207010BD10B58C4C2078002804D120464030007E002803D087498D4812F089
:202200009CFE0821A01D0FF04DFA00202071012060712B21E170207010BD70B57F4D044620
:202220002878002804D128464030007E002804D07E487949B83812F080FE7D481022214653
:20224000303800F0FCFB7A481022A118203800F0F6FB774830380FF02CFB754910221039C3
:202260002C46A81D00F0EBFB002020710E20A0702A20E07001206071207070BDF8B5674CB9
:2022800005462034A07B26462036002802D1307E002804D023206049400112F04EFEA97881
:2022A000052912D0132910D014290ED015290CD01A290AD0292908D03D2906D03B2904D002
:2022C0008D205549C00012F038FE28885A49884204D953485049E13812F02FFE09F00CF848
:2022E0000C212827022809D151482A888089904215D14A484838027E002A01D0E17310E081
:20230000A97841760121017637760020E07348484030407C002804D009F0ADFD01E00220CE
:20232000E07327740120A073F8BDF8B53B4F064638783D1D002804D138464030007E0028A8
:2023400004D03C483449D13012F0F7FD3146012008F0F8FB01242870002807D12F480622D2
:2023600060303146054612F04CFCAC717C711720F8703C70F8BDF0B52B4F85B0403F3D7A2D
:20238000064626480078002804D13846A038007E002804D0D3202049800012F0CEFD3078ED
:2023A000002806D0012804D022481B492C3812F0C4FD082D4CD21C4820380190C4693078B8
:2023C00000283FD0012804D01A4813491E3812F0B4FD294608310120884004430120A84021
:2023E00020430090B1790D4C08027279690009191043FF3101318881B01C12F063FC717813
:2024000000020843A9000919C031C862387A401C38720199009811E0B01B0000E0020020E1
:20242000520500002500002000040020E9060000D801002079030000FF0E0000C861002022
:20244000207108E029460831012088408443C5E7F748072101710121F5480B224171C270B6
:20246000017005B0F0BD10B5F14C2078002804D120464030007E002803D0EE49EE4812F034
:202480005CFD12F059FE00202071012060710A21E170207010BD10B509F09DFB002804D0BC
:2024A000E548E449583812F048FD08F043FA08F026F80AF040FE002804D0BD20DD498000E9
:2024C00012F03BFD08F085FA002804D05F20D949C00012F032FD12F02FFED84800240470D6
:2024E000FFF77FF9D2480121047141710222C270017010BD70B5CE4D04462878002804D150
:2025000028464030007E002804D0CB48C9498F3012F013FD20781F2801D8601C04D1C64856
:20252000C449903012F009FD002028712078611C08F022FB012068712021E970287070BD8A
:20254000F8B5BB4C0646207825464035002802D1287E002804D0B848B6499D3012F0EDFCAF
:202560003078012806D0002804D0F720B149800012F0E3FC012060710C20207130780027C8
:20258000AF4E012808D008F0B7FE032869D008F0B7FE032873D078E008F0AEFE002803D119
:2025A00008F0AEFE002804D008F0A6FE02283DD06BE008F04DFA002867D0287C002864D1BE
:2025C0009F4802210C300EF0F6FF002806D00F21B089090212F08FFBB18100E0B781012257
:2025E0000321974807F02EFE954808F0D3FBB08907F0A4FF002804D18F488E49B93012F0A9
:202600009CFCB089002108F09DF9002804D08A488849BD3012F091FC297F688B09F047FB49
:20262000002831D084488349C13017E008F068FE00282AD1287F002827D0012825D0042860
:2026400023D008F005FA00281FD0297F688B09F02EFB002818D078487649D53012F06DFCBD
:2026600012E0002009F056FA00280ED12771287C00280AD1B089FFF795F806E0FFE7002011
:2026800009F048FA002800D127711B20E07001202070F8BD70B5664D04462878002804D1BE
:2026A00028464030007E002804D063486149813012F043FC20781F2801D8601C04D10F2043
:2026C0005C49800112F039FC002028712078611C08F066FA012068711A21E970287070BD24
:2026E000F8B5534D044628780C272E46403600280AD1307E002807D108F0FEFD032803D0E4
:2027000008F0FEFD032804D14B484A49473012F014FC6079002801D0012829D1A0790028E1
:2027200001D0012824D1A07B002805D0012803D0022801D003281BD1607B400718D0628890
:2027400001208003824202D82188814201D920790CE02079002804D0022805D0032803D0DA
:2027600004E0202A12D20CE0A0290FD201280DD02079042805D12088202802D36188884298
:2027800004D92D482B495D3012F0D7FB20887083207930776079002802D0012803D00CE07C
:2027A000284A002105E0224A60329079002804D00121204608F050F9074601202F716871EE
:2027C0001821E9702870F8BD70B5194C05462078002804D120464030007E002803D0154903
:2027E000194812F0AAFB08F087FD0C2102280ED113482A8883899A4228D10246C032137F65
:20280000002B04D1807E0E2803D00F2801D0217103E005201077002020710E20A0702E204B
:20282000E0702888E08001206071207070BD0000E0020020B01B00003E0300000004002057
:20284000D801002025000020D30400000220E3E770B5814C05462078002804D120464030CF
:20286000007E002803D07D497D4812F066FB08F043FD0C2102280ED17A482A8883899A4227
:202880001FD10646C036327F002A04D1807E0E2803D00F2801D0217109E06F481022A91C1E
:2028A0001E3812F0AEF904203077002020710E20A0702D20E0702888E08001206071207030
:2028C000B4E70220F2E710B501780B0012F026FC3D878738878758878787873B3E878787E2
:2028E00051548787878787874228872C3087878787348787878787878746874A4E8720248B
:20290000876B5B5F6367876F877E827B77738700801CFFF79DFF60E0801CFFF755FF5CE048
:20292000801CFFF7DDFE58E0801CFFF7B3FE54E0801CFFF705FE50E0801CFFF7DBFD4CE020
:20294000FFF7A9FD49E0FFF78EFD46E0801CFFF712FD42E0801CFFF7E8FC3EE0801CFFF722
:202960008DFC3AE0801CFFF758FC36E0FFF73BFC33E0FFF712FC30E0801CFFF7D0FB2CE0FB
:20298000FFF7B1FB29E0801CFFF77BFB25E0801CFFF755FB21E0801CFFF70DFB1DE0801C69
:2029A000FFF7DBFA19E0801CFFF7B8FA15E0801CFFF76EFA11E0801CFFF725FA0DE0801CF5
:2029C000FFF7EFF909E0FFF7CAF906E0801CFFF79BF902E0801CFFF77AF9012010BD002076
:2029E00010BD10B51D49204812F0A7FA10BD70B5194A012411461B4D4031030012F08EFB9C
:202A000005191C1C04191C0001220021154807F019FC11480021483801774177C03809F05F
:202A2000C2F9002804D010480C49D33012F085FAFCE60C745565F9E608490C48F6E730B54C
:202A4000134606E0CC18203CE47FD51A44555B1EDBB2002BF6D130BDE0020020B01B00005A
:202A6000A7040000D8010020430600004907000010B56038030012F051FB0A060A0F131817
:202A80001F262A31363B086800F090FD10BD05C9114600F0AAFD10BD086800F044FE10BD73
:202AA00005C9114600F048FE10BD4B6808788A68194600F053FE10BD4B688A6808681946E8
:202AC00000F067FE10BD086800F07CFE10BD08884A6880B2114600F098FE10BD05C91146EA
:202AE00000F0C4FE10BD05C9114600F0FAFE10BD012010BD0120704701203F494006086060
:202B00003E4908603E490A68FF231B029A4383121A430A60384980390860704710B50246EF
:202B20000420384904E0C3005B181B79002B0AD00346401EC0B2002BF5D133A1432012F0FA
:202B4000FCF9FF2010BDC300CA50002259184A718A7101220A7110BD2A4A0021C000801816
:202B60000171704710B50446042803D326A1522012F0E3F92348E1000C182079012803D0FF
:202B800021A1532012F0D9F96079A179401CC0B2814200D060710120174940068031086027
:202BA00010BD70B5164800680004800F022803D015A1692012F0C1F9124E194C032520784D
:202BC000C10088190279012A07D1427983799A4203D042798271705880472078401CC0B20C
:202BE0002070042801D30020207028466D1EEDB20028E4D170BD000080E100E080E200E070
:202C000018E400E02C1200207372635C736F635F7369676E616C6C696E672E630000000079
:202C20003C00002010B5EFF31080C407E40F72B6D6484178491C41704078012801D10FF07C
:202C400021F9002C00D162B610BD70B5CF4CE07800280AD10125E570FFF7E4FF0FF01AF977
:202C6000002804D000200FF0EDF8002070BDC84865714560F9E770B5EFF31080C507ED0F3D
:202C800072B6C24C6078002803D1C2A18F2012F054F96078401E60706078002801D10FF0F2
:202CA000F5F8002D00D162B670BD10B5B748C178002904D000214171C170FFF7DCFF0020F5
:202CC00010BD10B504460FF0E5F8B049C978084000D001202060002010BDF8B50246AB4C70
:202CE0000026A6710820042101251027130012F015FA0D080A0C0E101214161E2621232597
:202D00002800257122E0022001E021711EE020711CE027711AE02020F9E7012616E0FFF70E
:202D200081FF0FF0B7F80028FBD002260EE02171A5710BE02771FBE7202000E0402020713E
:202D4000F6E7FF2093A17E3012F0F7F80FF0AEF8002809D00FF0B0F8B04205D130460FF01A
:202D6000AEF80028FAD024E001208007C5608D4A002151608C4A9661854B02225A608560E1
:202D80008A4803690569DB43DB06DB175B1C10273D430561834D00E020BF6F68002FFBD0A2
:202DA000002B03D1076910239F430761784882606960A07900280CD00FF06CF805460EF0F3
:202DC000C9FF7B4A002D02D0A260E06001E0E260A060002E01D100F0B1F8F8BD10B50446A5
:202DE0000FF05EF8002805D068490120C8704A78521C4A702046FFF770FF10BDF8B5694F90
:202E0000B8680025012802D1BD600FF01BF87868012800D17D60386801265C4C012814D10E
:202E20003D606079002803D000200FF00BF865712078002809D00FF02DF8002805D05948CE
:202E4000C038866300060661A670386901282CD13D6100F068F8012080074661A0790028C9
:202E600015D00FF017F800900EF074FF0099002901D0E16800E0A168411A022901DA8A1C92
:202E800013DC0099002901D0E06000E0A060FFF7C9FE0EF0FFFF002806D04248C03886636E
:202EA00000060661A67000E02670F868012819D100F039F800F037F800F035F8A078002809
:202EC00004D1FF2033A1053012F037F8FD60A5702570FFF7D0FE0EF0B4FA002802D03148DA
:202EE000C038C663F8BD10B5284CE078002801D10EF0CCFF01208107886100F014F8A07802
:202F000000280BD0274CE068002803D10EF0D7FF0028F8D10020E06000F005F800201C4960
:202F2000C043886010BD08B55020694608806A461088411E11800028F9D108BDF8B514487D
:202F400019278760174900200860C8600EF0A2FFBD0701240D4E002805D01248C038846321
:202F60002C61B47000E03470FFF75CFE084847600D4930798863FFF7D6FFAC61FFF7D3FF4B
:202F80000849002008616C61F8BD000040000020000300407372635C736F635F636C6F6349
:202FA0006B2E6300000100400005004000ED00E0FFFFFF7F10B510F020F810BD002004492F
:202FC000C863012001218140024A116000BF7047C01F004080E200E010B504460BF051F8DB
:202FE00020460CF066F810BD704770477047704770477047704770477047704770477047B0
:2030000010FFFFFFDBE5B151006001005A00FFFF03B40148019001BD09000020FE494870B1
:20302000704710B5030012F079F8080E050E08080B0B0E1104F06BF810BDFFF7CDFF10BD7D
:203040000DF0A0FF10BD01F077FE10BDFF20F3A19A3011F072FF10BD7FB5F44905464868AC
:203060008968082301910090F14A1946F1480EF043FD0024F0480EF05DFD641CE4B2082C03
:20308000F8D3EB490320803140020CF0E7F8002803D0E2A1BF2011F050FF1E220221E74801
:2030A0000AF09FFCE5481E22032110300BF013FAE2480722342174300AF0ECFBDF484C21E1
:2030C000283011F0FDFDDD496A46743108464C380164FF317B31416401211172039002F040
:2030E000AAF802A80CF008FC002803D0CBA1D32011F023FFCF4802222421A8380AF0CAFBE8
:20310000CC4802222C215C380AF0C4FBCC490B200EF03AF8002803D0C0A1E02011F00DFF04
:2031200003F0DEFF03F0E2F904F03EFE6B4600220821C4A001F06EFF002803D0B7A1E720A9
:2031400011F0FBFE284605F049F9002803D0B3A1E92011F0F2FE8521C900BD4811F0B0FD65
:20316000BB49B24A0020135C0C18401CC0B2E3700428F8D3A849002048608870C8707FBD5F
:2031800070B5B44E0546706A94B00C46401C04D1B06AC0430004000C0BD0306AC007C00FE4
:2031A0002870706A11F09FFDB06A2071000A607114E02B206946087009A968460AF0B0FB0F
:2031C000002804D0FF2095A10E3011F0B6FE0120287006220AA9204611F013FD28780028D8
:2031E00003D06079C0210843607114B070BDF0B5984C0646206895B00D463746401C083728
:20320000002808D16068401C05D1A068401C02D1E068401C11D02068314611F064FD6068CE
:20322000311D11F060FDA068394611F05CFDE06831460C3111F057FD25E02B206946087039
:2032400009A968460AF06CFB002804D0FF2073A1373011F072FE08220AA9304611F0D1FC85
:203260002B206946087009A968460AF059FB002804D0FF2069A13E3011F05FFE08220AA960
:20328000384611F0BEFC20692E46401C0836002808D16069401C05D1A069401C02D1E069E1
:2032A000401C12D02069294611F01DFD6069291D11F019FDA069314611F015FDE06929464C
:2032C0000C3111F010FD15B0F0BD2B246846047009A90AF025FB002804D0FF204FA15C305D
:2032E00011F02BFE082209AF0AA9284611F089FC6846047009A90AF013FB002804D0FF2024
:2033000046A1633011F019FE0822391D304611F078FCD8E710B5002108460EF0C3FC0021DF
:2033200001200EF0BFFC002102200EF0BBFC002103200EF0B7FC002104200EF0B3FC0021B3
:2033400005200EF0AFFC10BD10B5414CA0780B2804D3FF2031A1B33011F0EFFD2078602184
:20336000484300190830002101704178E722C908C900C91C11404170274A0121917010BD3B
:2033800070B5254CA07800280ED0314800250178491CC9B201700B2900D105708178491C39
:2033A00081700EF04AFDA57070BD70B51A4C05466068002804D0FF2018A1DC3011F0BDFD5C
:2033C000656070BD70B5144E214DFFF7BDFF71680446002907D06022FDF7F6FEFFF7D0FF02
:2033E00000207060F1E72879002876D011485C380AF060FA6060002804D1FF2007A1FA3007
:2034000011F09BFD60680AF0B3FA002831D0204600F03FFF60781FE0340000207372635C18
:20342000686F73745F636F72652E630048510100040400200C12002023300000840A002034
:20344000B41000206E52463531383232000000008C0C002080000010010707D5C008C000CC
:20346000401C60702879401E287127E0F74861682AE0F64861680AF026FA687900282CD049
:20348000F2484C380AF016FA6060002804D18720EF49800011F051FD60680AF06DFA0028A8
:2034A00016D0204603F072FE6078010709D5C008C000801C60706879401E6871FFF760FF3E
:2034C00083E7E24861684C380AF0FDF97DE704E0DE4861684C380AF0F6F970BDF7B5054653
:2034E0000078002700090C463E46062803D0D849D84811F022FD287A00280ED0012814D037
:20350000D448D349213011F018FD0298002C068001D0278066800020FEBD02270926002C03
:203520000ED0A889A080A87B08E003271426002C06D02869E060A88A2082287B2072E4E746
:2035400002980680E7E770B50E4600211C4619801546030011F0E2FD0723050B1711231D08
:20356000230022462946304603F0DCFD70BD22462946304601F051F970BD224629463046E0
:2035800004F00DFB70BD22462946304602F0E2FF70BD224629463046FFF7A0FF70BDAD48B1
:2035A000AB49473011F0C9FC032070BD10B5AA4C2178002901D0082010BDFFF74DFD0120E6
:2035C0002070002010BD0146A04810B54C380AF07AF9A2494879401CC0B24871012803D159
:2035E0009D484078FFF7BEFA10BDF8B505469C480F46814208D3002D01D0854204D3E81C44
:2036000080088000A84201D01020F8BD93488178002911D0398800914178602251430C18DF
:20362000083420783B460007000F00222146FFF78AFF060004D015E0002038800520F8BD96
:20364000002D13D039880098814201D90C260DE020783B460007000F2A462146FFF773FFD7
:20366000060005D00C2E01D0002038803046F8BD7A4D6878401CC0B268700B2801D10020EF
:203680006870A878401EA87061784807400F022810D00128EAD16D4861680AF014F9287931
:2036A000401CC0B228710128E0D16B484078FFF759FADBE7C806D9D46068FFF784FFD5E7DB
:2036C00070B50446674816460D46814204D161485F49C53011F031FC012E05D05D485C49C3
:2036E000D53011F02AFC70BD5B480121C1706620207000202072A581A17370BD70B51646CB
:203700000D46040001D1FFF71FFE662101700121017229680161A98881820673002C01D142
:20372000FFF72EFE70BD4E49884201D21020704707210170002070474B4A10B5904208D3A8
:203740000124A404464AA04201D3904201D3914201D2102010BD0DF050FD10BD424B10B5A4
:20376000994208D30124A4043D4BA14201D3994201D39A4201D2102010BD022803D01028F7
:2037800001D0092010BD0DF05EFD0028FAD0052010BD354B10B598420CD30124A404304BE0
:2037A000A04201D3984205D3994203D3002A03D09A4201D2102010BD0DF06BFD0028FAD0F0
:2037C000072010BD10B50446254894B0844202D2102014B010BD01F09AFD002801D0112028
:2037E000F7E70F2008A9087369460BA80AF098F80028EED16846007A2070684640896080AE
:2038000068468089A0800020E3E710B5124C0846E17800290ED000280AD0114A904202D312
:203820000368934201D2102010BD8288002A03D0012903D0082010BD092010BD04F018FB82
:203840000028FAD10021E17010BD0000B01100201C3400003E020000340000208C0C0020B9
:2038600000200020FFFF00000060010010B5244A94B091420DD301229204224B914201D3B2
:20388000994206D3441E1E2C24D8914203D3994201D210209DE701281AD108780024C00742
:2038A000C00F002803D001206946887001E06846847039206946087009A968460AF030F8F1
:2038C000002803D010498C2011F037FB204680E707207EE70246203A1F2AF9D801F03AFC79
:2038E00077E7084A10B5914201D21020ACE70246203A1F2A02D801F083FCA5E70720A3E778
:2039000000600100002000201C3400008107C90E002808DA0007000F083880082C4A800079
:203920008018C06904E080082A4A800080180068C8400006800F704710B50D20FFF7E6FF45
:20394000C4B20420C043FFF7E1FFC0B2844203D021A11A2011F0F1FA10BD0121234A48035A
:203960001060234B00221A60224A5160224A1060224A11601D4980390860704701211B4A32
:20398000480310601D4A5160194A002111601A490860704710B516490868012804D00EA19D
:2039A000562011F0CAFA10BD154880680022C0B20A600DF09DFE10BD10B50D4801680029AB
:2039C000FCD0FFF7E7FF01200B494003086010BD00ED00E000E400E07372635C736F635F79
:2039E00068616C5F726E672E6300000080E100E000D1004000D3004080E200E000D00040A4
:203A000000D5004030B40121BC48C9020160CD1005604A030260BA4803681B021B0A036058
:203A200004680023240A24020460B6480468240A24020460B448012444608460B34C2360F2
:203A40006360A360B24B19601D601A60B14B19601A600121016030BC704710B40121A74849
:203A6000CC0204600A0202600B060360A64841608160A6490020086048608860A44804606B
:203A80000260036010BC70470121A148C9020160C91001607047002805D0012805D0022891
:203AA00005D19D4870479D4870479D48704710B59CA18B2011F041FA002010BD70B5002140
:203AC0009F4CA04DA04A914B002808D001281DD0022822D093A1B32011F02FFA70BD012097
:203AE0000004A060A86011601960984B42109A60974A9060814A0012106096480160874875
:203B00000160954801609548017070BD01204004A060A8605160596070BD01208004A060E2
:203B2000A8609160996070BDF8B59446844A854D00240127754E002808D0012836D00228D7
:203B400044D078A1E82011F0F8F9F8BD891E0902090A012000049060346068607A4A11601E
:203B6000012B21D000217D4A7D4B517061463D31DC63DF637B4B5C6002249C6004241C61D8
:203B8000744B196074490F60614B89151960704B58606048016075487349C16086606B494E
:203BA000600348601770F8BD0121DCE701205C4E40046F4F012B04D1346050606860396066
:203BC000F8BD9060346068603960F8BD0120524E8004684F012BF4D1EEE7674840687047C6
:203BE00070B54A4D28680026554C012806D1A068C00303D501200004A0602E606868012863
:203C000009D1A068800306D501204004A0606E6001200FF02EF9A868012809D1A06840038C
:203C200006D501208004A060AE6002200FF021F970BD10B549490878002818D00120434AF9
:203C4000C0039060424A400090602C4A00121060404A00201060314A10603F4A1060087087
:203C60004A78002A02D048700FF003F910BD0320FAE70120414900060860704701202449A4
:203C800000060860704701203C4940050860704701201F4940050860704731490020C86343
:203CA00088151B4908607047410A354AC005C00D5043801C5143400A0818704710B4314C63
:203CC000430B63431B0C5C020C602D4C6343C31A2D485C0258432A4B400D4343E31A01242B
:203CE000DB0324041B191B1613700A681018086010BC704710B50FF094F910BD80E100E0F2
:203D000008E400E018E400E000B0004040B1004080E200E000E100E048B10040408100409D
:203D200044B100407372635C72656D5F68616C5F6576656E745F74696D65722E6300000040
:203D400000B3004040B3004040B5004000F5014000830040408500400082004050000020D8
:203D6000C08F0040008500400080004080F5014044B5004048B5004000B5004000E200E04C
:203D8000093D0000378600006F0C01000E4A12680C498A420AD118470B4A1268094B9A4278
:203DA00004D101B50DF0BFFD03BC8E46074909680958084706480749054A064B70470000C6
:203DC00000000000BEBAFECA1C01002004000020881D0020881D002010B5F84C94B02168E2
:203DE000087A002836D017206A46107000A806220931023010F005FF09A9684609F090FD86
:203E0000112825D02168C0318979062920D007291ED008291CD004291AD0092918D00A293A
:203E200016D00B2914D0052912D0002803D0E4A1F42011F082F82168B820405806221C30F8
:203E4000093110F0DEFE2068017A8030806BC17614B010BD3220C7E770B5D84D04462968C1
:203E60000300C03111F05AF90C077C0B1A212E3B48515C677080FF20D1A10A306EE0887956
:203E800001286DD009286BD0052869D00A2867D00B2865D0FF20CAA10F305FE088790128E7
:203EA0005ED0FF20C6A1163058E08879062857D0072855D0082853D0052851D0FF20C0A105
:203EC00019304BE0887909284AD00A2848D00B2846D0042844D0FF20B9A11F303EE0887968
:203EE00003283DD007283BD0082839D0092837D0FF20B3A1253031E08879062830D00A28A5
:203F00002ED0FF20AEA12B3028E08879062827D0072825D00B2823D0FF20A9A12F301DE09D
:203F2000887906281CD00A281AD00B2818D0FF20A3A1343012E08879092811D00A280FD052
:203F4000FF209FA1393009E08879092808D00A2806D0082804D0FF2099A13D3010F0EDFFE8
:203F60002868C030847170BDFF2095A14230F5E79249C9220968525CD206920F05D1A031F7
:203F80008A8B824201D1887F70470020704770B50446112020700021884D61702968C03168
:203FA000897A002908D003290ED0042910D0FF2083A16B3010F0C1FF20780009012802D9A3
:203FC0002868807D607070BD0007000F203002E00007000F30302070EEE730B503887C49FF
:203FE0007C4C8B4202D09A1FA2421ED242888A4202D0951FA54218D2934216D883887D2471
:20400000E400A34211D8C088884205D0714D04460A3C2D1FAC4208D2884208D08A4206D061
:204020005B1C5A43C000824201DD072030BD002030BDFFB50022099B002802D0994205DCB9
:204040005CE0002902D1002004B0F0BD0920FBE7845C002C12D085186F780D2F4CD010DCE6
:204060003B0011F05BF80A421B2A2A303032323A3A42835C002B3FD1521CD2B28A42F8DBD1
:20408000E1E7122F31D004DC0E2F35D00F2F2CD132E0142F11D0152F27D116E0022CD5D17D
:2040A000AB78039C072B237001D25B0701D40A20CAE7029B01241B7814E0E343DB0708E05B
:2040C000012C08D011E00620BEE70F2523072D075B19002BF4D03046B6E7029B1B789C0744
:2040E0000AD402242343029C2370835C521C9A18D2B28A4204DDA9E70B20A5E719267602F7
:204100008A42A5DB9FE705E00278401C002A01D0002070470A46491E89B2002AF4D101203E
:20412000704770B5254D00212868C943A030818300248477214606200DF0B4FD0021052000
:204140000DF0B0FD002102200DF0ACFD0120FFF783FE2868C030C471047201F062FF70BD8A
:2041600030B5164C95B02268C0329279042A0CD0052A0AD028236A4613705080132906D0B9
:204180003B2904D0072015B030BD0820FBE71171104609A909F0C4FB05000BD12068C03069
:2041A0008179062908D0082906D0072904D00520FFF752FE2846E6E70420F9E754000020D5
:2041C0007372635C6761705F636F72652E630000FFFF00007B0C000030B587B0040003D0F2
:2041E000002107200DF05EFDF74D012128686A4601720421117003210C300DF053FA296825
:204200004022887B8006800E1043887368460BF094FB00280DD12968098A00290AD0002C46
:2042200008D08B000122002107200DF096FC072802D0032007B030BD0020FBE770B500250D
:204240000646002803D0002107200DF02BFDDE4C012120680172062109300DF023FA206861
:20426000817B8906890E8173FFF7B6FD2068008A00280AD0002E08D0830001220021072077
:204280000DF06BFC072802D00325284670BD0025FBE7F0B59BB0040003D1CC49CC4810F0FE
:2042A0004CFE72202070616800260A780825521F0127C548130010F031FF0F097CDFFD7C1F
:2042C0007EFCFBBB7C7C7C7CFAF97C00BE480068C0308079032804D0BD48BC49093010F0B6
:2042E0002CFE002108460DF0DDFC002107200DF0D9FC6078B44A2843607010681025014630
:20430000C0314B7A2B434B7263689D783C2D4DD002469D88A032977763688030DB890B809F
:2043200063681B8A4B8063685B8A8B8095836168826BC97911756168806B08311530062297
:2043400010F05FFC0620FFF787FD9F48FB2300680146C0318E72027E1A400276B822125827
:20436000937A9B089B0093724682487A4006400E4872284602F0C0FE002804D09448934943
:20438000243010F0DAFD284602F0D0F8002804D08F488E49273010F0D0FD284603F016FD88
:2043A000002806D08A48894929303EE10120FFF753FD1BB0F0BD074600688E88C030807950
:2043C000062812D0072810D008280ED004280CD009280AD00A2808D00B2806D0052804D089
:2043E0007B487A49353010F0A8FD6078284360703868C030417A294341728079092811D0A5
:204400000A280FD00B280DD005280BD0FFF789FE304602F07AFE304602F08EF8304603F0BF
:204420000BFDC6E7FFF77DFE0220FFF715FDEFE70068C0308079062812D0072810D00828B6
:204440000ED004280CD009280AD00A2808D00B2806D0052804D05E485C49593010F06DFD19
:204460006068807902F004FF0028A2D06178294361706168C8809CE707460068C0308079A4
:20448000062812D0072810D008280ED004280CD009280AD00A2808D00B2806D0052804D0C8
:2044A0004B484A496C3010F048FD04E037E1A1E190E090E015E06078284360706068C1887E
:2044C0003868C0300180616809894180616849898180002102200DF0E5FB3868C030C6712C
:2044E00067E706460068C0308079062819D0072817D0082815D0042893D0092811D00A28BC
:204500000FD00B280DD005288BD031482F49833010F013FD3068C03080790428ABD005281B
:20452000A9D03068807C40063AD5606802210C30FFF7E9FD002833D060680821001DFFF7E7
:20454000E2FD00282CD03168B8204058807A800708D1CA20405C002808D1488AC20505D5FB
:20456000C00703D1488A4022904348824A8A802082434A822D2268460270BC20425A684635
:2045800042801022973101A810F03BFB09A9684609F0C6F90028A3D03D200C49000144E0F6
:2045A00062683068AC2192890A5261680822091DAE3010F026FB10A805743068AE301590F1
:2045C00014A80BF0BAF9F4E654000020C0410000260300008F7106460068C030817906292C
:2045E00019D0072917D0082915D00429EBD0092911D00A290FD00B290DD00529E3D0FD2089
:20460000FA49800010F099FC3068C03080790428D9D00528D7D060688179002902D0807863
:20462000002805D02320F149400110F086FCC0E66078B8212843607030680958897A89071F
:20464000890F012951D1817C09064ED4017E490701D5042100E00321C03081722B2069469D
:20466000087009A9684609F05BF9002803D0DF49DF4810F062FC68463168008D88820E225F
:2046800010A80274DB48B82215905258083242610A4660324260927902700A4614320261C9
:2046A000521D82601032C260133A82619632C261921C0262473A4262103282621032C26267
:2046C000473AC263521E0264921F50314264816414A80CF01BFB022815D0002813D0C448AD
:2046E000C249293010F029FC0DE0817C4906017E490701D5042100E00321C0308172002126
:2047000006200DF0CFFA3068418A0A0602D440229143418289B280229143418249E6B648CA
:204720000068C0308079032804D0B148AF49573010F003FC002108460DF0B4FA0021072050
:204740000DF0B0FA6078AC4A28436070106810250146C0314B7A2B434B7263689D783C2D8B
:2047600000D123E602469D88A032977763688030DB890B8063681B8A4B8063685B8A8B80B2
:2047800095836168826BC97911756168806B08311530062210F035FA0620FFF75DFB9648A8
:2047A000FB2301680A46C0329672087E184008764E82507A4006400E5072284602F09CFCE4
:2047C000002804D08A488949723010F0B6FB284601F0ACFE002804D085488449753010F0A2
:2047E000ACFB284603F0F2FA002897D080487F4977301AE7607828436070DAE500290BD028
:2048000088807D480068C0300288CA8002880A8142884A81808888817047F7B506460078BD
:204820000C460027010982B03D46012974D0724800680090C03002296FD0072904D00A298F
:204840006CD06A496D480DE271680A78521F130010F064FC0F09A451A4A42F585847A4A4C3
:20486000A4A4656FA4008A783C2A1BD010271625002C7DD08888A0807068A21DC089208288
:204880007068C089E0817068008A60827068408AA082716808460831C07901F0B1FB002038
:2048A000607375E019270725002CE2D00021A17171E011270725002CDBD089880091A18004
:2048C0007168F7228979A171417A11404172009802F01CFC009801F033FE009803F0BAFA78
:2048E000D2E101270925002CC3D08888A080706880792072C8E1888812270E252146FFF7DB
:204900007DFFC1E118270825002CB2D08888A080A01DFFF73CFBB7E144E0A6E15CE01A2785
:204920000725002CA5D04888A08070680079A071AAE18A783C2AB5D010271625002C98D0DA
:204940008888A0807068C08920827068C089E0817068008A60827068408AA0827168607B26
:20496000497D40084000C907C90F0843607300E093E17168C007497DC00F490849000843B5
:2049800060737168A21D08460831C07901F038FB19480068C030417AEF2273E1A7201349CC
:2049A000C0005FE1307A012803D014480F49C83858E112270E2570892146FFF71FFF002C58
:2049C00092D070784007400F032889D10A480068C030417AFB2255E107490968A031002CFC
:2049E00001D08A8BA280327A921E09E0C041000015040000AC1200205400002017060000E1
:204A0000130010F08BFB073D4853FDEB6F05FD0013270C25002C85D0009900224A82F168F9
:204A200089788907890F0129217A26D0490849002172FD231940F3689B785B07DB0F5B00D7
:204A400019432172E323E2801940F3681B785B07DB0E19432172DF231940F3685B78DB0713
:204A60009B0E194321726272F1680122C978A172017A1143F7221140ADE001231943D7E7F6
:204A800015270C25002C9BD0F06806220068A11D0EF05CFFF8E016270725002C90D0317B9A
:204AA000A171017A08221BE00172EDE014271225002C85D00098A21D8030806B0146153192
:204AC000007D01F09DFAB089E081207C01210843F92108402074FD480068C030017A0222FC
:204AE0001143E1E717273825002C94D03221A01D10F0E4F80020A071207A032108432072B7
:204B0000FB210840F14909680A7E5207D20F920010432072B8204058807A800757D0A07A1B
:204B20008A7C4008D2074000D20F1043FD221040A0728B7CFB229B07DB0F10409B00184363
:204B4000A0728B7CF7269B07DB0F3040DB001843EF231840A072E07A10408A7CD206D20F08
:204B600092001043E0728A7C3040D206D20FD2001043E072888AA0812046102267310E30B7
:204B800010F03FF8D149A07F0968C0078A7DC00F52001043A0770A7E400852074000D20F91
:204BA0001043A077084640304DC820344DC4303C3F20405C22463032393101F021FAC348A1
:204BC00000688030806B817A890889008172BF480068C030017AFB22114065E7327B022A5D
:204BE00018D017273825002C11D0017AFB2319400172012A17D0032A22D0042A23D000E08E
:204C00002DE0052A1FD0B249B24810F096F901F008FA39E019270725002CF8D0898BA18044
:204C20000121A17103E00121A1710021E171417ACA094906D201890E49000A434272E6E758
:204C40000220A07106E0707B0007000F8030A071052A02D00020E071D9E70120FBE79D485F
:204C60009B490C3010F069F90EE0317A00290BD119270725002C10D0491EA1800021A171E1
:204C8000417AFD22114041720498002C058001D027806580002005B0F0BD04980580F9E709
:204CA00010B58A4C94B02068C0308079022809D0032807D0052805D0092803D00A2801D096
:204CC0000B2837D11B2108A801730021817369460BA808F025FE002804D1684640781B2801
:204CE00002D0032014B010BD002108460CF0DAFF002107200CF0D6FF68468078002819D119
:204D00002068C0308079801E030010F007FA0A060613081313130D0F1113012000E00420B1
:204D2000FFF79AF80020DDE70620F9E70720F7E70820F5E70820D5E770B50025634C0028F3
:204D400007D0022817D0072828D062486049793046E0FFF7A5FF00280CD1FEF7F5FA22215C
:204D600001700572FEF70CFB2068C030417A02221143417270BDFEF7E7FA12210170012128
:204D800001722168BC22525A4281C031CD71FEF7F7FA2068C030417A0422E9E72168C6201D
:204DA000405C022809D0032807D0092805D00A2803D00B2801D00528DCD1887B81090129B2
:204DC00011D0800904D043484149703010F0B5F80020FFF733FA0028CCD03E483C4974307D
:204DE00010F0ABF870BD0020FFF7F6F9F3E770B50D46040004D137483549813010F09DF870
:204E00002078012805D0334831499F3010F095F870BDA18830482D4E814209D1E288824297
:204E200006D130681321A030808BFFF799F970BD814202D1E08800280AD012202870687895
:204E400008210843687007CC083507C5002106E000227823114602200CF07FFE02213068B9
:204E6000C030C17170BD00B5184A87B01268C032527AD20907D106236A461370019011723A
:204E800068460AF05AFD07B000BD00B587B007206946087068460AF050FDF4E70B480068DA
:204EA000C030807A704738B5084C05460278206813000146C03110F031F909A9061111A3D1
:204EC000204E738BA900FEF787FF38BD54000020C0410000F2050000FFFF000088790628B4
:204EE00005D0092803D0FE49FE4810F026F820680422017E1143017682E0A9880029E4D0C6
:204F0000A030808BF8498842DFD0A868002804D1F448F349103010F010F82068C030407AFD
:204F2000C00904D0EF48EE49113010F006F8A86806220A38A86000902068AB88A030808B7F
:204F4000042102F00DF80028BFD0DB20E449C0000FF0F3FFB9E788790528B6D9287901287E
:204F600002D0022808D103E0487A802210434872487A012210434872284601F05CF82068DB
:204F8000C03080790628A0D9082801D8062004E009289AD90B2898D80920FEF75DFF94E732
:204FA000887906280AD0042808D0092806D0052804D0CC48CA493D300FF0BFFF0ECDCB489D
:204FC0000361C2608160A2210170FEF7EEF97CE78879062818D0072816D009280DD00A288B
:204FE0000BD0C048BE4950300FF0A7FF2068C0308079062808D0072806D00B20FEF72CFFDB
:20500000284601F018F860E70820F7E7B548B44964309DE7FFB593B00124684603218470E0
:20502000C9021D4601800AF060F900226946012003F085F906460AF05CF9002E5CD1684667
:20504000152184704902018000271C2101A808970FF036FE01200146103108A80170002091
:20506000014608A841708178F9200140891C214308A88170684601790226314301711499A8
:205080008185C7851F21018608A80A9013980D90684609900AF029F90EAA09A901A802F0FD
:2050A0001CFF07460AF025F9002F02D0384617B0F0BD8F4F68463968008F48806846847057
:2050C0008C49018008A88078F9210840801C4108490008A8817068468685068615A80D9002
:2050E0000AF003F90EAA09A901A802F0F6FE06460AF0FFF8002E01D03046D8E76846396801
:20510000008F88807B4968468470C91C0180298810A8018069884180A9888180E988C180AC
:20512000082168468185018610A80D900AF0DDF80EAA09A901A802F0D0FE04460AF0D9F8FF
:20514000002C01D02046B2E768463968008FC8800020ACE7F0B5684E95B00C46B14235D38D
:205160000127BF04654DBC4201D3AC422ED3202804D0212824D0222837D13DE03C216846FE
:205180000170218841806188818009A908F0C8FB002806D108A98979002904D002290DD026
:2051A000032015B0F0BD6168B142FAD3B94201D3A942F6D36A46128D0A80F2E75048F0E72D
:2051C00008684B4C002812D0A84201D21020E8E706210EF0A5FB411C07D02168A822505016
:2051E0000120A03188750020DBE70720D9E720680021A0308175F6E7084600F028FFD0E78F
:205200003D4A10B5914206D301229204914204D33A4A914201D2102010BD202805D02128A6
:2052200003D0222803D0072010BD062010BD084600F042FF10BD70B504462C48CC21AC309F
:205240000FF03EFD29482A4EAC3000213060C943A0308183002585770120FEF7FDFD3068F5
:20526000C7210D54E121C57389000182B6210D54014609310830FDF783FF316808460A7ACD
:2052800060308271062209310FF0BBFC3168084629311930FDF7ABFF002C37D030688030D0
:2052A0008463FEF799FD1E20E081607A8F21084030306072306801461431216198316162A7
:2052C000933921601031616025721339A162091FE1628531E163303921631031616311E051
:2052E000C0410000C2060000FFFF00004C12002054000020012A0000006001000020002029
:205300000230000010310930A163A06470BDF7480068C0308079042803D0052801D00020FF
:2053200070470120704770B50646F1480C46814206D301208004844204D3EE48844201D235
:20534000102070BDFFF7E3FF002801D0112070BDE948E64D002E02D0012E46D12FE022786E
:20536000002A0AD00121012A09D0022A14D0032AEDD1A2799209EAD112E0002103E0A27986
:205380009209032AE3D128680622017260308171611C0FF036FC05E0A2799209012AD6D1C9
:2053A00028680172002107200CF07CFC28680622611C09300FF025FCFEF70EFD11E0217816
:2053C000002912D0012910D0022910D00329BED10120FEF733FF002803D0C849C8480FF08F
:2053E000ACFD2868C673002070BD072070BD0120FEF7F2FEEFE7BF4910B5884201D2102024
:2054000010BDBA49024609680B7A0931184600F0F7FD002010BDFFB599B0054600206946FE
:205420000871087208A90874144608750122B0499204B0481E46002D05D08D420BD39542E1
:2054400001D3854207D3002C08D08C4203D3944204D3844202D210201DB0F0BD284620436D
:2054600018D01F270CAB01AA009728461A99FEF7E0FD0028F0D10DAB02AA31462046009751
:20548000FEF7D7FD0028E7D16846007AC10703D00A20E1E70720DFE7800705D56846007939
:2054A000800701D50B20D7E7FFF731FF002801D01120D1E703AF002D0FD01A20694608737C
:2054C0001A9888732946F81C1A9A0FF09AFB0EA903A808F025FA0028BED1002C0ED02021D9
:2054E00068460173867332462146F81C0FF089FB0EA903A808F014FA0028ADD17B4908A899
:205500000968007C08700020A6E7F0B504467848002695B0844276D301208004844202D310
:2055200074488442F7D32378012B09D1704960688842F0D39904884202D36E498842EAD3F6
:205540006A490A681546C035A879022814D0032812D0052810D009280ED00A280CD00B283D
:205560000AD0012803D0002B06D0012B04D0687AC506AD0F06D101E0082012E6850701D4B2
:20558000400701D511200CE6208A5E4F0546203DBD4207D3012B6ED10028FCD1658A002D77
:2055A000F9D111E0022B01D0032B01D1A02862D3012B01D1002807D01578ED0704D0658AF4
:2055C000002D58D0B42D56D8002B06D0012B08D0022B04D0032BDED118E0002519E0022547
:2055E00017E0002802D1608A00280DD004256068007800280DD001280AD0022808D003282C
:2056000006D03D48CDE563E00125F0E7032500E00126D07B01281CD1108A002819D0907BF7
:205620008109012911D0800904D035483349EC300FF083FC0120FEF701FE00280BD0304855
:205640002E49F0300FF079FC05E00120FEF7C4FDF3E7FEF7C1FB207A002806D0012806D061
:20566000022806D0032806D106E0002705E0012703E0022701E087E00327002D01D0022D63
:2056800048D1002F46D0E06800287DD00179002920D0082978D8027B082A75D800290AD0DC
:2056A000134B0168994213D301239B04994202D3104B99420CD3002A10D080680C498842C9
:2056C00006D301218904884208D30A49884205D2102066E5027B002A6AD0DCE703480068D7
:2056E0000078800710D00448401E5AE554000020006001000020002002320000C041000098
:2057000086080000E13F0000022D03D1022F4FD0032F4DD0182168460170218A4180218ACA
:2057200081808571FE480068007A002801D001287ED16946C87168460672217809300129CF
:2057400023D006210FF0BAFA07216846C173077409A908F0E5F80028BBD10A20694608706B
:2057600009A9684608F0DCF80028B2D13A206946087009A9684608F0D3F80028A9D1002DDF
:2057800009D0022D07D04CE012E061680622491C0FF037FAD8E7002F43D00026374623E0DF
:2057A0000168B00009580978002903D0012904D00720F6E469468F7002E001216A46917090
:2057C000E16806220968095800A8491C03300FF018FA0B206946087009A9684608F0A0F8F3
:2057E0000028E6D1761CF6B2E0680179B142D7D800266F4611E08068B10041581022B81C28
:205800000FF0FFF93B206946087009A9684608F087F80028CDD1761CF6B2E068017BB14281
:20582000E9D81B20694608700120887009A900E036E0684608F074F80028BAD108A8407956
:205840001B282DD12B000FF069FC0504040606041E00032015E0B2480068C03080790300D7
:205860000FF05CFC091E061E1E0A1E080C0E1E00022006E0092004E0052002E00A2000E0DA
:205880000B20FEF7E9FA012D0CD0608A002809D000228300114610460CF05FF9002801D071
:2058A00003207EE400207CE470B586B00C00064609D09C48844248D301208004844202D352
:2058C0009948844241D3964D2868C030C179022902D0407A400702D5112006B070BD002C5B
:2058E00004D02046FEF779FB0028F6D13046FEF73FFB012803D0022823D08C48EDE721008F
:205900001BD1082069468882286801ABC08805AA002103F0F7F80028DFD16846808A0828C4
:2059200001D00320D9E7684681888181C188C181018901824189418203A9304601F068FC5E
:20594000CBE7002C01D00620C7E71020C5E770B50C460546FEF70CFB012803D0022801D033
:20596000724870BD21462846FEF7FAFB70BD00B50146143095B0192801D2880707D0084607
:205980001E3004D00A3002D0072015B000BDFFF7BEFC002801D01120F7E761483122006814
:2059A000417068460270817009A907F0B9FFECE701B582B0022069460880594802AB0068FA
:2059C0006A468088002102F00DFF69460988022900D003200EBD38B502216A4611805249DB
:2059E000884201D2102038BD4D49034609688C880021204603F086F8694609880229F2D05C
:205A0000032038BD3EB504460820694608804548844206D301208004844204D34248844214
:205A200001D210203EBD2046FEF7D7FA0028F9D12088694688806088C880A0880881E088A2
:205A40004881374801AB00686A46C088002102F0C9FE694609880829E4D003203EBD1FB501
:205A600004460820694688812E48844206D301208004844205D32C48844202D2102004B0B2
:205A800010BD27480B46006803AAC088002103F039F80028F3D169468989082901D0032005
:205AA000EDE769460988218069464988618069468988A1806946C988E180E0E7FEB50E46C0
:205AC0001849174605468E4206D3012292041648964203D3864201D21020FEBD1F2F01D9A1
:205AE0000C20FEBD0E4C8D4232D3954201D385422ED3206801A9408802F026FE0028F0D125
:205B0000287869464871206801A9408802F0FFFD0028E6D16946009008780221084307E0A2
:205B200054000020006001000020002002300000694608704979090703D00821084369462F
:205B4000087020686946408802F08BFD0028C8D169460F8120683346408802AA002102F0CC
:205B600041FE69460989B942BBD00320FEBD38B50C46F749002801D0884201D38C4201D28A
:205B8000102038BD21886A461180002801D000290BD0F049034609684D880021284602F0B0
:205BA000B1FF69460988218038BD0C2038BD30B50C46E94987B08C4206D3012189048C427A
:205BC00005D3E3498C4202D2102007B030BDE14D2968C0310A7A520708D48A79521F13005B
:205BE0000FF09CFA05040604040604000820ECE7497AC90901D00D20E7E7FEF7B9F90128C3
:205C000003D002282DD0D548DFE720881E2801D20720DAE72868C030807906281FD00A203E
:205C2000FEF71AF905216846017000798108A0788900C007C00F014368460171FB2001401E
:205C4000A0788007C00F80000143684601712188C18009F072FE0028B7D00320B5E707200A
:205C6000DEE70620B1E7F0B587B014460D46FEF77FF9012804D0022802D0B84807B0F0BD4E
:205C8000B44B18680146C0310A7AD20707D08A79062A04D9092A02D0002D02D050E00820AD
:205CA000ECE7AD4A944206D301229204944204D3A74A944201D21020E0E7A278D206520F21
:205CC000042A0CD8E378072B09D3102B07D822799A4204D3102A02D822881E2A01D00720E3
:205CE000CCE702468032966BF727F372966B23793373966B737A3B40A778BF06FF0FFF00D6
:205D00003B437372966B2388F381966BA778B37AFF079B089B00FF0F3B43B372FB273B4021
:205D2000A778966BBF07FF0FBF003B43B372926BA478537AE406DB08DB00640F23435372E1
:205D40000B226B461A70852D22D008DC002D17D0812D17D0822D17D0832D08D116E0862DE2
:205D600018D0882D18D0892D18D08A2D18D00B221A71B622125C774C002A13D0A83012E0C9
:205D80000022F5E70122F3E70222F1E70322EFE70522EDE70622EBE70822E9E70922E7E729
:205DA0000A22E5E7002002908879072806D0082804D00A2804D00B2802D004E0062000E03A
:205DC0000920FEF749F8684609F0B7FD002801D0032053E720680422C030017A4908490000
:205DE00011430172002049E770B55A4E0D46316886B0C031097A1446090701D408206CE571
:205E0000FEF7B6F8012803D0022801D0534864E5002D10D05048844206D301208004844255
:205E200004D34B48844201D2102056E5012D0BD0022D02D106E0002C01D007204DE500208D
:205E4000029005E0022000E00120694608710294032069460870684609F06FFD002801D094
:205E600003203AE53068F722C030017A11400172002032E570B594B014460E46FEF778F84D
:205E8000012804D0022802D0344814B070BD314D2868C030007A800701D40820F5E7002C98
:205EA00001D00720F1E7FFF732FA002801D01120EBE7002E1DD02D21684601702C68BC20FC
:205EC000015B684641801022B11C01A80EF099FE207EFB210840B17CC907490F0843207682
:205EE000B07CFF214008A075608A82310843608207E02E21684601702868A030818B6846C0
:205F0000418009A9684607F00BFD2968FD23C0310A7A1A400A72B8E710B50C46FEF728F89A
:205F2000012803D0022801D00C4810BD0A48844206D301208004844204D30548844201D230
:205F4000102010BD2046FEF722F8002010BD0000002000205400002000600100023000009B
:205F600010B594B00446FEF703F8012804D0022802D0644814B0E9E763480068C0308179A8
:205F8000042910D005290ED03820694608704C8001200871487109A9684607F0C1FC00280E
:205FA000E8D00B20E6E70020E4E710B594B00446FDF7DEFF012803D0022801D05148D9E7D2
:205FC00051480068C030817904290DD005290BD03820694608704C8000200871487109A974
:205FE000684607F09DFCC5E70020C3E746480068C0308079062801D301207047002070475D
:2060000008B51346002806D040A00068009048796A468009105C18700622581C0EF0F1FD1E
:2060200008BD00B587B0012069460870684609F084FC07B000BD10B50446FDF785F9A22188
:2060400001700ECC08300EC0FDF79AF97EE770B52D4C054601682068002911D02C4A9142D6
:2060600006D301229204914204D32A4A914201D2102070BD102277300EF0C3FD206801212C
:206080008030806B01722068A9880182C17B01290CD1807B800901280AD00120FEF7CEF810
:2060A000002803D01C491D480EF047FF002070BD0120FEF791F8F3E770B505460068124CDB
:2060C00000281AD01349884201D2102070BD2068B8210958097A012909D0014677312930C8
:2060E0000AF063FF206801218030806B017221681022286877310EF084FD2068008AA880E0
:20610000002070BD02300000540000200302FF010060010000200020C041000003030000DF
:20612000FFB581B001980E46C078174610360E37022809D0032840D005287DD0F2A1F748E3
:206140000EF0FBFE05B0F0BDCC890A2060430E30188031230A98002A0380F3D04868008850
:2061600090800020D0801081097B9481891FCDB21AE030887168388048780A780002104374
:20618000F880C8788A78000210433881BA1C091D28460BF058F8002D01D0002802D000206A
:2061A0003871788008360A372046641EA4B20028DFD101990020C870C4E7CC890A206043EA
:2061C0000E30188032230A98002A0380BAD04868002500889080D5801581087B401FC0B20F
:2061E0000090948142E0716832880878FA803A79C30752085200DB0F1A43FD231A408307D7
:20620000DB0F5B001A43FB231A404307DB0F9B001A43F7231A400307DB0FDB001A43EF2386
:206220001A40C306DB0F1B011A43DF231A408306DB0F5B011A4300E020E0BF231A404306EB
:20624000DB0F9B011A433A71C00978718A784B781002184338813A46C91C00980AF0F3FF2A
:20626000002801D0BD703D8008360A372046641EA4B20028B7D10198C57063E7087BCC89DE
:20628000801E85B22846083060431030188034230A98002A03808FD048681746008890805E
:2062A0000020D080108194811037E000D581C0190CE030883880009878602A4671680098C5
:2062C0000EF09FFC009808360837401900902046641EA4B20028ECD16BE7FFB50546C0787B
:2062E00081B00C460A9E03000EF018FF0BA3071733414F6D8F9D9D9DA300207B174608282E
:2063000006D0032804D085487FA154300EF015FE04990E20088030200CE0207B1746042873
:2063200004D07E4878A171300EF007FE04990E20088031203080002F44D060680088B880E7
:20634000607AFF300130F880E08938810020B88137E0207B1746042804D070486AA18D3081
:206360000EF0EBFD04990E2008803220E2E7207B1746022804D0694863A1A9300EF0DDFD6D
:2063800004990E2008803320D4E7207B1746042804D062485CA1C4300EF0CFFD0498102172
:2063A000018034203080002F0CD060680088B880607AFF300130F880E08938810020B88198
:2063C000F881E870BEE6207B1746052806D0062804D052484CA1E1300EF0AFFD049812213A
:2063E000018035203080002FECD060680088B880607AFF300130F880E0893881E089B8812E
:2064000000203882A988F981DBE7207B1746072804D042483CA1F8300EF08FFD04990E2056
:206420000880362086E700962846049B00F02DFD88E635A13A480EF080FD83E670B505463A
:2064400000780C46082603000EF068FE124C3434241C380A0A0A0A0A0A0A0A0A0A0A0A4CDB
:206460006878002804D02E4827A12C300EF065FD002C03D11F2024A1400108E060783043CE
:20648000607020E0002CF9D17D201FA1C0000EF054FDF3E7002904D03F201BA100010EF0D9
:2064A0004CFDFCF751FF0446407830436070FCF767FF08E01A4814A1473002E0184812A147
:2064C0004C300EF03AFD002C0AD06078000707D5932020702046582229460830FAF774FE1D
:2064E000002070BD0E4808A15030EAE710B500200C4C0D490346C2008C525218401C0006B7
:20650000D370000EF7D010BD7372635C67617474635F636F72652E63000000005A020000EA
:20652000B3030000FFFF000058000020FE4908800120887000207047FB490020887070475D
:2065400010B50021F848C94301800021C17007F021FAD8E7F7B584B00546002768460781DD
:20656000878068680C46008800F0ECFB0646287A032805D0002E03D1EC49ED480EF0DDFC62
:20658000297A2046C91E123000900B000EF0C6FD0FF2F1F03D09AA465C6D34B3CDF38B8BCF
:2065A000F000F078012803D0E049AD200EF0C5FCA8896946C0000E30888030200881002CE7
:2065C00022D068680188A180E7802781A989A18100200DE0C100B27909190A74B288CA81CE
:2065E00082005219D3894B82128A401C8A8280B2A1898142EED8D7E002A8009001AB224697
:206600002946304600F0CCFBF1E002A8009001AB22462946304600F005FCE8E0F07806288B
:206620001AD0FF20C149223014E068680188A180E7802781A989A181B188E181E989218274
:20664000EA89296900982BE0F078062804D0FF20B6493C300EF071FCE889694612308880C9
:2066600035200881002CE0D1C1E0F078072804D0FF20AE4956300EF060FCA88969460E303F
:20668000888036200881002CBED068680188A180E7802781A989A1812046AA890E30296913
:2066A0000EF0AFFA80E0E8896946123080B2382288800A81002C79D068680188A180E780FC
:2066C0002781A989A181287A102809D00221A173E9892182EA89296900980EF092FA86E032
:2066E0000121F4E702A8009001AB224629463046FFF716FD7BE0F078082803D08B498D48F2
:206700000EF01BFC14206946888037200881002C6DD068680188A180E7802781A989A18153
:20672000678227820120A0733EE0F078092804D080487E4918300EF000FC288A6946143092
:20674000888037200881002C51D068680188A180E78004212781A173A989A181E9892182D9
:20676000298A618220462A8A1430696998E702E038E01CE024E0F0780A2804D06D486B4903
:2067800033300EF0DAFB14206946888037200881002C2CD068680188A180E7802781052121
:2067A000A173A78127826782F77020E017E002A8009001AB224629463046FFF78EFD16E003
:2067C0000D206946392288800A81002C07D00120E08055480188A1802781277307E006995C
:2067E000088010E08F205149C0000EF0A6FB6846069980880880002C05D0684600892080C4
:20680000684680886080002007B0F0BDF7B594B015460F46149800F0A0FA04000AD0032087
:2068200000F088FB022802D2E078002804D0112017B0F0BD4048FBE71720694601260883EC
:20684000002D0FD00321684601711021018210A80246059004A928460AF01BFD00280DD06D
:206860000720E5E708216846017100210781C943418105218673C90281810CE0A878A0715C
:206880002888A080684605218673C902818100210781C943418109AA023206A901A807F0E1
:2068A000B2F8002802D000F06BFAC1E707A800906846038B04220321149800F051FB002862
:2068C000B6D1E670B4E770B592B00D0006460ED000F043FA04000CD0032000F02BFB022832
:2068E00002D2E078002806D0112012B070BD1020FBE71148F9E71721684681800421017284
:20690000298881816988C181012181740B4901820AAA023201A902A807F075F800280FD0FC
:2069200000F02EFAE1E7000058000020086500003C04000063020000023000000228000091
:2069400008A800906846838804220321304600F007FB0028C9D10221E170C6E770B592B042
:206960000D0006460DD000F0F8F904000BD0032000F0E0FA022802D2E078002805D01120B0
:20698000B3E71020B1E7FA48AFE717216846818004210172298881816988C1810121817441
:2069A000F44901820AAA023201A902A807F02BF8002802D000F0E4F997E708A8009068468E
:2069C000838804220321304600F0CAFA00288CD10321E17089E770B592B00D0006460DD031
:2069E00000F0BBF904000BD0032000F0A3FA022802D2E078002805D0112076E7102074E7F8
:206A0000DB4872E7022168460172298881816988C181172181800AAA023201A902A806F065
:206A2000F2FF002802D000F0ABF95EE708A800906846838804220321304600F091FA002836
:206A4000DBD10421E17050E7F0B591B015000E4607460ED000F081F904000CD0032000F006
:206A600069FA022802D2E078002806D0112011B0F0BD1020FBE7BE48F9E7172168468180E1
:206A800004210172298881816988C181B1788174318801820AAA023201A902A806F0B3FF3A
:206AA000002802D000F06CF9E1E708A800906846838804220321384600F052FA0028D6D1F3
:206AC0000521E170D3E7F7B592B015460E46129800F043F904000AD0032000F02BFA0228D2
:206AE00002D2E078002804D0112015B0F0BDA048FBE70627002D12D0684607728681C58151
:206B0000A5801720694688800AAA023201A902A806F079FF002807D000F032F9E5E70521AC
:206B2000684601728681EBE708A800906846838804220321129800F013FA0028D5D1E7704C
:206B4000D3E7F7B592B016460D000ED0129800F004F904000BD0032000F0ECF9022802D2DA
:206B6000E078002805D01120BFE71020BDE78048BBE707276846077286811721049581807D
:206B80000AAA023201A902A806F03DFF002802D000F0F6F8A9E708A8009068468388042200
:206BA0000321129800F0DCF900289ED1E7709CE7F3B5172091B00C46002915D021780B00AD
:206BC0000EF0ACFA062B05051A041C2B1520C01EE28880B2002A02D0A368002B04D08242F8
:206BE00004D90C2013B0F0BD1020FBE7042905D0A088002811D101E00620F3E7119800F05C
:206C0000ACF805000BD02078092701281AD0022807D0042824D0052835D00720E2E7544836
:206C2000E0E76846077161880181E1884181A06808260390304600F07DF9072829D34C486D
:206C4000801CCFE70C216846017161880181E1884181A06803900EE0E878002811D118E014
:206C60000D216846017161880181A1884181E1888181A06804900326304600F05BF902285C
:206C8000EAD31120AEE70E2168460171217B0172F1E717216846018309AA023206A901A892
:206CA00006F0B1FE002802D000F06AF89AE707A800906846038B04223146119800F050F968
:206CC00000288FD12178012907D002298AD0042905D0052905D0032084E7082102E0EF7010
:206CE00080E70A21E9707DE730B591B00C46054600F033F8002808D0032000F01BF9022816
:206D000005D31B48801C11B030BD1948FBE70F216846017104811721018309AA023206A984
:206D200001A806F070FE002802D000F029F8EAE707A800906846038B04220321284600F047
:206D40000FF9E0E70C49884205D00C490988814201D10A4870470020704710B5FFF7F2FF69
:206D6000002802D08178C90700D1002010BD00000230000003280000FFFF000058000020BF
:206D8000002806D0012805D0052805D0062805D00320704711207047082070475C487047F6
:206DA000FFB583B003980C9EC0781D4614460F46012803D05749D2200EF0BFF8F889C000D9
:206DC0000E30288030203080387B001FC0B20190002C26D078680088A0800020E08020812D
:206DE000F889A081002616E0F0000519C01900902A4641690E3201980AF025FA002802D058
:206E000000202874E8810098761C008A68820098B6B2408AA882A089B042E5D80399002027
:206E2000C870F1E4F8B50646C0781F4614460D46042804D0FF20374903300EF07EF8A8898B
:206E4000062148430E30388033210698002C01801AD068680088A0800020E0802081A98936
:206E6000A18103460CE01946062251434A190919D789CF81977C8F74128A5B1C0A829BB269
:206E8000A1899942EFD8F070F8BD70B514460546142204981A8037220280002C18D048683C
:206EA00000260088A080487AFF300130E080C8892081C889A0816682E878082809D009289C
:206EC00011D00A2819D0134913480EF036F8EE7070BD087B0C2804D00F480E490C380EF0CD
:206EE0002CF8012012E0087B0D2804D00A48094908380EF022F8042008E0087B0E2804D03A
:206F000005480449001F0EF018F80520A073DEE70330000008650000820300000146002021
:206F2000F74A02E0401C082803D24300D35A8B42F8D1704730B50446F14A0020163A1179AC
:206F400053790AE05518AD79A54201D1401CC0B2491CC9B2102900D100218B42F2D130BDD9
:206F6000FFB5E74881B0163841790A9C491CCDB21E46102D00D10025E14816380079A842FA
:206F800002D1042005B0F0BD0820FFF7D3FF0746072804D9FF20DBA1A1300DF0CEFF02987F
:206FA000082801D1072F17D001982080301D6080002060712071E68003982081204606F0CC
:206FC000D3FC00280AD0CE48029916384379821D995445710020D5E7CF48D3E7FF20C9A1AD
:206FE000B3300DF0AAFF0320CCE7F0B58DB0044600256846057116468C460620FFF79AFFDA
:2070000000281CD121780127C807002801D0132917D9684687766178C17602218183C5837C
:2070200004A8009070680C23008805220621FFF797FF002803D0B3A184200DF07EFF0DB081
:20704000F0BDAF4816380278002AF8D0427863789A42F4D1012918D0132919D1614606298E
:2070600016D10570002101200AF01CFE68460771706801886846C1800021C9430181607960
:2070800022790102114368461AE06146062908D0684600790028D2D0314601A8FDF7A7FEFE
:2070A000CDE70570002101200AF0FCFD684607716079227901021143684601810021C94324
:2070C0004181E9E78E4810B50021163801704A1E428041700171417101200AF0E3FD10BDDC
:2070E00010B5FFF7EFFF0020854902464300401CCA520828FAD310BD10B50446FFF7E2FF46
:207100007F4816384480002010BDDBE770470EB501216846017081498180C1800021FDF70B
:2071200066FE0EBDF7B505460078002700090C463E46012804D0FF2072A164300DF0FDFEF0
:20714000287A02280CD0FF206EA17A300DF0F5FE0298002C068001D0278066800020FEBD3A
:20716000EA89702710460A3086B2002C0BD068680088A080A8892081E28020460A30296958
:207180000DF03FFDE4E702980680E7E7F8B543680246D9799C79090221435C7A1E7A2502F2
:2071A0005C88981D3543241FA1421DD11B79022B1AD1042D19D0052D26D0062D19D0402D33
:2071C00012D3061D0F4614462846FFF7A7FE08280AD01120207002202072A581E78126615B
:2071E0006078082108436070F8BD001D00F0D9F8F8BD041D0D46FEF7F9FE0028F8D029466C
:207200002046FDF730FEF8BD001DFFF7EEFEF8BD10B53B4C8AB0163C2278012A26D01223B5
:207220006A46937363789B1CD373082313820B8853824B8893828B88D382C988118301A9B9
:2072400000910C2305220721FFF78AFE00280BD10022F023114601200AF07FFC01202070CA
:207260006078801C607000200AB010BD1120FBE7F8B5234C0027163C0646A51D1BE0607999
:207280002179884204D187201EA180000DF055FE2079405D042804D0082804D17F1CFFB2F8
:2072A00001E0FDF7F2FD2079401CC0B22071102801D1002020713046761EF6B20028DED1CE
:2072C0003846F8BD10B50446402801D2072010BDFFF724FE082802D03120000210BD0021E2
:2072E000074802E0491C082903D24A00825A002AF8D1082914D049004452002010BD0000F8
:20730000DA1300207372635C6C326361705F636F72652E630000000004300000FFFF00001F
:207320000420EBE700B5402801D2072000BDFFF7F5FD082805D000213B4A400011520846FF
:2073400000BD052000BDF0B58BB016460C00074607D0002E05D06188402904D207200BB015
:20736000F0BD1020FBE72088002801D0172801D90C20F4E70846FFF7D1FD08280FD02588BF
:2073800003A82A46314602300DF03BFC01A8009062882B4608213846FFF7E2FDDFE70520FA
:2073A000DDE7F0B50E46074601468BB014460125304606F0A5FC08281CD10020694608853B
:2073C0000120FFF7B7FD002802D117206946088503AB02330AAA39463046009407F0A3F8C2
:2073E000002809D0022818D0032803D00F49FC200DF0A3FD2846B2E76846038D002BF9D032
:2074000001A800906068042200880121FFF7A8FD0028EFD00549E720EAE7607800251021C5
:2074200008436070E6E70000DA13002004730000002803D08178012939D101E010207047F0
:207440000188FA4A881A914233D01BDCF84A881A91422ED00BDC00292BD00320C002081A29
:2074600027D0012825D001210903401A07E001281FD002281DD0FF281BD0FF3801380028AF
:2074800015D116E0FF220132811A904211D008DC01280ED002280CD0FE280AD0FF2806D17F
:2074A00007E0012905D0022903D0032901D0002070470F20704700B50A2821D008DC03006F
:2074C0000DF02CFE0A1C2024241A24282224261A102819D008DC0B2816D00C2814D00D28A0
:2074E0001AD00F2808D111E011280FD0822807D084280DD085280DD0032000BD002000BD38
:20750000052000BDCB4800BD072000BD0F2000BD042000BD062000BD0C2000BD70B50029EE
:207520000BD0CB1FFA3B81241E46CDB2112B1BD2012805D0022806D009E0002010701DE01C
:20754000FF20043001E0FF200330814218D033000DF0E4FD111613131613161613161616F2
:2075600013131313161316000846FF3881381F2803D9FF39FE39022902D81570002070BDD9
:207580001470072070BD00B503000DF0C7FD060406040C080A0C002000BD112000BD07206A
:2075A00000BD082000BD032000BD00780207120F04D0012A05D0022A0AD10EE0000907D1FD
:2075C00008E00009012805D0022803D0032801D00720704708700020704706207047002891
:2075E00007D0012807D0022807D0032807D007207047002004E0112002E0212000E031204A
:2076000008700020704738B50C4605004FD06946FFF7CBFF002822D120880321890288430C
:20762000694609788907090D084320806946681CFFF7BBFF002812D1218803200003814308
:20764000684600788007800C01432180A8784007820F2020012A03D0022A03D0072038BDBB
:20766000814300E00143218088B20105890F08D0012189038843A9780907C90F8903084378
:20768000208080B28104890F0AD0A9784004C906C90F400CC903084320808004800F02D12C
:2076A0002088400403D52088402108432080002038BD70B504460020088015466068FFF7CD
:2076C000A2FF002815D12189A089814210D86168594E8978C90707D0711E884208D83146B5
:2076E0000DF009FB298009E0FF21FF31884201D90C2070BDFF30FF300330288060688078B1
:20770000C007A08903D031460DF0F5FA03E0FF30FF30033081B2298020688178474801736F
:2077200020684649008820394885002070BD10B5137804785B08E4075B00E40F23431370E6
:20774000FD2423400478A407E40F640023431370FB24234004786407E40FA4002343137055
:20776000F724234004782407E40FE40023431370EF2423400478E406E40F24012343137047
:20778000DF2423400478A406E40F6401234313700078BF244006C00F2340800103431370FF
:2077A000002906D00878C10701D1800701D5012000E00020C0015906490E0843107010BD23
:2077C00030B50A8803239B0204889A4323059D0F02D1A3049C0F01D09B0F00E001239B02F1
:2077E0001A4303230A801B039A4303889804840F02D11805830F01D0800F00E001200003E1
:2078000002430A8030BDF3B591B00D0018D01198002818D0122128460DF050FA01A9012062
:2078200007F07DFE00242646374677E0022900000128000003300000010200000C140020A8
:20784000102013B0F0BD0720FBE76846007C01280BD16846C1890520C002081A0AD001284C
:207860000AD002280CD003280CD0042C0ED0052C0FD10DE0012400E002246846868908E045
:20788000032406E068460424878902E0052400E0062468468189119881423FD12C74002EDE
:2078A0003AD00BA800900CAB10220021304607F0C8FE002820D16846808D2A46C0B20CA9D3
:2078C00009F0C1FC002817D1AE81002F24D00BA8009006AB13220021384607F0B2FE0028F9
:2078E0000AD16846808D06A9C01E0331C0B22A1D09F0A9FC002801D00320A2E76846817E88
:20790000427E08021043E881062C05D16846007CA8726846C0892881002092E701A807F0BC
:2079200006FE002891D0FFF7C6FD8AE7002804D0012903D0022904D003207047F949C98D26
:2079400002E0F8494031C988814201D1002070470720704730B5F34C0025608B91B0C00BB8
:207960002ED1216900292BD0207B800728D4012268460271027200224272228B8281A28AD2
:20798000828204911721018309AA0023023206A901A807F07BF9002803D0FFF7F4FD11B022
:2079A00030BD207B02210843207307A8009069460B8B208804220121FFF7D2FA05460BE0D2
:2079C000FBF7C2FC842101700921017218341ECC0C301EC0FBF7D4FC2846E0E710B5D14C1B
:2079E000034621690020002909D02146012210311846FBF783FE00202061A0820120217B76
:207A0000F9221140217310BD70B50C4605461C2120460DF053F900202080002D08D0012DF8
:207A200004D0C1A1C5480DF088FA70BD062000E00520A07070BD10B507F050FB10BDFEB568
:207A40000546007800260C46374603000DF066FB0C91070C1D962F462F46486C8991686822
:207A60000A38FBF7B0FD89E0002904D0B348AEA11B300DF062FAFBF767FC04464078082151
:207A800008436070FBF77CFC78E0002C04D1BB20A5A180000DF051FA284601F0A2FA0028FC
:207AA0006CD06078082108436070022666E0E888694608800190002C04D1A0489AA12F3045
:207AC0000DF03BFA287807281CD10198C00B19D0944800218171A988818012E003264DE002
:207AE000002C04D1C52090A180000DF026FA8D48017B89070BD50069002802D0E888C00B73
:207B00003CD00226607808210843607036E0291D8EC918308EC02838018802260122204632
:207B2000FBF7CEFD0127EDE7002C04D183487EA164300DF002FA7B480821007B4007C00F97
:207B40004600607808436070002E17D12879012802D16879002811D02046FFF73FFF074668
:207B60000CE0002CCED10D206FA180010DF0E5F9C8E772486CA17A300DF0DFF9002C0CD0B8
:207B80006078000709D5002F07D1842020702046582229460830F9F717FB3046FEBDF7B587
:207BA000027A88B00C46054620460C300490069216300027921E02903E460A315948130084
:207BC0000DF0ACFA0ADF06E62AE62AE66A98C6E64288002A02D052270726DDE051271E267A
:207BE000002C7DD06A684F481288A2800122A2718079C0004019C089FFF705FE002877D1ED
:207C000048488179C9004919C98921818079C0004019408AA083BFE0688A009006980728CE
:207C200017D1E889C00B14D000985127223086B2002C55D0A8890499FFF7E5FD002857D15B
:207C400068680088A0800220A071A8892081012041E000985027203086B2002C40D0A88961
:207C6000FFF7D1FD002843D168680088A080A889E080287A07280AD002202072288AA083C7
:207C80000098E083204669692030009A01E00120F3E70CF0B6FF7FE0698A009101690029C4
:207CA00002D0E989C90B22D00099512722318EB200218171A9898180002C5FD00088A080CD
:207CC000A8890499FFF79FFD002811D10220A071A88920810420A072288AE083009801E071
:207CE0004CE005E020846969009A0298D1E703200BB0F0BD007B400702D55127222601E04C
:207D000050272026002C39D06868502F0088A08016D00220A0712146287B0831FFF774FEB6
:207D20003AE00000EC1300207372635C67617474735F636F72652E6300000000CB020000DD
:207D4000287BA11DFFF760FE0020FFF747FE23E0A9890089884207D154270626002C0DD003
:207D600068680088A08017E053270826002C05D068680088A080A889E0800DE00A980680CD
:207D800010E055270726002CF8D00020A07103E0FD49FE480DF0D1F80A98002C068001D0CB
:207DA000278066800020A3E7F94800210172203801814181418081718180027BF923520874
:207DC00052001A40027301618182704770B5F04C86B0203C208000206080A071A0806946F3
:207DE000012007F09CFB102608E00199088802461207D20FB043120110430880684607F0C4
:207E000096FB0500F1D02069002804D0DF48DE4933300DF092F8207B800704D5DB48DA490D
:207E200034300DF08AF8822D04D02846FFF743FB06B070BD0020FBE7D54810B52038017B9F
:207E4000012211430173002141808171818006F019FB10BD10B5CE4C0020C043203C20808D
:207E60000020FFF7BBFD207B40084000207310BD70B5C74D0446203D287B800704D5C348C3
:207E8000C1494B300DF059F8287BC00706D12888C049884202D02869002801D0082070BD9A
:207EA000002C08D0A088162801D2092070BD20682861A088A882FFF74DFD70BD10B50C4648
:207EC00007F001FB002804D0C520AF49C0000DF034F82046FFF7EFFA10BDF0B5AC4D0446F3
:207EE000203591B00020089068820E462882E8812946E880403908866946088308850886B0
:207F000088838882A2480E90007A1746012808D0022806D0032804D0042802D0082011B006
:207F2000F0BD9D498C425FD301208004844202D39A4A944258D398498E4255D3012080040B
:207F4000864202D3954886424ED36068002814D09149884248D301218904884202D38F4905
:207F6000884241D360892189884203D801225202914201D90C20D2E7089010AA0CA9304665
:207F8000FFF797FB0028CAD106A92069FFF73BFB0028C4D1206900280CD060788007002861
:207FA0006846008B03DA8004800F6ED002E08004800F6AD16846008B810617D58004800F6B
:207FC000606805D0002811D0744988420CD301E000280BD07049884206D3012189048842DC
:207FE00004D36E49884201D2102098E705A96069FFF709FB002892D16069002808D0684634
:20800000808A0105890F01293FD18004800F3CD007A9A069FFF7F7FA002880D16846808A8E
:20802000800632D46846808B81062ED4A169002906D00105890F012927D18004800F24D0A2
:20804000E068002804D0007800281ED01C281CD24F4A611C123220460992FFF768FB032144
:2080600000208902884301218902411868460D910185012181744A490182454A0FA91532F7
:20808000306809F006F9002801D0072047E708A8007F3F49C01CC2B26A7100201031FF328E
:2080A00000900190FF3203460291039003320AA904A807F0A3F9002827D135482038008E55
:2080C0000B90334833893830326901461239029100930192039010A90A8873890CA9306859
:2080E00007F08CF901007DD12948E98811308170090AC1700026009631386A79008E314650
:20810000099B07F0FAF8002802D0FFF7D4F906E70E98807CC00928D068460D9901850121C9
:208120008174292109020182AE81287B61784008C9074000C90F08432873FD210840617872
:2081400002228907C90F490008432873104800922A30811C0191029000230396114A0AA995
:2081600004A807F04BF901003CD1606800283BD0206900281ED106A90CA8FFF721FB607822
:20818000800717D469460FE0287D0000220400000C140020FFFF0000006001000020002025
:2081A0000328000003020000088B03210903884369460883012069468874FD480882208983
:2081C000FC490CF098FD6268089BFB480192009302900A460396002306A904A807F00EF9FC
:2081E000010000E07EE07DD12078C10601D480062ED568460684606900280DD105A90CA8CC
:20820000FFF7DEFA6846808A032189028843012189024118684681826946888A4821084332
:208220006946888201208874E14808AA401C0882E1490192891C0220DE4A029100900023B5
:208240000396921C05A904A807F0D8F8010063D12078C0072ED068460684A06900280DD1DD
:2082600007A90CA8FFF7ACFA6846818B032080028143012080020918684681836846818BAB
:20828000402001436846818301218174C84908AA891C0182C8480192001D0221C54A009103
:2082A000029000230396921C07A904A807F0A6F8010031D1E068002832D068460D99018582
:2082C00001218174BA49C91C0182E16808A80A78027049784170E068418868464184E068F1
:2082E000017900E018E008A80171E0680722C18808A84171090A8171AF4808A9801D009212
:2083000001910290412200230396D2000AA904A807F074F8010003D00B98FFF7CFFDFEE56A
:2083200003210E98002F017207D0E8883880E8897880288AB880688AF8800020EFE5F0B57C
:2083400001248BB016460F46012802D002281BD104E0684605218474C90202E06846974910
:2083600084740182002F11D003210020890288430121890241186846018506AA05A93846C2
:2083800008F087FF002803D00720B1E41020AFE4894DB8782E3D287338882F46203F788548
:2083A0006A46127D0020294606AB00920E310193FF32029103900346FF3203320AA904A874
:2083C00007F01CF8002802D0FFF775F890E4002E01D0F88D30802C72002089E470B592B0FB
:2083E0000446012508A8857075496846018406F07CFF002208A90120FFF7A1FF064606F03A
:2084000078FF30003AD120780024C00700283FD01C2168460CF054FC68460178202001430E
:208420006846017008A8857066496846018411940794817FF9200140891C68468177002091
:20844000014668460177002001466846417704218185C485018607A80A9011A80D9008A898
:20846000099006F042FF0EAA09A96846FFF735FD054606F03EFF002D02D0284612B070BD12
:208480004D486946098F4E3801816946898F418149482E3804720020F0E7F7B5464E9CB07F
:2084A00000212E3E0091317A012904D0022902D008201FB0F0BD40494E39CA8D824201D058
:2084C0000620F6E71D98824201D10720F1E73B48012110AA9176401C1083002003239B0217
:2084E00002469A438B02D31810AA93846A4691843549D18410AA9077908317AA0A926A4695
:2085000091850C9009A807F031F800242546274604A909A807F02DF8002810D082287BD164
:20852000002C7CD0002D7AD010A8048145810024047518A8807812AD012872D07AE06846C2
:20854000807D002F1FD0012862D16846818A1B48401C814219D114A800906846408A0EAB02
:208560001022002107F06DF8002877D110A8008A042801D006285BD16846018F1D9881428D
:2085800046D10F2095E7012842D16846808A0521C902884202D0491C884239D106484E388B
:2085A000C18D6846408A814210D101270FE0000001290000010200003A1400200128000076
:2085C00001180000052A0000FFFF00000027002C01D0002D0DD01D99884219D114A900916F
:2085E00004460EAB1022002107F02BF8002835D101E0009D0CE010A8008A022801D01028FE
:2086000016D1C0B218AA0EA908F01DFE00280FD16846408A00907BE720E000E001E005201D
:2086200047E72A1D15A918A808F033FE002801D003203EE710A8007D0023001DC2B210A83C
:2086400002751E98029019A901950394009216A806F0D4FE002801D102213172FEF72BFF75
:2086600027E73EB50B46401E84B201AA00211846FFF75DF806F039FE02A8009001AB012269
:208680000021204606F039FE044606F032FE68460089012803D0FE49FE480CF04EFC20464A
:2086A000FEF709FF3EBDF0B5FB4E0446307A89B00F46032804D0042802D0082009B0F0BDC7
:2086C00004AA06A92046FEF7F4FF0500F6D1F2482389383022690146103902910093019201
:2086E000039069460A8A638906A9206806F086FE002802D0FEF7DFFEE0E7002F03D0E64844
:20870000203000893880042030722846D6E738B50C00054608D00022694606F0ECFF0028E1
:2087200004D0FEF7C8FE38BD102038BD69462046FEF769FF0028F8D1A0786946C207D20FBC
:20874000284606F0F3FFECE73EB50C0008D002AA694606F0D0FF002804D0FEF7ACFE3EBD63
:2087600010203EBD032120460CF0A8FA6846008801A90005800FFEF732FF00280BD168465A
:20878000007920706846008801A98004800FFEF726FF002801D003203EBD684600796070B5
:2087A000A278EF20024068460088C10B09010A43F7210A404104C90FC9000A43A270F92134
:2087C0000A40800601D5012000E00220400069460243097A50084000C907C90F0843A0707E
:2087E00000203EBDFEB51D4614460E46074606F07CFD01A8009022882B463146384606F09F
:208800007CFD054668468088208006F072FD2846FEF751FEFEBDF0B50C46002199B00746BE
:20882000684681850D46002C11D0E068002806D0A06800280BD002886B469A850180A078E0
:20884000012806D0022804D0072019B0F0BD1020FBE72088002807D0401E80B201A906F095
:208860005EFE002842D136E08C48EEE769468A8921888A420BD26846007C002501282CD119
:208880006846C0898649884227D1012525E08A4203D1002D2FD06D1C01E0022D02D0032DBE
:2088A0001BD31FE06946097C012916D169467C4BCA895B1ED11A9A421DD005DC7948101AC4
:2088C00019D0012809D116E0012914D0FF39013903D1032506E00D26B60201A806F027FEA5
:2088E0000028C3D0822804D0002806D0FEF7E3FDABE7022DFAD13046A7E7E068002813D089
:2089000006F0F3FC0BA800906A46A1882088928DE36806F0F2FC054606F0EBFC002D19D121
:208920006846A168808D088002980078C00601D55D488AE706F0D9FC0EA80090684680895F
:208940000CAB0222002106F07CFE054606F0D1FC002D01D02846C9E76846008F022801D049
:20896000032072E7A078012808A8007C03D080070ED4082069E7C007FBD00820FEF7DAFAD7
:20898000072802D34548401C5FE70825022001E0022503206946087621886846818317216A
:2089A000818611AA002302320DA906A806F06EF9002802D0FEF7E7FD47E70FA800906846E7
:2089C000838E042229463846FEF7CAFA3DE770B5064615460C460846FEF72AFD00280AD10B
:2089E00006F083FC2A4621463046FFF7A8FC044606F07FFC204670BD70B514460D460646AF
:208A000006F073FC224629463046FFF746FD044606F06FFC204670BD70B51E4614460D003D
:208A20001AD0002C18D06168002915D00121FEF77DFF00280FD12068FEF7FAFC00280AD150
:208A400006F053FC324621462846FFF746FA044606F04FFC204670BD102070BD70B5154653
:208A60000C0023D00221FEF761FF00280ED12068FEF7DEFC002809D106F037FC2946204621
:208A8000FFF711FE044606F034FC204670BD0000287D00003E0600000C1400200330000072
:208AA0000328000000280000013400001020EDE7FEB50746FF481C4615460E46824218D323
:208AC000002C01D0844214D3384600F047FA00280AD1002C0FD101AA6946384606F00BFE57
:208AE000002802D0FEF7E7FCFEBD68460088800601D41020FEBD23462A4631463846FFF7A9
:208B000071FEFEBDFFB585B01E4614000F4609D003AA02A9059806F0EEFD002804D0FEF7D5
:208B2000CAFCCBE51020C9E568460089C00601D5E148C3E506F0D9FB01A800900023DF4AEE
:208B40003946059806F07DFD054606F0D2FB002D11D1002E0CD006F0C8FB0020009022884F
:208B600033463946059806F06CFD054606F0C1FB6846808820802846D1E7002906D0D04B6E
:208B80000A885B899A4201D8CE48704743E610B586B004236C46A382C94B1C89002C07D0FF
:208BA0005B898B4201D2914204D9C64806B010BD0620FBE76B4619825A820021009101917C
:208BC0001C800221997005A9029104A903916946FFF721FEEAE7F0B591B00D46812069462D
:208BE000087105F081FC0646002D08D02878B44C012806D0022828D0072011B0F0BD1020B3
:208C0000FBE7A98801AAFEF789FC0028F5D1B00734D568460079002820D1A879C0071DD059
:208C200006F063FB002000906A892989A088EB6806F063FB6946087106F05BFB6946087918
:208C400000280BD0FEF737FCD7E7A98801AAFEF765FC0028D1D1342006420FD001216846E4
:208C60000172017301794173F00609D5A18868460182A18A01832069059004E00820BCE735
:208C8000A08869460882FAF75FFB05461720694688830AAA2B46023207A902A805F0F6FF4F
:208CA00007466878000701D5FAF76AFB002F03D03846FEF768FCA0E7F00603D5207B062164
:208CC00008432073B00602D50020FEF787FE08A8009069468B8B208804220121FEF740F96C
:208CE0008BE7F0B5002695B014460D4600290FD0022C4FD3A71EBAB270480AF037FE291993
:208D00001039CA7B8B7B11021943884242D1BCB201A9012006F003FC7AE0029F3888010782
:208D200076D5002D41D0A9190691CA788B78361D1102B6B219438919A1422BD869468A8998
:208D400006994B7809781B020B439A4222D1C00623D506F0CAFA07A800900698AB19C178A4
:208D600080780A02069902434878097800020843002106F0C2FA009006F0BBFA00980028AF
:208D80003ED10698C178827808026946898B1043884202D00B2015B0F0BD0698C1788278C9
:208DA00008021043801986B22EE0C0062CD5002007AA01461154401C80B21028FAD306F0AA
:208DC00094FA06A800906846002380891022194606F037FC0090002803D006F08AFA009896
:208DE0000EE00BA86946009088890A8B07AB002106F083FA009006F07CFA0098002803D018
:208E0000FEF759FBC7E703E0388810218843388001A806F08CFB002800D17EE7284D69881A
:208E2000002921D00122684602760277002444770184172181850EAA234602320BA906A8FD
:208E400005F024FF002802D0FEF79DFBA3E70CA8009069468B8D288804220121FEF780F879
:208E6000002898D16C8096E7002094E7F0B5002487B015460E46002A04D002A9012006F0EE
:208E80004EFB4CE0102007B0F0BD03980078000745D506F02AFA01A8009068460023008AE7
:208EA000064A194606F0CDFB074606F022FA002F2ED109E00020002001340000FFFF00005C
:208EC000EC13002003300000002E23D068468088298820183719001D814230D36946098A0B
:208EE0003970090A797069468988B970090AF97006F0FBF901A869460090088A8A883B1D9A
:208F0000002106F09EFB074606F0F3F9002F01D00320B8E7684680882018001D84B202A8C5
:208F200006F005FB0028B0D0822802D0FEF7C3FAA9E7002E0ED02988A01C814201D20C209A
:208F4000A1E72246314639480AF010FD31190870000A4870A41C2C80002094E700B585B0AD
:208F60006946FEF750FC00280AD16846007C03000CF0D4F808052F2F2F2F080805310320D7
:208F800005B000BD68468078012807D1684600880321C902401A1CD001281AD06846807993
:208FA000012806D16846808815214902401A05280FD96846807A012811D1684601892920D7
:208FC0000002081A05D0022803D0032801D0042805D10F20D4E7164916480BF0AEFF00202E
:208FE000CEE738B5144A0021518003791AE0CC002418A46800946C462488250707D5E50610
:2090000005D5D90008182038C08B508006E0640406D59171C9000818C0889080012038BD88
:20902000491CC9B28B42E2D8002038BDFFFF0000287D000033020000EC1300200120F9495A
:209040004006C861704770B5F64D0024AC7028466C7020304470C4736C61AC72AC6209F0CB
:20906000FEFEA861284630300AF098FD002804D0FF20EDA13A300BF060FFEF48C4630120A2
:209080004006E86170BD70B50125EC4902260E60E949CD63EA49C96A09070ED4E8494031A2
:2090A000CB6AE84A53620B6B93624B6BD3628B6B1363C96BD30519435163DA49E24CC96933
:2090C00000282BD001282DD0FF20D7A169300BF034FFDE48A063FF20043060632563DC49FD
:2090E000032008602061D849962040314860DA48D8494163D649FC390163D649091FC1636A
:20910000D349F03981630320D349000340394860D24910204860D248066070BDD148606149
:20912000D14804E0D048E0306061CF48801F0143A161CEE7BB49012008707047B949002022
:209140000870704770477047BF4940310028086802D00122104301E0400840000860704791
:2091600070B50C46AF4D01460622E81C0BF049FD6C7270BDAB48203040787047A94A917017
:209180005070704770B50D460446082904D9FF20A5A1C6300BF0D1FE0022B44809E09100CB
:2091A000635809180B6053001B191B8C0B62521CD2B2AA42F3D3206BAC494031086070BDA3
:2091C0000B23DB4310B5C21A9F4998421FD008DC1C3222D00A2A20D0142A1CD0182A08D164
:2091E00017E0083011D004280DD0082809D00C2805D0FF208CA1F2300BF09FFE10BD04204D
:209200000CE000200AE0FC2008E0F82006E0F42004E0F02002E0EC2000E0D820C86010BD93
:2092200080482030007B704710B5874CC17861620BF048FD0002E06110BD252808D026288D
:2092400008D0272808D041000A2807D8091D06E0022105E01A2103E0502101E0891DC9B218
:20926000794A916078494031486170476D494861704770B56B4CA07200F01FFBA07AC007B9
:2092800040D0734D2868800703D467A178480BF054FEA07A01061DD5800707D5744862A1C6
:2092A000801C0BF04AFEA07A000613D520786A4E012816D0002804D051205BA1C0000BF044
:2092C0003CFE6C487061A0693061FF206249013040394860A07A800714D52868C00708D15F
:2092E00002E06448001FEDE761484FA11A300BF024FEA07A4007286801D5042100E00821F8
:209300000843286070BD70B50021464C01256174002807D0012818D002281AD0544842A1D7
:2093200045380BE000F0C9FA52482178001F012907D0002907D011203BA140010BF0FDFD7C
:2093400070BD056070BD456070BD8120FFF791FF70BD00F0B2FA6069002804D1452032A18E
:20936000C0000BF0EAFD6169A06A40184249C86039484249403001603E490C31416008140E
:2093800035494039486027482030C57370BDF8B50C2069460870314C6068C006C50F1026F5
:2093A000A66034480021FC300161324B01221B1F1A610BE000BF00BF00BF00BF00BF00BFC2
:2093C00000BF00BF6B461A78521E1A706A461278002A02D00269002AECD0016168460078C3
:2093E000002804D1224810A131380BF0A6FD002D00D06660F8BD0B490020C861704710B5BD
:209400000BF060FC00021049000AC86310BD0B490220086070470949022008601049086066
:2094200070470000481400207372635C68616C5F7263732E63000000C01F004080E100E088
:209440008000001000170040001500405B060000001200404480004040F501400013004050
:2094600080E200E00601020025000300001600407702000004100040408500404C81004044
:20948000F74902200860CBE7F6490870C8E710B5F5480AF08BFB002803D0F449F4480BF0F9
:2094A0004CFD10BD10B5F0480AF098FB10BDF1494860B5E7EC4910B53039EF4B0022C860DA
:2094C0005A60896A0818ED49486000F0FDF910BDE54810B5C6213038C160E74A00215160C9
:2094E000806AE649C630486000F0EEF910BD0120E34940028860DC4900203039C860DF499C
:2095000048608DE7D84900203039886288E7D648DA493038806AFE30886081E7D7490020DB
:2095200088607DE7D7480168102291430160D6490120886174E7D5490020C861D148016883
:209540001022114301606BE700B5FFF7EBFFC64900203039087400BD00B5FFF7ECFFC249CB
:2095600001203039087400BDC849CA69012A01D0002055E7BF4A403292685206520E5242CB
:2095800002700020C86101204AE7F8B5BF4C2069012806D00021B44830380078012802D086
:2095A00004E04021F7E7E268012A04D000220A43012802D004E02022F9E76168012905D007
:2095C00000211143B24A002802D007E01021F8E71368012B02D1E368012B04D000230B43F3
:2095E000002802D007E00823F9E71168002902D1E168012905D000221A439F4E002802D05C
:2096000004E00422F8E77168012904D000211143002802D004E00221F9E76068012829D04A
:2096200000259C480D4301680906090E02D06169012900D000218C4F103F39730068000647
:20964000000E02D0A069012800D0002078738B488068002803D000F03BFA012800D0002029
:20966000B8730021E160216161606161A16171602846F8BD0125D4E77B4930394874CFE6E3
:20968000F8B5794E0127103EF07B0025002826D07C4C206800902560FFF779FE0098206048
:2096A0007A48C56005614560456185617449001488603446203C2178734801290BD000291B
:2096C0000BD06B486949B9300BF037FCF573607C022879D0F8BD0760F8E74760F6E7FFF707
:2096E00054FF0446604D0020303D6874634842686A620068A8622978002909D1A978002936
:2097000006D05C4B5B681B780B406978994309D000213170E10707D0104602F016FD012197
:20972000A86A08E03770F5E7A10601D5022102E0A10702D5002102F017FD4E4F79680622DE
:209740000931E81C0BF030FA002807D1687A79680978C909884201D1012000E000207070F3
:20976000204600F0BBF83F48C6260078002816D001282AD002283DD003285AD093203B4901
:20978000C0000BF0DAFB287C002804D02878002864D0FFF7C7FE2878002860D086E0A007DD
:2097A00001D501F0CDFB200703D50120EE6001F0EFFB600703D50020EE6001F0E9FBA006A9
:2097C000E1D501F06DFBDEE774E0A00701D503F005FF200703D50120EE6003F07EFE6007A9
:2097E00003D50020EE6003F078FEA006CBD503F0FFFDC8E7A007BF27002802DA3C40F9F7D9
:20980000F5FB200704D53C400120EE60F9F7EDFB600704D53C400020EE60F9F7E6FBA006F4
:2098200002D53C40F9F7E0FB6006ACD5F9F7DFFBA9E7A00701D5F9F7DDFB200703D5012064
:20984000EE60F9F7D6FB600703D50020EE60F9F7D0FBA00697D5F9F7CBFB94E71CE01EE054
:2098600000E100E0600000207814002028940000AD02000000150040408100404085004035
:2098800000F501400012004000100040001100400014004040160040FFF74DFE7BE7E868C2
:2098A000002803D0A96A091828484160687C012800D00FE7F9F7ACFBF8BD25490320086050
:2098C000881524498860ABE5224823494030C161224981611F4940154860A1E570B50546F6
:2098E000FFF7EBFF1E4CA17A080701D568071CD41C4AC80605D5507B002802D0907B0028B9
:2099000013D0880602D5107800280ED1480602D55078002809D000208A070026002A07DAA0
:209920004A0704D50122227002E00120F4E72670CA0709D0AA0705D4890705D5002803D03B
:20994000A80601D4FFF723FDA67270BD408500400012004000F50140101000404481004037
:2099600048140020681400202E48002101704170704770B5064614460D460120F7F7ACFE88
:2099800028490120284B08709E60DC601D6170BDF8B504460120F7F79FFE224901200870BE
:2099A00021494C60214900264E600321204D8902A960204F002C0AD0012C03D01EA140209A
:2099C0000BF0BBFA3E60032080026860F8BD386001208002F9E710B51248017800290ED05D
:2099E0000321134A8902916010494A680021002A03D0154A1268427000E041700170002094
:209A0000F7F76AFE10BD07480178002907D007484068002802D00C480068C0B270474078CD
:209A2000704700006100002000F5004000F1004000F5014000F200407372635C68616C5FE8
:209A400063636D2E6300000000F40040364800210170417010218170704770B506461446A9
:209A60000D460220F7F738FE01202F492F4A0870E41E14619660556070BD10B50220F7F79F
:209A80002BFE294901200870294800210160416081602849C014486010BD10B5224C207898
:209AA000002811D001202349C002886000F02EF80021002804D0012060701F48006801E092
:209AC00061701020A07021700020F7F705FE10BD10B515480178002905D000F017F8002846
:209AE00000D0012010BD407810BD10B50E480178002909D000F00AF8002803D00E480068E2
:209B0000C0B210BD102010BD807810BD08480168002905D04168002902D08068002801D008
:209B200000207047012070476300002000F5004000F1004000F5014000F4004010B5282115
:209B40000BF0BCF810BD40788006800E704740788006800EC01C70472820704770B5054638
:209B600000780A0700090001120F104328700B000BF0D4FA07050705070509050B0006240B
:209B800008E00C2406E0222404E00024FEA158200BF0D3F96878800980012043687070BD49
:209BA00000780007000F704710B50622C01C0BF028F810BD0B4610B5C11C062218460BF03B
:209BC00020F810BD10B5062209300BF01AF810BD0B46014610B50622093118460BF011F87F
:209BE00010BD0278BF23C9071A40490E0A430270704700784006C00F704702785206520ECF
:209C0000C9010A43027070470078C009704770B50C460546C11C2046062209300AF0F1FFBC
:209C200020784006400E207029784906C90FC9010843207070BD70B515460E4604461F2A67
:209C400003D9D1A1A9200BF078F920462A46314609300AF0D6FF6078AD1D80098001A906D1
:209C6000890E0843607070BD70B5054640780E468406A40E062C03D2C3A1B9200BF05DF9B8
:209C8000A41FE4B21F2C00D91F2429462246093130460AF0B6FF204670BD70B515460E4667
:209CA00004461F2A03D9B8A1CD200BF046F920462A46314609300AF0A4FF6078AD1D800967
:209CC0008001A906890E0843607070BD70B5044640780E468506AD0E062D03D2AAA1DE2063
:209CE0000BF02BF9AD1FEDB21F2D03D9A6A1E2200BF023F921462A46093130460AF081FF51
:209D0000284670BD10B504220F300AF07AFF10BD0B46014610B504220F3118460AF071FFB3
:209D200010BD10B5032213300AF06BFF10BD0B46014610B50322133118460AF062FF10BDAC
:209D40004176090A81767047817E427E080210437047C176090A01777047017FC27E080275
:209D6000104370474177090A81777047817F427F080210437047C175090A01767047017E94
:209D8000C27D08021043704781757047807D704720300279C90652095201C90E0A43027130
:209DA000704720300079C006C00E704720300279D206D20E49010A430271704720300079CB
:209DC0004009704710B505221F300AF01AFF10BD0B46014610B505221F3118460AF011FF2C
:209DE00010BD30B5411C837E0A461902D37D447E927D1B0221431343674D827D8C1FAC42A4
:209E000010D8002A0ED0082A0CD88A420AD28B4208D8817F427F08021043A91D884201D860
:209E2000012030BD002030BD00210A464254491C2229FBDB70474078C006C00E7047407808
:209E4000C006C00EC01C70472220704710B502788B07920892009B0F1A4302704278520957
:209E600052014270012908D0022906D0032905D0FF2045A1A3300BF060F810BD01210A4372
:209E8000427010BD10B502788B07920892009B0F1A4302704278520952014270012908D0B1
:209EA000022906D0032905D0FF2037A1BD300BF044F810BD01210A43427010BD00788007CB
:209EC000800F70470278FB23C9071A40490F0A430270704700784007C00F70470278F723D3
:209EE000C9071A40090F0A430270704700780007C00F70470278EF23C9071A40C90E0A43CB
:209F0000027070470078C006C00F704770B50546C1700B000BF002F90E080A0C0E10121244
:209F20000C14141212160C180C2413E0082411E002240FE017240DE00D240BE0012409E0E8
:209F4000092407E0062405E0452000240EA1C0000AF0F3FF6878400940012043687070BD28
:209F6000C078704770B5044640780E46C506ED0E1B2D03D904A109480AF0DFFF6019C01C6A
:209F8000042231460CE000007372635C756C5F7064752E63000000007A0C00003A020000B8
:209FA0000AF02FFE70BD70B5044640780E46C506ED0E1B2D03D9A049A0480AF0BEFF6119E6
:209FC000C91C042230460AF01CFE70BDC171090A01727047017AC2790802104370474172D3
:209FE000090A81727047817A427A080210437047C172090A01737047017BC27A0802104353
:20A0000070474171090A817170478179427908021043704701717047007970474173090A32
:20A0200081737047817B427B08021043704730B5411C037A0A46C479190221435379147984
:20A040001B0223437E4D00798C1FAC4210D800280ED008280CD888420AD28B4208D8D07A01
:20A06000917A00020843A91D884201D8012030BD002030BD10B50522001D0AF0C2FD10BD75
:20A080000B4610B5011D052218460AF0BAFD10BD4172090A81727047817A427A0802104305
:20A0A0007047017170470079704710B50822001D0AF0A7FD10BD0B4610B5011D082218465D
:20A0C0000AF09FFD10BD0A780273497841737047027B0A70407B4870704710B508220E30AC
:20A0E0000AF08FFD10BD0B46014610B508220E3118460AF086FD10BD10B5042216300AF074
:20A1000080FD10BD0B46014610B50422163118460AF077FD10BD10B50822001D0AF071FD1E
:20A1200010BD0B4610B5011D082218460AF069FD10BD10B504220C300AF063FD10BD0B46CA
:20A14000014610B504220C3118460AF05AFD10BD017170474171090A81717047C171090A38
:20A16000017270470079704781794279080210437047017AC27908021043704701717047C9
:20A1800000797047017170470079704710B50822001D0AF036FD10BD0B4610B5011D0822D2
:20A1A00018460AF02EFD10BD10B50822001D0AF028FD10BD0B4610B5011D082218460AF0A1
:20A1C00020FD10BD70B515460E4604461B2A04D93720194900010AF0B0FE2A463146E01C10
:20A1E0000AF00FFD6078E90640094001C90E0843607070BD70B5054640780E46C406E40EB1
:20A200001B2C04D9DF200C4980000AF096FE2246E91C30460AF0F5FC204670BD4078C006D9
:20A22000C00E1B2801D8012070470020704710B522220AF0E6FC10BD889F00004302000067
:20A240007A0C0000FEB50F4604460146064620302546C031603640350190032F04D0002F16
:20A260002DD0012F2BD04BE000206080A080E08020816081A082E085E0826874A074E0745C
:20A28000A076E076A073E07320746074019B987401232B74A88228830876E883B070688350
:20A2A000A873E87320776077019988720199087430727072B0723274B074A883FEBD00209A
:20A2C000A8822883012F52D0E08B0090608C0290C00000990AF00FFD401C80B2E8820099EE
:20A2E000192241439202914201DD401EE8827D20000200990AF0FFFC401C3080002F01D059
:20A30000022FDBD10198007AC1060198C90E017200206873221824218B5C4032D9075B088D
:20A32000DE07C90FF60F71185B08DE07F60F71185B08DE07F60F71185B08DE07F60F711850
:20A340005B08DE07F60F71185B08DE07F60F76185908891911726A7B401C5118C0B26973CE
:20A360000528D7D3002FA9D10020A874FEBD4A7F2046E030022A12D0097F022913D050A192
:20A3800073200AF0DAFD012000900290E08BA98B484300990AF0BDFCA883029898E7818853
:20A3A00000910089F1E7018A0091808AEDE770B504464034667B0546002E68D0252E66D8AB
:20A3C000002964D03E20405DA27B4843101825210AF091FC0846A1734207C908520F3C4B24
:20A3E000691820319A5C09798A4367D031460AF082FC491CCAB2002006E0002804D02918FC
:20A400004031C979511ACAB2291848235B5C93423AD320310979C943CB07DB17D21A521E5E
:20A420001206120E34D08B07DB17D21A521E1206120E2FD04B07DB17D21A521E1206120EF1
:20A440002BD00B07DB17D21A521E1206120E27D0CB06DB17D21A521E1206120E23D08B0697
:20A46000DB17D21A521E1206120E1FD04B06DB17D21A521E1206120E1BD00906C917511A4B
:20A48000491E0A06120E17D0401C0528B5DB70BDC00013E0C000401C10E0C000801C0DE0F0
:20A4A000C000C01C0AE0C000001D07E0C000401D04E0C000801D01E0C000C01DE07370BDF6
:20A4C0007372635C6C6C5F7574696C2E630000005451010010B5FF4800210170417081706C
:20A4E000C17041718171C171083009F057FB002804D0FF20F8A184300AF01FFD10BD10B5C2
:20A50000F44900204872081D09F048FB002804D0FF20F1A1C3300AF010FDFFF7DBFFF14813
:20A52000FFF782FC0021EF48FFF7E4FC0121ED48FFF78CFC10BDE2E71B207047E5494A7A2A
:20A54000002A01D000207047488101204872704710B5E0494A7A002A02D04989814201D0BA
:20A56000002010BDDB48001D09F020FB002804D0FF20D9A1B4300AF0E0FCD648001D09F017
:20A580002DFBFFF7A7FF012010BD70B5D14C0025627A002A02D06289824201D00D700DE0E0
:20A5A000227863789A4203D322786378D21A04E062782378D21A10239A1A0A70FFF7C8FFB0
:20A5C000002801D06572012070BDC2494A7A002A04D04989814201D101207047002070477A
:20A5E000BC490A784B78521C1207120F9A4207D0097822225143BC4A89180160012070477D
:20A6000000207047B34801784278491C0907090F914206D00178491C0907090F0170012067
:20A62000704700207047AB494A7A002A04D04989814201D10120704700207047A5490A7850
:20A640004B789A4207D0497822225143A64A89180160012070470020704710B59D4C207804
:20A660006178884216D06078401C0007000F6070201D09F09BFA002804D0E078401CE0706C
:20A68000012010BDA078401CA0709248001D09F0A5FAF5E7002010BD8E4801784078814226
:20A6A00001D101207047002070478A4801784278914202D30178407803E041780078081A05
:20A6C0001021081AC0B270470F20704770B5814C0D46617A002916D06189814213D1002632
:20A6E0002E70201D09F062FA002805D1A0782870A670201D09F072FA2878E17840182870DB
:20A70000E670012070BD002070BD76490160704770494A7A002A04D04989814201D101206E
:20A720007047002070476B494979002901D0002070476E49016001207047664841790029C3
:20A7400001D000207047012141710846704761494A7A002A04D04989814201D101207047CD
:20A76000002070475B494979012901D0002070475E4901600120704756484179012901D097
:20A7800000207047002141710120704751484079012801D001207047002070474D494A7AE2
:20A7A000002A04D04989814201D1012070470020704770B5474C0546A0790721401C0AF0EB
:20A7C0009AFAE079814208D0A079222148434749223140182860012070BD002070BD10B5E7
:20A7E0003C4C0721A079401C0AF085FAE079814207D0A0790721401C0AF07DFAA171012087
:20A8000010BD002010BD33488179C079814201D101207047002070472E494A7A002A04D053
:20A820004989814201D1012070470020704710B504462848083009F0B9F9002815D1254924
:20A840008879CA7990420CD0C8792221484327492231401820601F48083009F0BFF90120EB
:20A8600010BD1C48083009F0B9F9002010BD10B504461848083009F099F9002815D1154939
:20A880008879CA7990420CD0C8792221484317492231401820600F48083009F09FF90120EB
:20A8A00010BD0C48083009F099F9002010BD094810B5083009F07AF9002822D1054CA07988
:20A8C000E17988421AD0E0790721401C0AF013FAE1710DE0660000207372635C646D5F717C
:20A8E0002E630000AC1700207C1400209C1600202046083009F072F9012010BD0C4809F025
:20A900006DF9002010BD0A4808388179C079814201D1012070470020704705480838817954
:20A92000C079814201D1012070470020704700006E00002070477047FF207047704770475A
:20A9400000207047002070470020704700207047002070470020704700207047002070473F
:20A96000002070470120704700207047002070470020704700207047F8B5FE4D0446287FE3
:20A98000002600280AD0002921D1667010202070687FA070A87FE0702E7718E0A879012889
:20A9A00001D00020F8BD002911D16670F149E87901270831002801D0132000E00520207053
:20A9C0001422A01C0AF01DF9A771EE71AE710120F8BD70B5E8480078002802D00C2630469A
:20A9E00070BD0026E34D3446203DAE74EE746E75AE752E7528466E7320384673E87D0028E3
:20AA000004D0FEF78BFDFFF748F8EC75D9488471C47104772030FFF791F8D6484830FFF72D
:20AA20008DF8DCE710B5D44C00232370D14C203CE375D04B01241C71603B583307C3FFF7AF
:20AA4000C8FF002803D0CDA1FF200AF076FA10BDC8482038807C7047F8B5C64D0646407B8E
:20AA6000203DE873C34837791346AF73B27B42710446603C217006221946601C0AF0C1F8DB
:20AA8000B07960730622F11DE01D0AF0BAF8687B0126002800D0EE74B6484038407B00281E
:20AAA00000D02E753B000AF039FB050406234706490000211DE0AF4801212030FFF74EF82F
:20AAC000AC48E11D2030FFF77DF8607B002807D0012807D0FF20A9A142300AF02EFA0CE006
:20AAE000002100E00121A3482030FFF786F804E00621A0482030FFF731F800206875A87508
:20AB00009C48611C2030FFF74FF89A4821782030FFF767F8974804214830FFF71FF89548C1
:20AB2000611C4830FFF740F8924821784830FFF758F8AE740020F8BD0221DAE7FF208FA197
:20AB40004C30CAE770B58B4C0125203C0246A57588488079002801D03A2070BD854860383A
:20AB60000378934206D1002262750622401C0AF048F86575002070BD70B504467D4D002077
:20AB8000203D28752846224632380AF03AF82846203844730120287570BD764908717047F8
:20ABA00010B5744C0022203CE27460730246204612380AF026F80120E07410BDF8B500F07A
:20ABC00044FB6C4C0025203CE07D002804D0FEF7A5FCFEF762FFE575674E3570FEF762FCB1
:20ABE000A07B012804D00021084601F077FAF8BD0021022001F072FA5E4CA0790127002804
:20AC000007D0207F0028F2D105206077A5772777F8BD70780028FBD0564906226039487B6A
:20AC20006073C91D0846673009F0EBFF3C202072A7717570F8BD10B54E4C203CE17B207C40
:20AC4000CA0701D0C2070BD08A070FD582070DD42620FEF7F2FA207C02210843207410BD3D
:20AC60002520FEF7EAFA207C0121F6E74907F6D54007F4D42720FEF7E0FA207C0421ECE747
:20AC800070B53D4D2878002873D13A4C203CA07C00287DD0FEF7FBFB0026267466746E7023
:20ACA0003046FEF7F1FB0020FEF7EDF93748FEF7BBFA2546403D296E8857FEF781FA3348D0
:20ACC000C01EFEF79CFBFEF712FCFFF7B4FFFEF731FAFEF7D5FB0120FEF715FB0F210520FE
:20ACE000FEF74CFA2978681CFEF73AFAA07B01280CD004280AD0E07C002807D02146123998
:20AD00000846627B5230FEF796FFE674207D002808D0184840380146427B12398830FEF731
:20AD2000BCFF2675607D00280BD01248691C2030FEF73AFF0F48691C4830FEF735FF667528
:20AD4000A675E86D0178002903D00178001DFEF719FAA86D0178002907D00178054A401CBE
:20AD60007332FEF77AFE0120E075FEF79BFB002070BD0DE030180020740000207372635CE6
:20AD80006C6C5F6164762E63000000005F5101000C20EDE7FE494860704770B50546FEF7F4
:20ADA000A6FB002D06D00020FEF763FAFEF7C2F9FFF741FFF74C607C002809D0A07B012833
:20ADC00003D1F549F5480AF0B8F8FFF7F7FECFE7002D15D0A07B01280CD0FF202D30FEF736
:20ADE00045FA0220FEF78FFAEA4820300079012803D005E099208000F1E70220FEF73CFC38
:20AE0000E4484030FEF753FB012008F084FDFEF799F9A07B03000AF081F905040404060485
:20AE20000A00032000E00120FEF723FA04E0DB48D9492A300AF081F8E17B207C81430120FF
:20AE4000002903D1A17B012903D06074D04908708EE700212174F9E710B5FEF718FBCC488B
:20AE6000007800280ED1CB48807C00280AD00020FFF793FFF6F7A5FAC6482030007901280E
:20AE800006D007E000F0E1F9FEF70CFB0C2010BDF8F7BEF8002010BDBD490120487070470E
:20AEA00070B500F0BEFF00281BD0B94E3078B94C2034012818D0022801D0032834D0B6496B
:20AEC000B7480AF03AF83078002809D0F6F779FA3078022804D12079012801D1FEF7CCFB47
:20AEE00046E7FFF76BFE43E7AA4DA87B03281BD0FEF7EEFAE87D002803D0FEF7BEFDFEF78A
:20AF000006FBA4489030FEF7D2FA012008F004FDA87B01280CD004280AD061796F200129E8
:20AF200008D0032906D006E00120FFF736FFCAE7012000E07F20FEF79CF902203070C2E7BF
:20AF400010B59448C07D002803D0FEF7E7FAFEF7A4FD00F066FF002817D08D4C20780228AD
:20AF600004D08F488C492B3009F0E7FF0120FFF714FF2078002807D02078012804D08848F1
:20AF80008549333009F0D9FF10BDFFF717FE10BDF1B582B0FEF744F90746FEF799FD0128FF
:20AFA00029D000267A480078022804D07C487A49563009F0C2FF774DE87D002803D0FEF75A
:20AFC000ADFAFEF76AFDFEF792FA72489030FEF7E7FD0446029800286DD0FEF7CBF8002871
:20AFE00069D020466B4C030020340AF097F806646464066425640126D4E7A87B01285AD09E
:20B00000042858D0374304D16079002801D0022851D160486830FEF74AFA012008F07BFC66
:20B020000120FEF726F95A48032101702079012844D1FEF721FB41E056489030C178D038FC
:20B04000C27991421DD10146D0310A79037A9A4217D14A79437A9A4213D18A79837A9A42CC
:20B060000FD1CA79C37A9A420BD10A7A037B9A4207D10978407B4906C90F814201D10121E8
:20B0800000E00021A87B012801D0042801D1002908D100280FD1374304D16079002801D069
:20B0A000012808D13B489030FEF79BFE002802D0A87D002812D00120FFF76FFE344801781B
:20B0C00000290AD00178012907D00078032804D0324831492A3809F030FFFEBD2C4F2D4952
:20B0E000786804229F31343009F08BFD29484021903000784006C20F78680A5425490622A0
:20B100009331413009F07DFD224978680322A331383009F076FD1F483B219030827D78680D
:20B120000A541C4990310A7ECB7D12021A4382878A7E4B7E12021A43C2830A7FCB7E1102D5
:20B1400019430184134990318A7F4B7F11021943418410490522AF31243009F052FD0D4998
:20B160007F68B0310879C20638462030D20E0090827709794909C177A079002819D0207FB2
:20B18000002856D1E07900280CD013200BE0000074000020101800207CAD0000E7030000F6
:20B1A00093020000052060770020A077012020773FE0E97D2B48002924D000212172B98904
:20B1C00061814021C95D617339460622413109F018FDF88BA082388CE082788C2083009801
:20B1E000C07FA076E07E400840003043E076FEF77CFCE17E4000C907C90F0143E1760120DB
:20B20000E07115E000212172B98961814021C95D617339460622413109F0F3FCF88BA0820F
:20B22000388CE082788C20830098C07FA0760120A0710D4C0020207000F007F8FEF732F90A
:20B240000120616800F04AFF38E710B5FEF75AF9FEF74DF9FEF79BF80020FEF70AF8FEF7D0
:20B26000DAF810BD3E180020740000208107C90E002808DA0007000F08388008FA4A80001A
:20B280008018C06904E08008F84A800080180068C8400006800F704710B500F079FF10BD71
:20B2A00070B5F34C0546A26800290DD0002A04D0FF20F0A1363009F040FEA560F6F782F818
:20B2C0000220F6F779F870BD002A04D1FF20E9A13E3009F032FE0020A060F6F774F80120E8
:20B2E000F6F772F870BDE2480C30C07E002801D00020704701207047DD480C30C07E704728
:20B30000DB483430C07E70470021C176817601604162D7480C30C07E002807D1D448343045
:20B32000C07E002802D1D24901200870704710B50B46C17E847EA14204D01146184607F0AF
:20B34000A6FB10BDFFF7E0FF10BD38B5C84C606801684978012924D00121684606F050F9BD
:20B3600068460078C749000209F0C5FC60680268C0685268511807F0A7F96168C860BC49D1
:20B38000606834310022884215D0018B002912D04272032101720271021D017FFFF7C7FFFF
:20B3A00038BD7D21C068C90007F08EF96168C860B5480861E3E7018B491C0183022141721F
:20B3C000E7E7FFB5AA4E01460C36706A3468056885B060680190306A03906A880798801AA1
:20B3E00080B202900898002804D0274638372046483002E0371D284664300090032038719F
:20B40000002915D001297DD0022951D003297AD0AF2098A1C00009F090FD0898002838791E
:20B4200072D0032803D093A1984809F086FD3BE1306A002804D195488EA1723809F07DFD60
:20B440009249A88F9F3948434018069900F0A6FEA0618E49E88B9F394843069900F09EFE13
:20B46000E0618A4AA88F9F3A316A50430918A069874A091A89183B22A162844B525D9F3B02
:20B480005A4382181018FF30163020626062306A081AFF38ED213538C9008842BDD27D493E
:20B4A000884204D2794873A1653809F046FDB7E0764AA88F9F3AE16850430818069900F04C
:20B4C0006DFEA0617149E88B9F394843069900F065FEE061306A002804D16C4865A15D3857
:20B4E00009F02BFD5820405B6B4A0028A88FE16820D050430818A169401AA0622169A06820
:20B50000484302E01FE04EE0C9E0A169624A40183B21495D514341180818FF3014302062D6
:20B52000E88BE1695043411A0F208001081A6062A06A35E050430818A169401A3168D338F2
:20B5400049684018D9E7284640300190008B002802D0306A002804D14C4846A1453809F0A6
:20B56000ECFCE88B4C49E3694843C01AA06201999C460A8B2169A368521A4B43A16959180D
:20B5800063465343C9183B22525D434B5A438A185118FF31143121620F218901411A616279
:20B5A000316A401A35E00898002803D03420005D002873D1E88B38494843E169401A02990B
:20B5C0004843A062284640300490008B0028019829D0002804D02D4826A11F3809F0ADFCF6
:20B5E00004982D4A018B02980818E16948434000FF3014302062E88B5043411A0F208001D7
:20B60000081A606200F0C4FD00281CD0A16A0398081AFF38ED212338C900884200D3FCE6D1
:20B6200002203871F9E6002802D00398002804D1164810A1263809F080FC0198A16AD3383D
:20B640000818A062CCE706F0A8FD0146706907F0CDFFA16A081AFF38ED211E38C90088423C
:20B66000DDD2012009B0F0BD00ED00E000E400E0C81800207372635C6C6C5F6C6D2E73307E
:20B680002E63000010270000B78913008105000036040000A3020000E20400002AE003280F
:20B6A00002D1FD4907200870A16A706907F00CF8B860616A206A884202D90098016001E007
:20B6C000009908600098F54900680818F860A9880798081A00B2002801DD022000E00020E7
:20B6E0007871089838700898002805D03420005D002801D00220B5E7089801214840203476
:20B700006075317F3A463046FFF711FE0020A9E710B5E14900284A68516A096807D01268B3
:20B72000C98BDF4BD2695943891A09F0E4FA10BDF8B5D94F35227868416A0C680168525C2B
:20B74000002A0AD0498E6288914206D1407A002803D1D449D44809F0F0FB06F01EFD01464F
:20B760007868406907F042FFFFF7D2FF796865880B682E185A8EB24202DB521C5A8602E0D1
:20B78000401C2818588608683622125C002A05D1428E23899A4201D1521C4286088B0328DB
:20B7A00002D2401C088302E00868408EA08020464030C18A808A081A6188401E401885B26B
:20B7C000203416E0496AE67F097976004B00B749007DCB5A895BC91889B20023FFF7F1FD1B
:20B7E000002811D0012810D0AF48AE493A3009F0A4FB79680868428EAB1A1BB2002BE1DAAE
:20B800000820E07400F00DFEF8BD78680068418E491C4186EDE770B59F4D1F202870A868ED
:20B8200000210162C27E130009F078FC045454034654426A146802681170026851600068E5
:20B840002030407D002808D106F0A7FCA9680968096C07F0CBFE002815DCA86801684A8E20
:20B8600061888A4204D12289511A6181628004E0511A61810168498E61800268C16811640A
:20B88000C16841610FE0A8680168098E6288891A61810168098E618001680A6CC2600A6C17
:20B8A0004261886C6066204601F06FFC00280ED07B487C49D33808E0C1684161FFF7E0F94E
:20B8C000002804D076487749CD3809F036FBF5F778FD70BD72487349C638F6E710B56E4A63
:20B8E0000B00526809F01AFC0906090F1F0C2D2D082A2D00FFF78FFF10BD00F05DFC10BD02
:20B90000FDF7BEFE10BDD07E022806D0D07E032806D00120634940020DE0FFF709FF10BD46
:20B92000FFF713FD10BDD07E0228F6D0D07E0328F6D05C495E4809F000FBF1E706F013FC9B
:20B9400010BD5B4857490F3009F0F7FA10BDF3B581B0514C02982546002601270C350300D4
:20B9600009F0DCFB0906313C3C3143433C3C4300494801210C30FFF793FC02990198FFF72F
:20B98000ADFFE87E022828D1A0680468406A066806F0E2FBF18B424A5143E269891AD3397D
:20B9A000FF223232E162904202D24248081802E0081A41494018E0624048E16A814200D8D9
:20B9C0000846E06206E001460198FFF787FFE87E022802D1286820300775FEBD014665600F
:20B9E0000198FFF77BFF6660FEBDFF202D49AB3009F0A3FAFEBDF8B5064627480D4600241D
:20BA00003430254F0B0009F089FB09060C10100C161610101600204801213430FFF740FCFD
:20BA200029463046FFF75AFFF8BD78603046FFF755FF7C60F8BDFF201A49DF3009F07DFAF3
:20BA4000F8BDF0B5144C0020616885B003268E76CA7E0746032A03D0C97E00293FD03FE0AE
:20BA6000087F002804D112480E49CE3009F065FA6068057F684606710221417106F08DFB77
:20BA80000290FF20F53003900121684601706946284606F0FCFF14E0C818002019170000CA
:20BAA000E204000074B6000062060000645101000B0200007CF8FFFFADF9FFFF38120000EB
:20BAC00020BF6068007F07F01DFE0028F8D06068007F06F048FB60680777FFF715FC012050
:20BAE00061688F7605B0BEE5FE494A68907600E020BF4A68D07E002803D0D07E937E98422E
:20BB0000F6D0D07E002803D000200021917670470120FAE770B5F34900240C31CA7EF14DCD
:20BB2000032A03D02831CA7E032A17D16960002810D001280AD0EC49EC4809F0FEF9002002
:20BB40006968002C0860686008D070BD0320FFF7CBFF01E0FFF775FF0446F0E70C2070BD0B
:20BB6000F8B5E04F04461F25E67E330009F0D6FA042A20031B20DB480C30844203D0DA4954
:20BB8000DB4809F0DAF902207C60FFF7ADFF002805D07968002008604862786012E00C250B
:20BBA000002078600BE00120FFF7B4FF054604E0CF48CD490C3009F0C0F9002D02D0E07E31
:20BBC000B042D1D1E07E002804D0C948C649123009F0B3F9F8BDC34810B50C30FFF7C0FFFA
:20BBE000C0483430FFF7BCFFBE4900205C310875C0494870BB490C3148610A4628325061F1
:20BC00008876907601220C390A708860486010BD70B504460120FFF729FBC5B20B20FFF79F
:20BC200025FBC0B2854204D0B148AF49343809F084F90120FFF71AFBC5B21820FFF716FB22
:20BC4000C0B2854204D08920A749800009F075F90420C043FFF70AFBC5B21920FFF706FB8E
:20BC6000C0B2854204D0A2489F49323809F065F9A0489C490C38047000200C31C876887606
:20BC80000A462832D07690769A4B0124083B1C7118604862506208601060FFF79CFF70BD6A
:20BCA0009048007870479349083908717047F3B50D468C4983B00C31CA7E08462830894C2D
:20BCC000002A02D1C27E002A03D0C97E022903D005E08948616006E0C17E002901D00C2023
:20BCE00000E76060854806F0EAF961680877606880490160007F002804D17C487A49623820
:20BD000009F01BF906F028FA7D49884200D20846FF30C83086B260680321C1760027012D77
:20BD20002FD0734A03991A32514302685160006801210170684605F063FC684600787149D3
:20BD4000000208F0D8FF019106F027FA0199711806F0BAFC6168032DC86021D06A4808616D
:20BD6000606803210172022141720771021D017FFFF7DDFA606807830720207000206760BA
:20BD8000B0E606F00AFA314606F09EFC6168C8605E48086108680770096801204870DFE715
:20BDA0005B48DCE77047F8B54E4E0C36F17E002904D131462831C97E002901D00C20F8BD7C
:20BDC0000221F176474C4B4F5C34083F77623460002538602575397920304A004D49C07FF0
:20BDE0008A5A4000085A2B46101881B22A462846FFF7E7FA002804D03C483B49323009F0DD
:20BE00009CF825610120A56020756586258635487C30857539684888401E48803583002025
:20BE2000F8BD10B52F4801248068817E03290CD001684978002906D0006A3749884202D945
:20BE40000024FFF729F8204610BD0024FBE72548806802681178491C1170016A0068C26A41
:20BE6000914204D8007D012801D0012070470020704700207047F8B51A481A4C0C306060A5
:20BE8000416A00260D68006834212F460E544037B97C002966D1007D032863D106F07DF974
:20BEA00001466068406907F0A1FB00285ADDFFF72FFC6988401C41186068026811860068E0
:20BEC000018E2A89511A09B200294BDD012120308175F88AB98A401A6988401E401887B242
:20BEE00039E00000C818002074B600007703000057020000880000204FB90000F7B90000CC
:20BF0000F605000010270000F7130000B7891300E2090000645101002C841300496A0979F9
:20BF20004A00CE498B5A028E007D94463F22525D5200895AC91889B201236246FFF741FA76
:20BF400000280FD001280FD002280BD0C920C449C00008F0F2FF61680868028EBA1A12B2CD
:20BF6000002ADBDA6660F8BD60680068018E491C0186F0E7F8B5BB4D0026AA680128516A14
:20BF80000C6810D00720287006F052F8B6480078F6F7E8FDA86806830268618851860068DB
:20BFA00020308675F8BD087913684100AB481F7D415A032F17D01A7D022A21D01A7D012A8B
:20BFC000E2D13F231B5D22895B00C05A0023401881B20120FFF7F5F90028D5D0A049A34860
:20BFE00008F0ABFFD0E71E6112683F2396601B5D22895B00C05A0023401881B20320E9E75E
:20C000005822125B1A613F231B5D22895B00C05A0023401881B20220FFF7D3F9AA680121FE
:20C0200012681175D8E738B58E4C0021A0680D4600684278002A01D045701FE0007800288D
:20C0400009D00121684605F0DBFA684600788849000208F050FEA0680268C0685268511871
:20C0600006F032FB0146A068C160057102214172021D017FFFF75BF9A068058305F0D8FF9C
:20C0800079480078F6F76EFD38BD10B50146754A0B00906809F042F8060D150408190C1CA4
:20C0A000012100F0A8F807E00021506800F0A3F810BD0120FFF75EFF00210846FFF7F0F8F5
:20C0C00010BD00680321017510BD00F0A7F810BD3D206349400108F030FF10BD70B5614C58
:20C0E000002809D0012816D0022821D05F485C49C73008F022FF70BDFFF795FF0021084693
:20C10000FFF7CEF8A068807E002801D01F2000E00720207070BDA068002501684D70FFF718
:20C12000F3F80320F6F763FC05F082FFA56070BDFFF779FFA068FFF7E7F800210846FFF74D
:20C14000AFF80420F6F753FC70BD46498968CA7E022A08D10A681378002B04D150600968C0
:20C16000CA6A1018C862704710B53E4A002992680CD0012907D0022907D03C483849E73017
:20C1800008F0DBFE10BD401E00E0401F106210BD34488068002800D00120704710B50446E2
:20C1A0000020002907D0334808F0A5FD0146204608F0A1FD401C10BD10B52A488068C07E81
:20C1C000030008F0ABFF041414030A1401F0E5F800280BD02249284806E0FEF73DFE002883
:20C1E00004D025481E49001D08F0A7FE10BD22481B490B30F8E710B50446002903D00020FD
:20C20000FFF7B8FE03E018480078F6F7ABFC2046FFF77AF80020F6F7EAFB10BD10B5114878
:20C220008268506A11680068CB698B60124BC18BB13359431368D9600146E0314B88838748
:20C240000C783B231C548B88C383CB8803840989418411680220087510BD00006451010067
:20C2600074B60000C81800207C000020FD0600001027000040420F0031040000F8B5FEF756
:20C2800014FA0646FEF782FAF94D07466879F94C002809D0012823D0022826D003282ED0B4
:20C2A000FF20F5A1C63033E0F2481830FEF75AFA002801D003200FE0EE481830FEF7BEF9C0
:20C2C000002804D060696030007A002806D0E9481830FEF71AFA012068711BE00220FBE716
:20C2E000E4481830FEF711FA14E0E2481830FEF7A5F900280ED1FF20DFA1B83008E0DD4836
:20C300001830FEF72FFA002804D1FF20DAA1C03008F013FEA169F722087810400870AA7999
:20C32000D207120F1043FB2210400870EA79D207520F104308706B79EF22022B04D0012B41
:20C3400007D0032B07D00CE0012E06D8002F04D007E07F1E3E43002E03D01040102210432A
:20C3600000E010400870287C002811D0687901280ED0BF485438FDF79AF8BD49606954390B
:20C380007830A269FDF7F5FA0020FDF701FB04E00846FDF78CF8FDF71EFBA0690078C006F9
:20C3A00006D4E0690078C00602D4E079002802D0A079002801D0012000E00320FCF759FF72
:20C3C0000320207001202071F8BDAA4810B51C30FEF7EFF9A74C002802D00020607004E0A2
:20C3E00001206070A2485438E061A148407C002802D06078002805D0E069FDF758F8FDF7A0
:20C40000EAFA10BD9A485438FDF751F8984A6069543AA030E169FDF7ACFA0120FDF7B8FA0C
:20C4200010BD10B593490022486932238276C27601221A544030807C002803D00A700021A3
:20C44000022001E000210320FFF71FFE10BD70B5884C6079C2062046416908464030002A23
:20C4600001DA002202E0028B4B89D2180B460283C0331A7E002A03D0828B4D8952198283E1
:20C48000627A002A03D03D2001F0BEF852E08A7E032A4FD0227A002A13D0500701D4D0068E
:20C4A00001D51E2036E0100701D53D2032E0D00705D1900703D470A1734808F03EFD2A2092
:20C4C00028E060318A78002A05D0C28B551CC5830D88AA420FD25A7F062A02D01A7F062AB6
:20C4E00005D1428B531C438309888A4203D2828BC18A8A4201D322200CE0027C808A002A5A
:20C500000FD006280FD35A48C07B012801D03E2000E0082001F078F86069807E032809D0C3
:20C5200001E08842F5D20120207000210846FFF7ACFD70BDFFF775FF70BD10B54C494D4817
:20C54000CA7B002A2BD0012A29D0022A27D0032A04D049A14D4808F0F0FC10BD897B0229CA
:20C560000FD007291BD0406901464031CA8A898A511A891E89B2032900D303210289511895
:20C580000BE04069014640318A8A032A01D2018903E04288C98A5118491C818010BD40696C
:20C5A000F5E700B5030008F0B9FD0604070B0F12121700290ED00FE0491E02290AD90BE07D
:20C5C000491F012906D907E0072903D004E00A390C2901D8012000BD002000BDFEB5054612
:20C5E00024481830FEF79FF8002804D1274822A1CF3808F0A2FC1F4CA069FDF715FC032192
:20C60000A069FDF73FFCA069EF220178114001702946FDF77BFC002601272B0008F07EFDC7
:20C620000E5D5D085D1D6161155D4D5D613D385D60697121095C002901D0062101E0C030ED
:20C64000417EA069FDF72DFD4BE0E069FDF788FC0146A069FDF796FD43E06169A069D0313A
:20C66000FDF759FD6169A0699531FDF762FD38E0C4190020900000207372635C6C6C5F7371
:20C680006C6176652E6300006B020000780800000621A069FDF772FD23E020690178A069D3
:20C6A000FDF756FD20698188A069FDF753FD20694188A069FDF752FD13E0009601966069CD
:20C6C0006030007C002803D069460878384308706946A069FDF768FD03E0FE49FE4808F0B8
:20C6E0002CFCFEF72AF8002804D1FB48F949801D08F023FC0C2D07D0072D04D060695E2165
:20C700000E5260308770FEBD606940304683FEBDF0B5F24CDC2061698DB0405C042809D033
:20C72000052834D16031487A002829D001204874022026E01022EA31684600F09DFF6169FD
:20C740001022C83104A800F097FF684605F0B1F8616908AA6CCA0F46CB6778378A67084609
:20C76000FE608030BD60074620376CC70023036343630120A0310876D9494874052000E035
:20C780000D20FFF72BFF61690020C03108770DB0F0BDF8B5D1481830FDF7C5FF002842D088
:20C7A000CE4C207A00283ED160690025C030007ECB4E00280BD0B17B0120FFF7F2FE0028BB
:20C7C00005D1B17B0420FFF7ECFE002806D060690127C030407F062807D00CE060695C217E
:20C7E0000D526030457402202FE0B17B0420FFF7D8FE002810D0B07B030008F08FFC173F35
:20C800003F3F3F1E3F3F3F3D3F203F3F3F292C3F3F3F3F3F3F2F3F0060696A21095CC90761
:20C8200002D0C0304577F8BD0C20FFF7D7FE60696030817A39438172F8BD072005E0FDF756
:20C84000E2FF0028F8D075740B20FFF7C7FEF8BD00F021FFF8BDFFF75BFFF8BD60690021CF
:20C8600080308160C160057437740620FFF7B6FE606960308570F8BD0920E6E700F0CDFE5E
:20C88000F8BD70B5964DA87B072834D1934CDE2260694188125A491C91422CD1217A0029AE
:20C8A00029D10146E0318B88C28B934207D1CA88068CB24203D10A89468CB2420DD0884A65
:20C8C0008689303A56819381CB88D3810989118201462E3151600121117001221146FDF7C0
:20C8E000B1FC00210420FFF7D0FB61690020C0314877A873E87370BD70B5794CA07B162805
:20C9000003D07449774808F018FB74480021426973486032117291703038067E0B25012324
:20C92000002E06D0027D002A12D14575817503750EE0567A002E06D0517222888283817614
:20C940000C22027604E022888283817683770576A17370BDF8B5614DA879800723D5287A54
:20C96000002820D15E4C0120A17BFFF71AFE002819D1A8690127C0780026030008F0CEFB3C
:20C980000E626208622E3B4F0A62146220524562022021E0A07B042804D052484D493338CF
:20C9A00008F0CBFAA673F8BDA07B082804D04D4848492D3808F0C1FA686960308670F1E760
:20C9C000A07B0A2804D047484249263808F0B5FA6869603007720B20A073F8BDA07B0E28F9
:20C9E00004D0AB203B49C00008F0A7FA6869603007720F20F0E7A07B0F2804D039483549B6
:20CA0000183808F09AFA1120E6E7A07B0F2804D034483049123808F090FA1320DCE7FFF769
:20CA20006BFFF8BD69690846C0310A7F062A04D16030807A800700D50E77487F0628F0D117
:20CA40004E77F8BD274823496E3008F076FAF8BD10B5234C0020A17BFFF7A3FD002804D1C3
:20CA60001E480122017A114301720420A07310BD10B51A4C60690146C0314A7F002A06D0F2
:20CA8000097F062903D0217A0122114321726030807A800715D4E069FDF764FB6169603176
:20CAA000C872E069FDF760FB616960318881E069FDF75FFB616902226031C881887A10438C
:20CAC0008872606900220146C0310B7F062B00D10A7709E078C60000ED0700009000002061
:20CAE000C4190020770500006A231B5CDB0703D106234B774030428310BDF8B5FE48817B27
:20CB00000020FFF74EFDFD4C0126002807D160696030407A002802D1207A304320726169CD
:20CB200000255E20455262204654C831E069FDF7DAFA6169E0699131FDF7E4FA61690422FE
:20CB400008469131B93008F05CF8EB483038017E0827002906D0017D002912D14775857508
:20CB600006750EE06169054689894183E249E0691439FDF7A0FAE049E0690C39FDF7A8FAC5
:20CB80002F76DD480E218173F8BD70B5DA4D0020A97BFFF706FDD94C002803D1207A01218D
:20CBA00008432072E069FDF742FA00280ED0E069FDF738FA6169DE225052498800F0B6FDCA
:20CBC000002806D0282000F01FFD70BDFFF740FF70BDE069FDF720FA6169E0310870E06981
:20CBE000FDF713FA6169E0314880E069FDF7F2F96169E0318880E069FDF7F5F96169E03180
:20CC0000C880E069FDF7F8F96169E03108810720A87370BDF8B5B94CA079C0076FD0207A60
:20CC200000286CD1B44D0120A97BFFF7BAFC002853D1E0690027C178022201260B0008F05A
:20CC40006DFA0D161308354A4A384C474A1929444A00FDF728FA6169DA225054AE735E2062
:20CC6000475260318E7038E000F06BFD35E0FFF78CFF32E0A97B0020FFF793FC002802D1B0
:20CC8000207A3043207260695E210F52603086700A2018E0A87B0B2802D0207A10432072FD
:20CCA0002F746069603046720C200CE0FFF725FF13E0A87B112802D0207A10432072606925
:20CCC000603087701620A87307E0FFF7D1FE04E000F004FD01E0FFF7BBFEFDF780FD0028D2
:20CCE00004D14F208649000108F027F9606900238030016B426B491C5A4142630163F8BD95
:20CD0000F8B57D4F012814D1787C002802D1387C002801D0FCF75FFEFCF7F4FBFCF7E7FBE9
:20CD20000020FCF7A6FAFCF732FBFCF774FBFCF7B9FBF87B01260025704C00280FD16079BB
:20CD4000C10705D00220F87360694030057402E0800717D5FE7300210120FFF796F9F87BF7
:20CD6000012802D0022808D00CE06079C00709D00220F8736069403005746079000701D55C
:20CD80000320F87300F00EFDFFF703FD2079002801D03D8102E03889401C38816079C0076C
:20CDA000606904D072210D544030858203E04030818A491C8182E079002806D061696031F3
:20CDC000887C022806D8401C887460696030807C022804D93D817D81606960308574B97B51
:20CDE0000020FFF7DEFB002802D1B87B06284BD160690146C0310A7F062A45D0497F062906
:20CE000042D03D49C97B03293ED16030807C00283AD1FDF741FC002836D0FDF7B7FC00280E
:20CE200032D06169C88801282ED90A4640325674D08A978A831E9F4201DB012002E0C01B63
:20CE4000401E80B22C4B1F89A3899F4201D3012302E0DB1B5B1C9BB2984200D91846012848
:20CE600000D155742A22525C002A11D0224A898D52898A4201D3012102E0891A491C89B2CF
:20CE8000884205D9084603E06169012040314D7461694A8810180881FFF74FFB6069122212
:20CEA00015490C3007F0ADFEFFF7D1FAFEF7E1FF00280AD0104810388179002905D161693B
:20CEC00002468989203A118586710C481C30FDF7CEFC00280FD0E06900788007800F0128AC
:20CEE00009D0022807D0FDF7E2FC002803D10449044808F022F807E0C4190020900000204B
:20CF000078C600007F030000606940308574F8BD70B5FE4C607900283CD0FD4D022810D199
:20CF2000FDF79BFB002803D1FA49FB4808F005F86A69002380329068D168401C5941D160F0
:20CF40009060002666712079012804D12671A87910210843A871E078012816D1E670A87921
:20CF600008210843A871FDF707FC002804D1EA48E849183007F0E1FF6969002380318A6816
:20CF8000C868521C58418A60C860A079012802D00120A07170BDA67170BDF8B5DC4CDB4D94
:20CFA000E26900271078042183079B0FE8790126012B11D0022B0FD0032B01D0207A30E0D4
:20CFC0006178002905D1AE70A1793143A17123E0EF71F8BDEE71F8BD5278D3061CD0607828
:20CFE0000028F8D1D006C00E1B2818D8607908436071FDF7F4FB002804D1C748C5494B30FC
:20D0000007F09BFF606900238030026B416B521C594102634163E8790128DBD1D8E7207A2A
:20D02000102108432072F8BDF8B5B84D0446303D287D002700280AD0002978D1677010207D
:20D040002070687DA070A87DE0702F756FE02878002814D000296AD1072067702E462070D1
:20D06000083607E0686807802F700A223146A01C07F0C7FD28780028F4D1A77057E0287EFA
:20D08000A24E143E002837D0002950D1297EA0480B0008F043F80D2C2C2C2C2C2C2C2C118A
:20D0A0002C2C20082C0067700C212170A97EA17040698089A08018E00821677021704069F3
:20D0C0000A468089914960801439201D07F099FD3089A08109E067700B212170A97EA17097
:20D0E00040698089A080A87FA0712F761FE089498A4807F022FF1AE0844810388279002A93
:20D1000008D0002913D1677011212170B189618087710CE0827A002A0BD0002907D16770B8
:20D1200012212170318A6180718AA18087720120F8BD0020F8BD76480078012801D00C2073
:20D14000704772490020303908700875087620318871704770B56E4C064620780D46002822
:20D1600004D093206B49000107F0E7FE01202661E07225622070FFF7DEFF002804D0674808
:20D180006449493007F0D9FE70BDF8B5604C2178012902D12178012901D00C20F8BD0146C3
:20D1A0000546606112220C31584807F02AFD01274035AF74554D2888FDF735FA002827D0E0
:20D1C0002888FDF7EBFA002822D02888FDF7A0FA00281DD02888FDF7BAFA002818D0FCF7FE
:20D1E00056F960690026C088002825D048481830FDF799FA00281FD06069C030007E0028B7
:20D200001AD0A97B0120FFF7CCF9002802D013E01220F8BDA97B0420FFF7C3F900280BD152
:20D22000606901464030868360314E740220FFF7D5F96069403046743448303800780028B5
:20D2400004D16169C88D098C884201D86069008CA08160694189491E8AB2298989182981F9
:20D26000297B002902D06E812E7302E0698989186981014640318B8A9B188B82C388012B1C
:20D2800001D85B1CC380002A01D060308674A87B032816D0487C002815D02889A1898842CC
:20D2A00011D2FDF7F9F900280DD060692A21095C002908D06989808D814204D3A670E77020
:20D2C00003E0A77001E0A670E670606951210E54A97B052901D0062915D1DE214288095A06
:20D2E000511A09B200290EDB01460522E0312430F3F76AFF012202216069FCF7A3FF606963
:20D30000C0304677AE736069418909E0C41900209000002078C6000039070000F10800009F
:20D32000FDF745F8A07800282AD160692030807A002800D06E810120FBF7A5FE60693830A0
:20D34000FCF75DF860693430FBF76EFF216A00200856FBF735FF0120FCF796F8FBF7EEFE4A
:20D36000FCF78EF80120FBF7CEFF6069406EFCF7A1F8FFF72AF860694030C07BFBF75DFF77
:20D380006671E671A6712672A6726672267102202070FCF787F80020F8BD10B5F74C207890
:20D3A000022801D00C2010BDA078002803D00020FFF7A6FC17E0FCF76AF800F01DF9606993
:20D3C0002030007C012809D0FCF7BEF8FBF7BBFEF3F7F7FFE07A012803D004E0FCF7BCF86A
:20D3E000F4E7F5F715FE002010BDE449C872704710B5E24C2078032803D0E149E14807F075
:20D400009CFDE14801218278002A06D0002282700171A27904231A43A271A2691378DB4342
:20D420009B0707D1C378002B04D1C170A07902210843A0711078C00606D4E0690078C006BF
:20D4400002D4E07900280CD06078002809D1A079002806D1FEF7FBFC002802D0207A0028FF
:20D4600003D00120FFF74CFC03E0FEF7AEFF00F0C3F82078012806D0F3F7A3FFE07A0128A4
:20D4800001D1FCF7F9F810BD38B5BC4C60692030007C012820D1A07A00281DD16846FCF794
:20D4A00063F8002818D061693120405C012810D1B54A0D236D460020D3562856834208D0FA
:20D4C00050738989303A918511462031887301208872A07A401CA07238BD70B5A74C064658
:20D4E0002078042804D0A748A549553007F025FD607910210843A44D6071002E47D0FCF7CA
:20D5000082FA61780126084300280ED1687C00280BD0E0694178C90607D00078E9790007CD
:20D52000C00F884201D1667247E0E078002809D0E0694178C90605D10078C00602D4FFF777
:20D54000A3FF3AE0FFF7A0FFE069A97900784007C00F884205D0FFF7DBFC607908210843C8
:20D560006071E069E97900780007C00F884201D1FFF713FD6079304360710020E071A07998
:20D58000000702D5A87B022817D0207A13E0022108436071E079401CC0B2E07101280CD828
:20D5A000687C00280DD0784854384078C106C90E052906D2C006002803D00120FFF7A0FB67
:20D5C00001E0FEF75BFE2078012806D0F3F7F9FEE07A012801D1FCF74FF870BD10B5674874
:20D5E0000078042804D067486549B73007F0A5FC0120FFF785FB10BD10B50720FBF739FE5E
:20D600005E490420087010BD5C493322496950545D4A032090738876704710B5574C6069F7
:20D62000C030007F00281CD0062806D05648817B0020FEF7B6FF002813D060690146C031F3
:20D640000A7F130007F06AFD070D0D0D0D0D0D050D006030807AC20704D0C043800700D1E7
:20D66000087710BD0C20FEF7B9FF606901226030817A1143817210BD10B5002A0AD000230E
:20D6800006E0D41A6418203CE47FC4545B1CDBB29342F6D310BD10B503F0B1FF0C281CD369
:20D6A000364C08216069D03003F0AAFF002806D060690421953003F0A3FF002803D130499F
:20D6C000324807F03AFC6169042208469531BD3007F097FA0420FEF781FF10BD7CB52A4E1B
:20D6E0000020B17BFEF75DFF0125244C002802D1207A284320726946E069FCF75BFD684674
:20D7000000780021C207D20F684602706069002A02D06030057401E06030017460695E22A9
:20D720001152603085700820B0737CBD401A184900B2884201DC002801DC0120704700206C
:20D74000704770B5104D0020A97BFEF72AFF0B4C002803D1207A012108432072E069FCF706
:20D760009BFC6169DE2250524988FFF7DFFF002810D02820FFF748FF70BD00009000002097
:20D7800078C60000320A0000C419002062060000FE7F00006169E069E031FCF771FC052084
:20D7A000A873E9E770B500F047F8384C384D6079400709D5A97B0520FEF7F3FE002803D0F9
:20D7C000207A082108432072FFF724FA00F012F8FFF7C0F8A079C00609D5A87B030007F013
:20D7E0009DFC06060606060604060620A873FFF748F8C1E710B525488179490714D5017A63
:20D80000002911D12249897B0B0007F087FC080D050D0D0D0E0D100D4069002262210A54E4
:20D82000C030807EFFF7F0FE10BD012100E002214069C030417710BD10B5144881790907DB
:20D840001DD5017A00291AD1114A947B230007F065FC1416160B161616161616161616163B
:20D860001616161616161716406960308170407C002801D0062000E01620FFF7C5FE10BD56
:20D880004069603001728170917310BD90000020C419002010B5031D03600020521E04E0B1
:20D8A0005C181C60401C2346C0B29042F8DB0020186010BD01460A680020002A02D010460C
:20D8C00012680A60704702680A6001607047000000B51A2822D00ADC030007F01FFC0D11BF
:20D8E0001F131F1F191915171F1F1F1B1F002A2814DD3A38030007F011FC030F11091100CA
:20D90000002000BD1E4800BD042000BD0D2000BD0F2000BD082000BD112000BD032000BD9D
:20D9200010B50C46F4F7CFFF00281AD02046F4F7CCF9002812D020780E280BD00F2809D02C
:20D94000022807D0032805D00EA1772007F0F5FA002010BDA078FFF7BBFF10BD09A17D20D1
:20D96000F4E708A18320F1E710B5F4F735F910BD10B5F4F7AAF910BD10B5F4F78CF910BDDB
:20D98000023000007372635C686F73745F6863692E630000F0B597B00021032004F082F930
:20D9A0000025FE4E022775807574347C12E0F068E1004018818800290CD0858069460F707B
:20D9C0004D700168029180886946888000216846F8F734FD2046641EE4B20028E7D117B0BB
:20D9E000F0BDEE4BD86019741A80D3E7EB49EC4B4A8800201A4200D00120497C002901D0BF
:20DA0000082108437047F7B504460E4600780121E34A8140521C114098B0E04A009151886E
:20DA2000E04B994205D0009B002B05D0DC4B194202D001201BB0F0BD009BD84A1943518099
:20DA40001A9D002D11D00020287022781A980027401C130007F062FB10EF0D152137555DE8
:20DA60006A39AFAB85B3EEEDECEF0B28EDD00420E0E702212970A1880170090A41700320A3
:20DA800093E004212970A1880170090A4170E1888170090AC170052087E006212970A188E4
:20DAA0000170090A4170E1888170090AC17021890171090A4171A289E81D216907F0A1F868
:20DAC000A089C01D71E0082129702178082901D110212970A1880170090A4170E18881700F
:20DAE000090AC1700520308020466A1D01A9083003F0CFFB00287DD16946308809794018CA
:20DB000053E00A212970A1880170090A417003200AE00C212970A1880170090A4170E18816
:20DB20008170090AC170052030809DE0A08884464000401C81B2308888425BD3052959D393
:20DB40000E202870002008E0A36842009B5A521953701B0A401C937080B26045F4D33180B4
:20DB6000B6E08E49487C002873D0401E4874C86821790822C9004518A9882868401808387C
:20DB8000A16807F03EF80221684601710021417128680390A98868460181002101A8F8F7FC
:20DBA0004DFC0020A880002E00D0308090E0297880221143297029784022114329702978F5
:20DBC0008909890112312970A1880170090A4170E288E81CA16807F014F8E088C01C308081
:20DBE0002878410640D5C00972D0012168460171002100E02BE041713188ED1C091D0181B4
:20DC00001A980390E08840190490001D634D0590297C68460176002101A8F8F70FFC07462D
:20DC200030880C303080022F06D0002F50D060E03CE032E01CE059E06946097EE868CA00F7
:20DC400080182A7C914202D28188002902D004274FE02EE0697C491C69741A99016031887F
:20DC600081800020308044E04C48A188C1802FE029788909890116312970A1880170090A58
:20DC80004170E1888170090AC1702289681DE16806F0B7FF2089401D46E728788009800133
:20DCA000183028702079687002207EE73B480A0401D405271DE00289A3889A4201D006276D
:20DCC00017E01E222A70012249043280490C4180009800280DD0314D002228881146830074
:20DCE000032003F03AFF2078287107E00020308003272A48009942888A434280384699E662
:20DD0000F7B59AB002000C4606D0172A04D82348244B4088984202D107201DB0F0BD23783B
:20DD20005D0601D4DB0901D00820F6E700236D462B706B701D462378611C9F06931E189329
:20DD4000531E19939BB2169302AB1793134BBF0EDE883B0007F0E2F9208511F15EF16BF169
:20DD6000A3F1C6F1F2F1FBF1EEF1EDF1ECF1F1F1EBF1EAF1E9F1E8F185F1052A71D1042296
:20DD800069460A7005490A7969460A71E178A3780A021A436946CA80227905E0D8190020F8
:20DDA000FE710000FFFF00004A7061788906890E0C2923D009DC891E0B0007F0AFF90913C3
:20DDC00052155219521B521D520012291CD004DC0E2915D01029D1D114E0162916D01829EB
:20DDE000CCD115E0800700E04007002839DA2AE10007FAE7C006F8E78006F6E74006F4E78C
:20DE00000006F2E7C005F0E7C004EEE78004ECE74004EAE7800724D5032AAFD105206A4680
:20DE20001070487809780002084390800BE14007F1D5062A15D31898617880B2012902D0FC
:20DE400002299BD101E0022700E01027062269460A7000228A8001AEA11C0236BA1C17926A
:20DE600018E0B6E04A780B7812021A433280801E891C1890B21C1691384603F0E4F916994F
:20DE800018986B469A88C919C01BB61D521C9A80179A80B28242E5D900289CD1D3E0000733
:20DEA000B9D51998694682B20720087000208880601C891D11E0437806781B0233430B800F
:20DEC000C37886781B0233434B806E46121FB388001D091D5B1C92B2B380042AEBD2002A45
:20DEE00077D1B0E0C00674D5022A72D31898082182B2684601700021C18063780371A01C31
:20DF000017990EE04678077836023E430E80861C4E606F46D21AFE88C0180831761C92B281
:20DF2000FE809342EED9DAE76FE076E065E051E046E01EE014E00AE000E0A0E0800648D5E6
:20DF400009206A46107096801698D0800FE040063FD50A22684602708680169AC28006E0E1
:20DF6000000636D50B206A46107016989080029169E0C0052DD5022A7FD318980C2182B245
:20DF8000684601700021C18063780371A01C179913E04678077836023E430E80C678877891
:20DFA00036023E434E80061D4E606F46D21AFE88C0180831761C92B2FE809342E9D98EE771
:20DFC000C0045AD5012A58D10D2168460170868039E052E0800450D5052A4ED30E23684684
:20DFE00003708680C8788B78010219436846C180521F0281601D039025E040043DD5012A8D
:20E000003BD10F20694608701DE0030435D44B780E781B023343244E3381032A2DD31B2F18
:20E0200027D011236E46337001261F4BF6033043588048780B780102194368468180D21E48
:20E04000C280E01C029020788006800E1B280AD01D2808D00021032003F024FE124841888E
:20E06000C90BC903418068461C99F8F7E7F9284653E610206B461870DBE70725F7E7082504
:20E08000F5E700B50022D243074997B04A80032807D1032268460270097901710021F8F70B
:20E0A000CDF917B000BD0000D8190020FFB589B00020019009981027FE4C1E461546082856
:20E0C00006D0E06901F05EF8002809D03770BEE0288809213843108013980227017016E074
:20E0E000E169012088710521E269C9029180E1698872E169F0480881E1690020887328880B
:20E10000202108432880112113980427017013980225801C0290307806900A203070E5481D
:20E120001830049001F022FA0020059020462C3003906DE00998102808D1022D06D001994E
:20E140000298A28D401A8270110AC170E08D0A99884202D901F0CDF806E0884204D10698D0
:20E16000002801D030701CE00298E18D0170090A417012980088401BC01B82B2FF20C01B37
:20E18000904200D2024607A8009002980021C319E08D01F056FA3070002805D0C0B2832855
:20E1A00058D0E08D20833EE00598002804D0206C00790A282CD336E06846808BC119C9B216
:20E1C0000191022D0DD01399019A4978914202D1228F824208D00191206C0178032908D00B
:20E1E00023E0084613994870206C0178042906D007E000790A2818D20120059008E0E18DDA
:20E20000818002990198081802900198281885B20399049801F0ADF9002804D11298008809
:20E22000401BB84286DA022D0DD00998102806D102990198A28D081A8270110AC170129800
:20E24000058000203070206C0078032802D000200DB0F0BD0220FBE7F8B5964A0026126DB8
:20E26000002A2ED0401F934D84B24035E88A23460833AF8AC318BB4222D88B784F781B0284
:20E2800010183B4303701B0A43700B79CF781A023A438270120AC2700471220A427122462D
:20E2A000491D801D06F0ADFCE88AA41D001980B28049E882096D002208180270427000E04F
:20E2C00009263046F8BD30B57A4B028840339B8A934213D9774B1C6DA3185C781D782402C2
:20E2E0002C430BD05C791D7924022C436404640CA41D1219028000200B6030BD822030BD87
:20E30000F0B585B0074600266846068155E00198417802780D021543417902790802104381
:20E3200000044AD43D8003A800230122009052021946284601F085F9040044D1684601899C
:20E34000018201984179027909021143437802781C021443AC421CD10A041AD44A0401211C
:20E36000520C89030A430096C1788078090201430023204600F0C1FF040010D101994879D7
:20E380000A79000210430122D20310430871000A487101A904A8FFF796FF0400D1D00199FE
:20E3A00000964878097800020843694600238A89194600F0A2FF822C05D101A902A8FFF796
:20E3C00082FF0400A3D06846068109E0019948790A79000210434004400C0871000A487128
:20E3E00001A902A8FFF76FFF0028EFD0822C02D0204605B0F0BD0020FBE7F7B584B01446FA
:20E400000646002700F071FF2A480025006D00282FD0059801282CD12046FFF771FF070068
:20E4200027D1002E29D06846058118E0019948780978000208432080019B00955879197935
:20E440000202D8780A4301029F78587839431F7800029B1D384300F050FF002805D101A902
:20E4600002A8FFF730FF0028E0D0822800D100200746002E01D00F48056500F03AFF3846A6
:20E4800007B0F0BDF0B597B00021042003F00AFC084F00243D467C8040356C73AC73287BDE
:20E4A000B96CC00008380E18B08800280DD00120694603E0EC1900200128000008703068C3
:20E4C000019000216846F9F7BAFAB4803C65AC82EC8217B0F0BDFE4B9864184640300173CC
:20E4E0001A803838D861CDE7F949002049880A0700D501200A06120F01D002221043CA05A3
:20E5000001D5042210438A0501D510221043490501D520210843EE494031497B002901D0AC
:20E52000082108437047FFB5A7B00400289816461B9022D00178E6484D0642882292024628
:20E5400040320092002D14DB8A06920E1E2A0ED0229A5205520E10D13288172A0DD3009A7C
:20E56000927B002A09D1DB4D229AAA4205D0CA0906D08A06920E122A02D003202BB0F0BD53
:20E58000D348826C0098007B2590C000083810181F9048060CD40098407B002808D00099B9
:20E5A00088731F99289808601F9884800220E5E7002718A90F7069460F72C54902AA0A6418
:20E5C000309A4A6410A90F850F861B981D46007820908106BE4B601F24901A462C3221926F
:20E5E0002898DA691833890E1E93401C0B0006F095FD1FFDFD11FD1AFD90FDFCFDFBFDFAE0
:20E60000FDF9FDFCFDF8FDFDFDF7FDF6FDFDFDFDFDF5FD00032C7BD10320287017226A7009
:20E620000022AA70E0E2052CF5D14178027809021143A74B10AA19831185C278807812022F
:20E6400002435A8300297DD091427BD80021184681720181491E01841E9800F087FF0520CB
:20E660002870A81C1D900220009021991E9800F080FF002803D047E018A90870F0E29448F7
:20E680002030807C012803D002206870102002E001206870022022908D483030239000224F
:20E6A00020A9239802F0F5FD00282AD120A800782299814225D132880099801C511A8142FE
:20E6C0001FDB83481D99C08D0870000A48701D9820A9801C1D9000981D9A801C009023983B
:20E6E00002F0D7FD20A909781D9840181D900098401880B2009021991E9800F03AFF0028DD
:20E70000CDD0009802288DD10A2018A908706CE26DE0072C6BD341780378090219436C4B7B
:20E720008446198310AB1985C37880781B021843674B0029588305D0814203D801211846C6
:20E74000817200E0A4E061464B7909791B020B43038100218173104600F014FD00280FD112
:20E760005B480121C26991710522C369D2029A80C2699172C26958491181C069002181739C
:20E780005349E01F08841B98C01D48621E9800F0EDFE07202870681C009001201D904C4852
:20E7A0000021C18530E01D98012815D04848C169897901292FD000981038C17B807B090218
:20E7C000014300980170090A41700098801C00901D98801C80B21D903D4809E013E2BEE132
:20E7E0007AE1D8E00DE2A0E080E03BE01EE2B6E0C18D00980170090A41700098801C0090A7
:20E800001D98801C80B21D9021991E9800F0B1FE002802D006E0818DD3E731881D98081A81
:20E820000428C0DA1D98012800D16DE72848C1698979012903D0828D26498A4205D1818D48
:20E8400000980170090A417009E000981038C17B827B0802009910430870000A48701D9804
:20E86000801CC1E1072C01D0152C78D14178037809021943164B198310AB1985C3788078A8
:20E880001B02034312480029438301D0994201D90120F1E60E48012181720021018181734C
:20E8A000052C07D024981B99C0B2491D02F0CBFC0028BAD100200649C04308841B98009655
:20E8C0000195007818AB8006800E1CAA002105E0EC190020FFFF000001280000FFF7E6FB64
:20E8E0000746FE4810A9008B08857EE1032CBCD1402210A90A86417802780802F74910431E
:20E90000088310A9088520A9009131886B1C491E8AB2002100F095FE18A90870002830D1E3
:20E920000B20287020A8008833E0052C9DD1802110AB1986014640780B780202E7481A4305
:20E940000283CB7889781B021943E44B1046198410AB1A85E24A914202D307208CE697E015
:20E960003F23DE4A9B021943118421AA009232886B1C521E92B200F064FE18A9087000287A
:20E9800003D08328B1D102272FE10D20287020A88088401C28E120990C22C9095143C91C12
:20E9A0001E91A14204D92098400671D500201BE1417800780902014310A801851B9800789F
:20E9C00042062898C01C1D90002A62DA05206A4610721B980078C00944D008226846027295
:20E9E0008181A01A87B268468782289806901E98201A81B26846C1811D980490401806F06B
:20EA000061F9079006982599C0190890491E08A8017102A83099F9F712F807460021684626
:20EA20000172002F1BD0022F18D1009808A9007B0979401E884210DDA848289A836CC9006A
:20EA40005A50816C08A80079C000001D0C5200980099407B401C4873C7E00527EAE00620F5
:20EA600069460872002000901E980021201A209082B21B9B10A8DB1C008D00F03EFC014665
:20EA800018A80170002268460272832903D003E093E00720E4E702271B98007840060ED5BD
:20EAA0008E484188C90506D510AA018B128D914201D100214162002018A9087094E0FF21D3
:20EAC000013110A80186018D84480183209901841D994162132085E0052C6ED34178037812
:20EAE0000A021A4310A90A859446092269460A720021009101222499D20311438AB2C17805
:20EB0000807809021B9B01435B1D604600F0F5FB18A90870002269460A720122520210A944
:20EB20000A86832802D0002805D099E06B48098D018302277EE06948006D002807D020467B
:20EB40001B99FFF789FB18A9087000284DD12B46324620461B9900F024FB074645E01B98D1
:20EB6000022C4078009064D1002801D0012860D10A2168460172009901731AAA00200099C1
:20EB8000FFF73BFC0146684641730021817302A83099F8F754FF0746002168460172012124
:20EBA000890210A80186022F08D04C48006C8079002807D018A9087020E04BE047490098FE
:20EBC000088337E0002F03D0812018A9087031E01AAA01200099FFF710FC18A908700028C5
:20EBE00003D119202870012030806846007A002804D002A83099F8F722FF0746002F2BD081
:20EC000018E0062038E522993448090711D5012C0FD10B2269460A72C08888810021042091
:20EC200003F040F8082010A90886BFE62098400610D50327294810AA4188128E11434180DF
:20EC40005005400E04D01F99289808601F988480384693E404200FE518A8007800280ED057
:20EC6000012028701B980078687010A8008DA870000AE87018A80078287105203080174814
:20EC800010AA4188128E91434180E1E7FFB506469FB000201B903178012088401149124A92
:20ECA000084010A908860D494988914203D0002804D0080702D5012023B0F0BD219D002790
:20ECC0002F7020983C46018810A8018418A8077100F00BFB6846077202A907E0EC19002089
:20ECE0000102000009F80000FFFF0000FA48016401464031826C1A91097BC900083957181D
:20ED000022994164307801282AD0022809D0032879D12878800980011D302870EE48B18852
:20ED2000C1803078022804D12878800980011B30287001A8009010A8008CEB1CC01E82B2C8
:20ED4000B088002100F07DFC0028E1D1B1886970090AA9706946888810A9C01C08842DE1EB
:20ED6000717918A801713079012802D00228CFD1E6E0D9487F2340881B010246184010AB41
:20ED80001886802840D006DC102810D020280ED040280AD120E0FF38013859D0FF380138B1
:20EDA0006AD0FF38FF3802387ED0052491E0D00601D5082000E010201B90042069460872AD
:20EDC0000020888118A800900195318919AB1CAA1B98FFF76BF977E0BF4B3289188B824250
:20EDE0004FD10A221B92002973D101A9009110A9098C6B1C491E8AB2002100F022FC18A90A
:20EE000008710B2017E0F6E0B34B3289188B824237D10C221B9200295BD101A9009110A935
:20EE2000098C491E8AB21946098C6B1C00F009FC18A908710D2028706946888810A9401C57
:20EE40000884042069460872A348008B888140E0A14A3389108B834213D112231B93002943
:20EE600037D1536A002B05D00091128C00F045FA18A9087113205EE097483289038B9A42C0
:20EE800001D00424E7E016221B92026D002A09D1F268002A06D002651A98328A82821A9A73
:20EEA0000020D082002900E02FE012D1B8883968FFF7D2F918A9087100280AD1B8882B4655
:20EEC00018AA396800F06DF90446022818D0042C16D0B88800280FD06846007A002804D09C
:20EEE00002A82299F8F7ABFD0446012069460872386803900020B880002C5FD0052C7BD020
:20EF00006846007A032873D0A5E018201B90002905D071483189018300210165D9E76E4801
:20EF20000246017E18320120FFF767FA18A908710028CED119202870012010A90884C8E761
:20EF40001A98407B002856D0307AC0001358001D0193105A1D9000291AD100F0CAF906206C
:20EF600069460872002000901D980F3882B201988178437808021843019B0021DB1C00F032
:20EF8000BCF918A90871002269460A72832830D0002118A8017110A80184012168460172B7
:20EFA000019803901A981A99407B401E48731A98807B002802D01A99401E887310A8008EF3
:20EFC0007F21090102468A431DD043480022008811468300042002F0C0FD3F483178017101
:20EFE00010A94088098E08433B4948800FE003E02BE002242FE00524374810AA4188128E85
:20F000009143418027E034494A8882434A806846007A002805D03048416C02A8F8F70FFD87
:20F02000044618A80079002815D01B986870012028702948008BA870000AE87018A800794D
:20F040002871052110A8018405E02348416C02A8F8F7F5FC044600F04CF91F48408840053A
:20F06000400E20D11A98807B00281CD1B888002819D0209910AA09881184229900913968B8
:20F0800018AA219BFFF74FFA044602280BD00120694608723868039002A82299F8F7CFFCC8
:20F0A00004460020B88010A8018C20980180204602E600B50022D243074997B04A80042869
:20F0C00007D1022268460270097901710021F8F7B6FC17B000BD0000EC19002010B5394C6B
:20F0E00003780022216C012B02D0022B44D126E00B78002B01D0042B03D10A71226C0321F1
:20F100001170216C83880A79D200921D8B52216C0A79D20008328918C2880A80216C03894B
:20F120000A79D2000A328B524289206C0179C9000C314252216C0879401C087120E00A7495
:20F14000226C81889180216CC288CA80226C01891181226C41895181216CC068C860616C68
:20F16000206CF8F76CFC0146022807D0206C007C002802D1002903D0812010BD832010BD87
:20F18000002010BD8178012909D100880521C902884202D0491C884201D100207047052073
:20F1A000704710B51488844201D2052010BD17241C701080421E491C581C05F022FD0020E8
:20F1C00010BD0000EC19002010B58B78002B11D082789A4207D10B88002B0BD003E0091D19
:20F1E0008B78002B08D08B789A42F8D103880C88A342F4D1002010BD812010BD10B500294F
:20F2000002D001290DD102E00088000501E000888004800F07D001281CD0022809D003280F
:20F2200010D0812010BD002901D0032010BD022010BDF5F733FE03280CD004280AD0002855
:20F2400006D009E0F5F72AFE042803D0022803D0052010BD002010BD0F2010BDF3B5C81C78
:20F2600080080E46800081B0B04201D08620FEBDFE4C354626600198A08000202081E080B8
:20F2800014E0B807A978800D0843F94905F033FDE088401CE080B80607D42089401880B26B
:20F2A00020810199081A8019A8600C352F887807E7D40020A072FEBDEC480C22C1880089FD
:20F2C0005143081880B2704770B51346E74A45189488AC4201D2842070BD126810180A46E5
:20F2E000194605F08EFC002070BDE049012088727047DE49002088727047FFB589B0970468
:20F300000E460546BF0C029200F034FA040021D0002069460873D548807A012812D001214E
:20F320002046FFF76BFF002815D12078400609D50221684601730582218841828682C782B4
:20F340000C9806900298000407D500273E46012501970CE001200DB0F0BD2078A1788007E1
:20F36000800D0843C249019005F0C5FC0D46029840040AD50198A84207D12088E178800572
:20F38000800F00020843B04201D3AE4201D90720E1E7B81980B20290A84201D90D20DAE7CB
:20F3A0006846007B002804D003A8F8F744FB0028D1D10198A8420BD1208803210902884384
:20F3C00002998905890F0902084320800298E0701298002800D007800C9800280CD0207823
:20F3E000000609D4A0683A4680190C9905F009FC20881021884320800020ACE7FFB59B4DD7
:20F4000081B00E46E8882F680C21009048433C189749039805F06FFC0A462889E11B844622
:20F420000C314018318880B28B0601D5002300E013461818AB8880B2834202D8842005B0FC
:20F44000F0BD0098894D401C80B2E88021800D99002900D00C600399A170E2702188039DA7
:20F460008908AD058900AD0F294303252D02A9439505AD0F2D0229430425294321800C9989
:20F48000002900D0088001998978A17101990988A1803178890601D50B9905E073496244F9
:20F4A00092B20A81991AC919A160002121733278920601D50020C2E700910B9B0A9A0499D9
:20F4C000FFF71BFFBBE7FEB5044600F053F9070008D0664D641EE8880190A6B228683446CA
:20F4E000009015E00120FEBD0C2000996043095A8A060BD489078A0D0099801C085C5C490C
:20F50000104305F0F8FB2889401A2881641CA4B20198A042E8D8EE8000203870FEBD0028D2
:20F5200003D0401E0880002070470120704710B54E490288CB889A4201D3822010BD0B6898
:20F540000C21514359180B88CC789B059B0F1B02234341608C7904738C884481C3818968AA
:20F56000521C016102800281002010BD012101827047FEB505460020C043088068680F469F
:20F58000817868468170686801886846018000218171288A2C88A04200D304462C8234E011
:20F5A000288A401C2882301D6968FFF70DFE002829D139882F48814201D1601E388068885F
:20F5C000A04227D33088F1788005800F0002084302906946301DFFF7F7FD002813D1298997
:20F5E000244881421AD000213046FFF707FE002809D12A890298824205D1E968B06805F019
:20F60000D3FA00280AD0641CA4B2204600F0B2F80600C5D1641E2C828220FEBD7C80B079F7
:20F62000B871B088B8803088388130788007810DB078014379810298B881B06838610020F9
:20F64000FEBDFFB585B014460F46059800F092F8050037D00548BE05807AB60D01281CD052
:20F6600000212846FFF7CAFD002805E0441A002001020000FFFF000022D1287840060CD5F8
:20F68000012168460170059981802988C18006814481F8F7D0F9002812D12888AA7881072F
:20F6A000890D11438005800FEA7800021043BE420AD0374A914207D3611E814204DD0B203F
:20F6C00009B0F0BD0120FBE7864201D90720F7E7801B82B2A24200D922460E98002800D088
:20F6E00002800898002804D0A8688119089805F088FA0020E4E770B514460D4600F03AF84C
:20F7000000280DD001882980002C0DD0017880788907890D01431E48814203D2012002E0CD
:20F72000012070BD00202070002070BD70B516460D4600F01FF804000DD02D882580FF2E3B
:20F7400016D0A807A178800D0843114905F0D3FA002E06D101E0012070BDFF31FF3103313F
:20F7600089B2A170A80880008905890F08432080002070BD0749CA88824207D3002805D072
:20F780000C22096850430C38081870470020704701020000441A0020F0B585B00E4605464B
:20F7A0000020694608707078FE49C00003900C58FD4F002D0ED0022D73D0002C72D020784D
:20F7C000801E030005F0AAFC09837F7F7F83797F77727F00002C03D1F4A16B2005F0ADFB44
:20F7E0002078801E030005F099FC09065E5E5E19365E50545E003078062803D0EBA17620A3
:20F8000005F09BFBB8687168806C032205F0F9F9012069460870002835D1CEE730780C2865
:20F8200003D0E2A1812005F088FBE0680078002806D0B8687168806B102205F0E2F928E0AD
:20F84000B8681021006B05F039FAB868816A006B0A787168F1E730780D2803D0D3A1942043
:20F8600005F06BFB04206946087071684878097800020843B9684A6A5178127809021143F4
:20F88000484069468880084608E0C8A1AF2005F054FB6846007800288FD06846F5F703FB32
:20F8A0008BE727E01CE0C1A1B420F0E7B8686169006CFEF708F8A16900E0E168B868006CBC
:20F8C000FEF701F803E0B9A1E32005F036FBB8682146006CFDF7F7FFB24A0399002050509F
:20F8E000022D07D0002D05D0012D03D0AFA1EF2005F023FB05B0F0BD10B50178012401299E
:20F9000002D0022910D112E04268A748002182600170A4486C38C166016741678167D28900
:20F9200002214C3001F0E1F90024204610BDFF209EA1163005F001FBF7E7F0B505469EA164
:20F9400003C997B014911390002008A9087595492A781031944C0491217805910126914F92
:20F96000A168130005F0DAFB0CEF07309AF0EDECEBEAE9E9E8EF20700124FF264F360546E4
:20F9800010A80570457001F0C1F90746012803D086A1304605F0D1FA10A93846FFF7FCFE0D
:20F9A0002046641EE4B20028EAD10A20694608706846029501F088FA002803D0FF207BA1A7
:20F9C000583068E0002646E3C86A0078C0072FD0012069460870684601F076FA002804D045
:20F9E000FF2072A16B3005F0A8FAA068006CFDF761FF050004D1FF206CA16E3005F09DFAAB
:20FA000008984078C0003D5006202870A068016869600069A8606448C01CE860284601F0A9
:20FA200053FA022804D0FF2060A1783005F085FAA068C06A00784007C4D50120694608706D
:20FA4000684601F041FA002804D0FF2057A1803005F073FAA068006CFDF72CFF050004D13A
:20FA6000FF2052A1833005F068FA08984078C0003D5006202870A068016869600069A8605C
:20FA80004948401DE860284601F01EFA022899D0FF2046A18D3005F050FA93E7A968002970
:20FAA00033D0694608712979012932D0022904D0FF203EA1A73005F040FA3A481022103056
:20FAC000A96805F09EF8374810303649203148602078C1062CD5EF21084020700320694639
:20FAE0000870304810300290684601F00FF90446022808D0002C06D0012C04D0FF202BA163
:20FB0000B83005F01AFA69466FE101216A461171DBE7244A04996C3AD06748608860C8603F
:20FB20000621A86803F0FCFE1E4910310860CAE720210843207045E7A1E15AE119E1E6E01B
:20FB400086E056E000E081E2886C40798009012804D0FF2015A1CC3005F0EFF9A068017A62
:20FB6000002906D1416B406801F01FFAA16801200872012069460870684601F0A5F90028D6
:20FB800004D0FF2009A1D73005F0D7F9A068006CFDF790FE050004D1FF2004A1DA3005F069
:20FBA000CCF90DE0BC1A0020B40000207372635C736D2E630000000004411A8800A48000A9
:20FBC00008984078C0003D5002202870A068416B6960806CC01CA860284601F075F90400A8
:20FBE00004D0FF20FD49E23005F0A7F929462831FBE0172268460272012202708078820810
:20FC0000287992008007800F024368468270FB20024028794007C00F80000243684682703D
:20FC2000EA8882804A6C02A901F090F9002804D0FF20EA49F73005F080F9052108A8017546
:20FC40006846017A0187A0680026406C0F9006E2012069460870684601F036F9002803D081
:20FC6000DE49DF4805F069F9A068006CFDF722FE060004D18320D949800005F05EF9A068E3
:20FC8000006CFDF717FE1290002804D1D448D349801D05F052F9D3488068006CFDF70AFED0
:20FCA000040004D1CE48CD49093005F046F908984078C0003E500A203070287A307168684F
:20FCC000C84DB060A868406C3061172030731298B4617061304601F0F7F80446022808D0A6
:20FCE000002C06D0012C04D01120BC49400105F024F92046316AFFF74FFD2878052101402E
:20FD0000042900D05EE6FB21084028702AE0059840084000207082071CD5FD22104020706E
:20FD20000F206A46107017201071486C0290684600F0ECFF0546022808D0002D06D0012D5F
:20FD400004D0A748A5493A3005F0F7F869462846FFF722FD2078052101400429D2D1FB2187
:20FD600008402070072008A908759E488078087628E6012069460870684601F0A5F8002840
:20FD800004D097489549543005F0D7F8A068006CFDF790FD060004D113209049400105F078
:20FDA000CCF890488068006CFDF784FD040004D18B488A495A3005F0C0F808984078C00010
:20FDC0003E500720307087488068406870606868F460B060304601F077F8040004D08048F5
:20FDE0007E49653005F0A9F8316A2046FFF7D4FCE8E5012069460870684601F065F8002811
:20FE000004D0774875497A3005F097F8089840781190A068006CFDF74DFD060004D151206C
:20FE20006E49C00005F089F8A068006CFDF742FD040004D16A486949823005F07EF811982B
:20FE4000C0003E50C019296941600920307068687060A868B060A889B081634830611030E1
:20FE6000B4617061304601F02FF8022804D05C485A49903005F061F811982875A2E55A4A4A
:20FE800000208C32107002206B46187001922879002801D0107098E0524803230C304068E0
:20FEA000FB2703708378504A9B089B003B4083704B7A00271B07DB0F43708C3257600B7BC6
:20FEC000C370CB7A1372537A0C7D5B08E4075B00E40F23430C461534D460FD242340CC7E30
:20FEE000E407A40F234353720B461C331361477107718B7A3B4A9C070C32A40F1268012C30
:20FF000004D19478A407A40F012C1DD09B089B008B7293785B0702D48B7A5B0728D54B7AE1
:20FF200013AF5B075B0FDC005B00E318147864001B19DBB2DC083C5D5F077F0F0623DB1BC0
:20FF4000DC40A3079B0F14E04C7A53796406640F23404371147906273C400471E4001C43C9
:20FF6000204B5C7083789B089B005B1C8370D0E700238478FB273C408F7A7F07FF0FBF00D7
:20FF80003C4384704C7A6407640F04705078012807D1487A000704D5032008A908750220F8
:20FFA0002DE0022B27D0012B2BD00F4B0020049AD86750609060D06018467C30024610322E
:20FFC0005060887AFB2210408872684600F09EFE040035D0012C34D0004907E0ACFB0000BD
:20FFE00009020000B4000020501A00206520C00004F0A3FF25E0032008A9087501200876C8
:020000040001F9
:20000000E3E77E4C0D21E01C04F058FE204610304460022008A908750E94A868002807D08D
:200020000068206005997648202211430170CCE705980007C9D57349734804F07EFFC4E7ED
:20004000002669462046FFF7A7FB04E06E486D49203004F072FF08A8007D002802D00DA8EC
:20006000F4F721FF304617B0F0BDF0B597B00C46054600206946087061482F785F4E017845
:20008000583E82683B0005F049F80BAA8407263B4C6B79798F9CAA002B20694608730CA926
:2000A00003A8FDF73DFC002804D057485549413004F043FF55490D9804F01DFE4F4801603E
:2000C0004F4869680C300160AA68426001910820694608708CE08A0610D5DF2211400170E2
:2000E00003202070454810304168A1604068002802D00020207177E00120FBE7102256E0C1
:200100002B20694608733D4903A85C39FDF708FC002804D03C483B496A3004F00EFF0420E9
:200120001BE02A206946087303A810220230696804F067FD07A810220230A96804F061FDA2
:200140002E4903A85C39FDF7EBFB002804D039202C49000104F0F1FE05202070666043E0C2
:200160002A79002A02D001221143017005206946087028798880A868029039E0D06A4023AB
:20018000018819430180D06B6968102204F039FD2AE0FB2211400170062069460870A9684A
:2001A00068680291019023E0CB0703D002221143017058E70F20207017202071506CA06038
:2001C00012E0937A9B0706D0D26A44781388FF3401342343138004221143017004E00A4893
:2001E0000849BD3004F0A9FE684600780028E0D06846F4F758FE36E701207047CC1A00203E
:20020000B4000020ACFB00001503000040420F0070B504780D460646230004F07FFF0B1CBE
:20022000181C1C1C1C07181C1C181C000021052001F038FDB068007805280CD0FA48002242
:20024000008811468300052001F087FC03E00021052001F027FD002D0ED000202870294633
:200260003046FFF702FFF1482978005D884201D1032070BD022070BD00213046FFF7F5FE1F
:20028000002070BD30B5E8494B68497A0A0111460C315C5C032C0CD00446002520342571CA
:2002A00025725C5CA500AA18641C5C549850032030BD062030BDF0B50446264620360D4649
:2002C0003279012008218FB0002A0CD0012A21D0022A2BD0032A04D12A78052A01D1297063
:2002E00000200FB0F0BD01203071606800280AD0A069017061684160216981606169C160AC
:20030000FFF7C0FFEDE707202870206968606069A86009E029780729E3D10220307105201D
:200320002870C248203868600320DAE729780529D7D1A08910280AD9103880B2A081A168B8
:200340001023091803A86A6800F054FE2DE0102804D0C1B20BAA1020A76809E01023226963
:20036000A16817E0491EC9B2401EC0B27B5C13540029F7D100280AD0401EC0B280211154C4
:20038000002102E0401EC0B211540028FAD1626910230BA907A800F02DFE102307A903A828
:2003A0006A6800F027FE032030716068019003A8029005206946087029466846FFF728FF76
:2003C0008FE7F0B5044626460D462036317901208DB000290BD0012938D0022905D12978C3
:2003E000052902D10920287000200DB0F0BD217D6846CA07D20F02738807C10F68460174BC
:20040000012203A905A800F0EDFD04A9012205AF481D00F0E7FD0722B81CE16800F0E2FDB4
:2004200007A807220130216900F0DCFD6068019009A80290102305AAA16800F0DBFD0120F0
:200440003071052168460170294621E029780529CBD1062203A8E16900F0C4FD04A8062239
:200460000230A16900F0BEFD042106A800F0B2FD6068019007A80290102303AA696800F0E8
:20048000B9FD0220307105206946087029466846FFF7BEFEA9E7F0B5074685B00D4600209E
:2004A000694608703E466248203632798179133801240078130004F031FE180DFEFDFCFBB7
:2004C000FAF9F8F7F6F5F4F3F2F1F0EFEEEDECEBEAE9E8E7B968039100291BD001226946B7
:2004E0000A7003220A710A224A7139690291397900297DD0039A1278002A7AD00C2A78D283
:20050000130004F00BFE0BEF09EF354D8498B0F1EDECEF000020C8E30021062001F0C2FB12
:200520003879072866D1424C133C2078022802D000287FD101E00020207003980079C11F36
:200540000A2901D30A2598E1607039480722C01F039900F047FD01203071207002206946A0
:2005600008703348801F01903869401C029037E211293DD12E4C133C0228DAD16068617829
:20058000007A884201D9062577E1039926481022491C303800F026FD03202070022045E1A3
:2005A0001129E6D1224C133C0428C2D10520207003991D481022491C203800F013FD062003
:2005C000307178690321017062685168416016492039816021460C31C160C91D0161017DBC
:2005E000537A49084900DB07DB0F1943017502E070E354E384E1D3688361FD231940537AC0
:200600009B07DB0F5B0019430175116976E10229AFD1002867D005206946087103984078A6
:2006200048713869029051E3201B00209C510100DB00002082E011299BD1F74C06287DD18F
:20064000A0680399806B1022491C00F0CBFC06216846017038690290002168460171FFF70D
:20066000D7FD072057E00B299BD1EB4C07287ED1A0680399006B0222491C00F0B3FCA068B4
:200680000822406B039917E00EE116E3FDE2DDE2C7E2BCE29EE267E248E241E21FE2F5E138
:2006A000DFE1C8E1BEE1B1E1A5E16AE147E128E1DAE0BEE0AFE075E0C91C00F093FC0621D7
:2006C0006846017038690290002168460171FFF79FFD204613304179490849003EE041E0B9
:2006E0001BE001E05CE0EFE2112991D1CA4C08283DD1A0680399C06B1022491C00F072FC5D
:2007000006216846017038690290002168460171FFF77EFD09202070C9E208298CD1BE49B5
:20072000092824D1039842788868016C0A700399406C0622891C00F055FC00E017E0062113
:200740006846017038690290002168460171FFF75FFDB14813304179FD221FE041715EE2AE
:200760003071F2E11129C0D1AB490A2801D0082583E088680399806C1022491C00F032FC86
:2007800006216846017038690290002168460171FFF73EFDA04813304179FB221140DDE757
:2007A00007256AE0297802297ED19B490128FBD16A684A6015780846002D5CD106216A4647
:2007C00011703969029107211171029902240C70CA785207520FCA704B795B075B0F4B71FA
:2007E0008B795B075B0F8B71D20701D18A714A7105460A794078824200D26A7086480722DF
:20080000133000F0EFFB00202C70307101466846FFF7FEFC4BE229780429C5D103286FD17D
:2008200008227E48696800F0DDFB032030710420F2E129780429B7D1774F0328B4D17748E9
:2008400008220830696800F0CDFB0420307178684168002906D00321297000212971406840
:20086000A86072E10320D7E1287803289CD1287900281AD00546002D16D0062168460170B3
:2008800038690290022168460171029805210170457000216846FFF7BBFC0121684601703F
:2008A00004210171457115E293E15B49A86849680028486001D15A48486005203071786988
:2008C000032202704A684260544A8260524A0C32C260D21D0261027D4B7A5208DB0752008D
:2008E000DB0F1A430275CB688361FD231A404B7A9B07DB0F5B001A4302750969C16130E184
:200900000DE12978092988D14349032885D1042008700620694608703869029011200871EA
:20092000029803210170401C1022696800F05AFB00216846FFF76CFC00203071B7E12978BD
:20094000092993D1052891D134496A6820391020401EC0B20B5C145CA34203D000200425F2
:2009600030718AE70028F3D10720307178690421017029494968496841602849816010392A
:20098000EEE028780A28BED10620694608703869029011200871029804210170401C102240
:2009A0001E4900F01FFB00216846FFF731FC1A48102140786A68091AC9B2101800F00AFBFC
:2009C0006868019014481330C178C9070BD08179002902D14079002805D0082030711BE1C2
:2009E00029466846EFE007206946087000216846FFF70EFC5FE128780E2884D10648696864
:200A000081608969407808700920A9E6C80701D00A20FFE00F20A3E6C8000020101B002087
:200A20007C51010028780F2879D1A8683861287938730B20FAE628780428F5D1FC4C69681C
:200A4000A0680822006A00F0CDFA0C20307178690722B9690270A268D3684360126A826092
:200A60007EE028780D28DFD1F14C6968A06802230269C06900F0BEFA0D2030717869062146
:200A80000170A1688A684260096966E028780C28CAD1E74C6968A0686278406A00F0A2FA05
:200AA0006078A2681021091A526AC9B2101800F091FA0621684601703869029011226846CC
:200AC0000271029810220170A168401C496A00F089FA00216846FFF79BFB0E206EE0287864
:200AE0000F2876D1062168460170386902900B2168460171029C0720CD4D2070A868022210
:200B0000C169601C00F06EFAA8680822016AE01C00F068FA00216846FFF77AFB7AE7C8E0A1
:200B2000880701D5102075E0132019E628780F284FD1A86838612879387311203071BC48D7
:200B4000816848690078002801D00324CAE0786906220270C9684160B6498160B549091D68
:200B6000C160FFF78FFB30E0B14880684169097800290CD129780C292BD1AD4C6968806A2C
:200B8000102200F02FFAA16801204969087006216846017038690290112168460171029851
:200BA00008210170A249401C89681022896A00F019FA00216846FFF72BFB12203071092153
:200BC000684601702946FFF723FB044601287DD088E06FE028780F286CD10620694608709B
:200BE0003869029008200871029809210170904989680A78D207D20F427049680622801CBF
:200C000000F0F0F900216846FFF702FB8CE7480705D514203071092069460870E0E616207C
:200C20009EE528780F2851D1A868386128793873152030717869062101707D4989688A684B
:200C40004260096981607B49891D89E728780C2845D1774C6968A0681022C06A00F0C2F938
:200C6000062069460870386902901120087102980A210170A168401CC96A102200F0B2F9AF
:200C800000216846FFF7C4FAC9E7694813304079002810D0C10703D065480621017006E0A6
:200CA000800701D5082000E00A2061490870002418E00BE013E0172052E55D49002805D078
:200CC0000020307108700A206946087068460078002804D000216846FFF79AFA002454484F
:200CE00000210170204605B0F0BD10B5524BFF245C72586019721A80002204E0491EC9B282
:200D00000B010C33C2540029F8D110BDF0B54A4E0546717A01208DB0FF2971D00127727A65
:200D2000736811015C180C31595C8900091F64586A7021780B0004F0F1F90B960709272C93
:200D400059888D4A4F5492002F707CE0214620310A9109790120002902D0012967D10EE06A
:200D60006068019005A802900D21C01C00F032F9032205A8A16800F035F90A984EE029784C
:200D8000052974D106215DE029462046FFF719FB69E021462031069109790120002902D067
:200DA000012964D10EE06068019007A802900822E16800F017F9082209A8A16800F012F9FA
:200DC00006982BE02978052951D10A213AE02946204600F01AF946E029462046FFF76BFA06
:200DE00041E029462046FFF756FB3CE021462031059109790120002903D0012937D11DE07E
:200E000056E06068019007A802900822A16800F0E9F8082109A800F0DDF80598694607719B
:200E20000520087029466846FFF7F2F91BE00BE0C800002074510100201B00202978052959
:200E400015D10B212970002011E02946204600F023F908E02946204600F04EF903E02946AF
:200E60002046FFF7C9F9002801D001280CD12562717A736809010C315A5C521E1206120E63
:200E80005A5401D003204AE70328FCD0737A726819011D010D312C46515C7172FF270D34E2
:200EA00017550C35545D002C02D0FF2903D173720DB0F0BD21460C010D34145DFF2CF9D170
:200EC00009010D315354F3E770B5AD4C0546607A214603464A6811E0010108460C30105CBB
:200EE00008E0401EC0B286008E199659AE4201D1042070BD0028F4D10D31505CFF28EBD151
:200F00009F480021007A01E0491CC9B2884204D90E010C36965D002EF6D1884201D80520E6
:200F200070BD08010D30135461722846FFF7AAF9032806D0617A626809010D31515C61728F
:200F400070BD28462830FFF7E1FE70BD10B504780123012C14D10C78022C11D30B231370DE
:200F600083785B075B0F537002220A708088002805D0830000221146062000F0EEFD002324
:200F8000184610BD0EB50022012105280AD0062807D1684601700221017142710021FFF794
:200FA00064F80EBD68460170F6E710B58EB00C4606216A461170019072480290001D0390D4
:200FC0006846FFF781FF102220460B9900F00AF80EB010BD002202E0491EC9B2425400298F
:200FE000FAD1704703E0521ED2B28B5C8354002AF9D1704730B505E05B1EDBB2CC5CD55C06
:201000006C40C454002BF7D130BD3EB5044620300D4602790121002A02D0012A3AD10FE08E
:20102000616801915749083102910121017105206946087029466846FFF7EAF8014629E0C4
:201040002878052826D169681022A06800F087F86868C07B000606D54A4AA068102318324D
:201060000146FFF7C7FF1022A168E06800F077F8A068C07B000606D5424AE0681023183216
:201080000146FFF7B7FF07202870A0686860E0680021A86008463EBDF0B5044626460F4664
:2010A00020363179012089B0002909D0012905D13978052902D10C203870002009B0F0BDC8
:2010C000606803AD01900295022203A8A168FFF789FF0222A81CE168FFF784FF0C21281DFE
:2010E000FFF778FF0120307105206946087039466846FFF78DF8E1E710B5034620331C790F
:201100000122002C04D0012C10D0022C25D11EE001211971C16806220A7040684860194855
:20112000801C8860801CC86008460CE00C780C2C13D102221A71C2680523137049685160A7
:20114000806890601046FFF79DF8024605E008780B2802D10D2008700022104610BD10B574
:20116000002409E00B78521E5B0023430370401C0B78491CD2B2DC09002AF3D110BD0000D3
:20118000201B00207451010070B50D46040012D0002D10D02101284603F090FD10225449E4
:2011A000284603F02EFD524801210838018044804560002070BD012070BD70B54C4E00243F
:2011C0000546083E11E0716820014018817BAA7B914209D1C17BEA7B914205D10C22294686
:2011E00003F0E2FC002806D0641C30888442EADB0020C04370BD204670BD70B50D460600FC
:201200000AD0002D08D03A4C083C20886188401C884203D9042070BD102070BD3046FFF778
:20122000CCFF002801DB401C0AE020886168000140181022314603F0E4FC2088401C2080AF
:201240002870002070BD70B514460D001FD0002C1DD00021A170022802D0102817D108E0DF
:20126000687829780002084311D00121A17010800BE02846FFF7A1FF002808DB401CA07096
:20128000687B297B000208432080002070BD012070BD70B5054614460E000AD000203070CD
:2012A000A878012807D004D9114908390A8890420BD9012070BD002C04D028782070288820
:2012C000000A50700220087010E0002C0CD049680001411810391022204603F092FC2878A5
:2012E00020732888000A607310203070002070BDEC00002073490968016000207047714986
:2013000008600020704701216F4A704B002803D0012805D06E48704791630020187001E015
:20132000D1631970002070476A49012008606848801C70470422684B6649002805D05A609B
:20134000086901221043086108E008694008400008619A605C490020C03188600020704784
:201360005C490622002808D0012809D002280DD003280FD05648401C70470869904302E0B6
:2013800008699043801C08610020704708699043001DF8E708691043F5E74E494A6A0243BD
:2013A0004A62002070474B494A6A82434A62002070474849496A0160002070474549CA69DD
:2013C0000243CA61002070474249CA698243CA61002070473F49C96901600020704730B56A
:2013E0000546002072B601463A4A384C4032002D11D00123012D0CD0022D02D0072062B61D
:2014000030BDA3706478002C01D09363F7E79163F5E7A170F9E7A170F9E72F4904208860E9
:2014200029490020C03188602849012008702B490A688023120A12021A430A6028490860DE
:20144000704722480078704770B5EFF31080C507ED0F72B61D4C6078401C0006000E607034
:2014600003D120A1CC2003F068FD6078012806D1A078002803D01749012040318863002D9E
:2014800000D162B670BD70B5EFF31080C507ED0F72B60E4C6078002803D112A1DC2003F0DF
:2014A0004CFD6078401E0006000E607006D1A078002803D00749002040318863002D00D115
:2014C00062B670BD0004004040000040FC00002004200000000500400003004000E400E077
:2014E00000E100E07372635C736F635F706F7765722E63008107C90E002808DA0007000FA6
:2015000008388008B94A80008018C06904E08008B74A800080180068C8400006800F70477E
:20152000B44948788978884201D3401A02E02122511A0818C0B27047AE4923314878897810
:20154000884201D3401A02E02122511A0818C0B27047A849463148788978884201D3401A99
:2015600002E02122511A0818C0B27047A04810B50C300168FF22120291430122D2031143EB
:2015800001609C490020233148708870233948708870463148708870974802F0FFFA964806
:2015A000401C02F0FBFAF2F7C7F900F015F910BD20207047B4E770B50C4605460026FFF704
:2015C000AFFF8C49A04214D30A46203A00232046641EE4B200280BD08878105C287088786D
:2015E0006D1C401CC0B288702128F0D18B70EEE7012600F0F1F8304670BD202070479BE7A6
:2016000070B50C4605460026FFF796FF79492331A04214D30A46203A00232046641EE4B22D
:2016200000280BD08878105C287088786D1C401CC0B288702128F0D18B70EEE7012600F063
:20164000CBF8304670BD202101700020704710B50446FFF77EFF2070002010BD70B50C4625
:201660000546FFF776FF63494631A04215D30A46203A00232046641EE4B200280BD0887879
:20168000105C287088786D1C401CC0B288702128F0D18B70EEE7002400E0584C00F09CF8F1
:2016A000204670BD70B50C460546212904D9FF2053A1473003F041FC4C484068103840B27E
:2016C000FFF718FFC6B20D20FFF714FFC0B2864207D2FF204AA14D3003F02FFC01E0F2F7CD
:2016E0006BF921462846FFF766FF0028F7D070BDF8B5404E07462336B1787078212200F015
:2017000060F8354623353B4C00280ED0A1786078212200F056F8002814D0A978687821224F
:2017200000F04FF800281AD025E032497078C91C0F547078401CC0B2707021281BD10020C5
:20174000707018E02B49607820390F546078401CC0B2607021280ED1002060700BE02549C2
:20176000687826310F546878401CC0B26870212801D100206870B1787078212200F021F8D9
:2017800000281DD0A1786078212200F01AF8002816D0A9786878212200F013F800280FD0AA
:2017A000F2F7ECF8144802F001FA01214903884203D013A1C12003F0C0FB0F4802F00EFA74
:2017C000F8BD401C884205D0904201D1002901D0002070470120704710B5074802F0E6F927
:2017E000002801D1F2F7B9F810BD000000ED00E000E400E04C1B0020FF000020072000002A
:201800007372635C736F635F72616E642E63000010B5284802F0C2F9002803D026A11D2069
:2018200003F08BFB2348401C02F0B8F9002803D021A1212003F081FB10BDF1B5224D6F689F
:2018400001261C4802F0B2F91A4C002803D10026601C02F0C3F91D4A1D490120506000BF51
:2018600000BF00BF00BF00BF00230B604B60009B6B60106000BF00BF00BF00BF00BF086832
:20188000002802D148680028F9D048680028E4D1002E04D06F60601C02F088F907E0601CFC
:2018A00002F084F90028D3D1024802F097F90020F8BDC2E7010100207372635C736F635F39
:2018C0006563622E6300000000E5004000E0004000E1004030B5EFF31081CC07E40F72B6A1
:2018E0001D4A116910230D461D431561002C00D162B61A4DC406E40E0120A0402C68044298
:201900000DD0C8060AD4EFF31080C007C00F72B6116999431161002800D162B630BD20BF69
:2019200040BF20BFEAE70E4908784A78401CC0B2904200D008707047084A094820BF40BF3F
:2019400020BF4178037843701368002B02D103788B42F3D00020704700ED00E000E200E0D7
:2019600003010020FEB5F64C07466068FF213E0181552178FF2913D009010831415832460C
:20198000491E083209020192090A805800F0CEF9002802D02478254615E061682078885532
:2019A0002770FEBDE648426801981158280100900830105800F0BAF9002806D1E0482C4666
:2019C000416800980D5CFF2DECD1DD482101406885554754FEBD70B5D94A04460020157A14
:2019E00053680AE00201561C9E5DA64203D10C329A588A4204D0401CC0B28542F2D8FF20C8
:201A000070BDF8B5CE4F3E7801F01AFE0146FF2E71D03401254678680835405900F086F996
:201A200002280CD97868405901F0FDFD01F008FE01467868405900F079F902285BD8C049B4
:201A40004868025D0A70A11C425C002A0CD0521E425441590122D20589180902090A4151B1
:201A60003046FFF77FFF30E0631CC25C0092221D94468258002A10D001239B029A420FD9BB
:201A80009205920D43595703DB191B021B0A43516346C3589A1A920A09E0FF21C1540AE034
:201AA000435952039A181202120A4251002242543046FFF757FFA2480C344168C2680098B1
:201AC000095980001258009890479D4C2078FF2811D0000161680830085801F0A4FD01F0DD
:201AE000AFFD01462078626800010830105800F01DF9022886D3F8BDF8B51C4615460E46F4
:201B00000746FF2B03D38FA1D42003F016FA8C48FF21C7604560047206740170002242705C
:201B2000104604E00201521C401CA954C0B2A042F8D3F8BD70B5824C06466578207C85424E
:201B400003D380A1E72003F0F8F9E068A90046506078401C6070284670BDFFB581B01D4635
:201B6000FF2401F06DFD764F064679780198814203D874A1F52003F0E0F971480021037A61
:201B8000406810E00A019446521C825CFF2A25D0019FBA4205D162460C328758029A9742B2
:201BA0001ED0491CC9B28B42ECD8FF2C18D021014A1C019B83540B460C33029AC250039BDC
:201BC0005F4F0022012B0ED00B1DC25001239B029D4216D9AA05920D08D008E00C46E0E73B
:201BE000FF2005B0F0BD0B1DC550EFE71A4653039B190E461B0208361B0AAA1A8351920ADF
:201C000009E0002D00D101256B039B191D022D0A0B460833C550891C42543D463E782046C4
:201C2000FFF7A0FE2878B04214D0000169680830085801F0F8FC01F003FD29786A680901DD
:201C4000083152580146104600F070F8022801D2FFF7D7FE0198C4E770B50C46054601F0ED
:201C6000EFFC064621462846FFF7B5FEFF2817D0334D04012046696808300858314600F0E6
:201C800055F80121090340186968A41C095D400B002901D089020818002800D1012070BD43
:201CA000002070BDF3B581B00F460198FFF793FEFF282AD0224E3578726829460C4604E0CC
:201CC000844205D025462301D45CFF2CF8D11CE0FF2C1AD0A5421CD10801105C3070FF2895
:201CE00015D000010830105801F09DFC01F0A8FC01463078726800010830105800F016F8D7
:201D0000022806D2FFF77DFE03E00020FEBD01F092FC39460198FFF79FFF22017168FF2349
:201D2000541C0B558A5C2B01CA54FEBD401A00020121000AC905884200D900207047000018
:201D4000981B00207372635C736F635F74696D65722E6300F0B500241C4A01211C4B0803F3
:201D6000546018601B4B1C601B4C20601B480469E443E406E6170469761C10252C43046188
:201D8000174C6160174D296000E020BF1F68002FFBD0002E03D107691026B74307619068F0
:201DA0008005906801D5104A10436960A160002119600121084A09031160F0BD10B5044612
:201DC000FFF7C8FF2060002010BD000000C5004080E100E000C1004080E200E000ED00E083
:201DE00000C3004000C0004000FCFFFF70B51F490A68002A17D000231D4601244A68521C0B
:201E00004A60092A00D34D600E792246B2400E6816420AD072B60B6893430B6062B6496837
:201E20000160002070BD052070BD5B1C092BE5D30FA1362003F081F8F5E7012010498005F2
:201E400008607047EFF31081CA07D20F72B6012181400648036819430160002A00D162B6AA
:201E6000EBE702480021016041607047080100207372635C736F635F6576742E630000001B
:201E800000E200E0012081070860704701208107486070471048C068C00700D001207047C1
:201EA0000D488068C00700D0012070470A484069C00700D0012070470748C069704706498E
:201EC0008A69D20306D589698907890F814201D1012070470020704700040040F8B5FE4CC6
:201EE000207BE17A88421AD00126FC4D0027E07A215C14200A4642435019037C052B0FD0CA
:201F0000062B1BD0072B28D0437C012B33D0F4A1F64803F012F8207BE17A8842E7D1F8BD90
:201F20000674E07A0A2807D0E07A401CE072491CC8B2AA5802210CE00020F7E70674E07AFA
:201F40000A2808D0E07A401CE072491CC8B2AA5803219047DFE70020F6E70674E07A0A28CA
:201F600007D0E07A401CE072491CC8B2AA580821EFE70020F7E74774E07A0A2807D0E07A2C
:201F8000401CE072491CC8B2AA580721E1E70020F7E770B5D64D06206872D648002444777F
:201FA000047738300473C472D34801F0F7FDD3480475EC72D249601E88606C71AC70EC70C9
:201FC0002C716C70CF48022104704470CE480470047528300470491EFAD10120F1F76EFDB1
:201FE0000020F1F76BFD0120A871F0F785FDC748F0F794FDC64C2070C648F0F78FFD607054
:20200000F1F700FD70BD10B5F1F727FDC04C2078F0F7A2FD6078F0F79FFDB54C207A002895
:2020200005D0FFF730FAF0F726FE0020207210BD70B5AF4CA079002804D0A9A1B64802F0B2
:202040007CFF70BDE07A002804D11320A4A1400102F073FF0126A6710025E572607A0421AB
:20206000142250439D4A80180174A5488168491C04D0691E81600120F1F720FD0020F1F7FE
:202080001DFDF1F701FD01F023FEF1F706FEA348056005600120A249C0030860F0F78EFFE2
:2020A00098480078022804D0032804D1E078002801D0A67000E0A570F1F7DBFD70BD034638
:2020C00086490520142242435218203A127F002A04D0401E0006000EF4D170471422424355
:2020E00051180A46403AD362012220390A777047012805D0032805D1002903D100207047F1
:202100000029FBD010B47A4C002363707D4A002890700CD002280AD007291AD20B007B4496
:202120001B79DB189F441505070D0F111300D37003E01B2000E03A20D0700120607010BC3C
:2021400070475820F8E77720F6E79620F4E7B520F2E710BC0020704710B56A484078F1F704
:20216000A3FD80B210BD411E1422504310B55B4A8418203C042902D8207F002803D158A19B
:20218000684802F0DAFE207F012803D054A1664802F0D3FE0020207710BD70B5554C607F9B
:2021A000217F884201D1012500E00025F1F715FDF1F77AFD617F227F914201D1012100E037
:2021C0000021A942EBD170BDF7B50646481E84468EB0C0B2142204905043404A8518284640
:2021E0000595007C2D1D07282AD13B4C0027E07A227B824221D0235C049A934201D101270F
:2022000001E0002F04D00A2811D0421CA25C22540A280ED0401C227BC0B28242EBD1002FCB
:202220000BD0207B002806D0207B401E04E00022ECE70020EFE70A202073059A0120107461
:2022400060462B4C04280FD814204143234808182038007F002807D00598007C012807D01C
:202260001098807A012807D01DA1304802F065FE1098807A012871D10598184B007C02287E
:202280001AD0154C207B0A2874D0207BE17A401C884204D1C92012A1800002F04EFE0599F9
:2022A00001204874217B04986054207B0A2865D0207B401C20731CE1607A049A014690423B
:2022C00006D0014614277843C018807C9042F8D1627A824235D12BE0A41C0020B41C0020FB
:2022E0007372635C72656D2E63000000D5050000381D00206C1C0020441D00208C1C002025
:20230000181D002012010020C41C0020031A010010010020DD1E01007F02000000F5004034
:2023200080E200E0CD020000CE02000017030000617A14225143C918897C61720121A1720F
:2023400007E014224243D21814277943927CC9188A74142206215043C01881741098007A2E
:20236000062819D203007B441B79DB189F440812100E0C0AE07A00288CD090E7002099E7D5
:2023800000210FE0B4210DE073210BE0322109E00A2107E0062105E0FF20FE49E23002F028
:2023A000CCFD0021109802910068401A28601099097A002912D00221401A0102090A29605B
:2023C00010980268406810180002000A68601098807A0228109803D0007B74E00421EBE73A
:2023E000007A002813D0022202981018844610984268604608301718E748029A40789042F4
:2024000002D9E278002A04D03846083005E00422EAE7029A801AC0190830627A062A1CD0B8
:20242000627A14235A43DD4BD2185268914214D0DB4B0793617A14225143D84A89184A688F
:202440008968921B891B12020902120A090A90423AD89A4238D8994236D83018C01B00020E
:20246000000A286010996044CE4AC9680002000A9446421A01239B0507929A4201D2104690
:2024800014E00A1A09929A4201D207980EE0079A6346624503D9591A0818401C06E0099A08
:2024A000624506D9181A4018401C404200285FDC03E0B849BC4802F040FD2868C019000249
:2024C000000A6860002028726868082708300002000A68601098407AA8721098007A6872ED
:2024E00003280ED200280CD0FFF7D4FC002803D007E0002011B0F0BD02983A210F1A322027
:202500000290A5480178012901D0032909D141780298814205D9E078002802D10298081ABF
:20252000C71928689E4A801B844601026868090A801B03021B0A8F421AD81746914217D851
:20254000BB4215D8617A062916D0677A61460622039200923A4614235A43904BD2189368B6
:202560009B1B8B4216D80397977C062FF2D177E0049801F059F9BCE7059802220499027498
:20258000627A062A00D0627A827461720120A07211B0F0BD062F63D0002239469446142200
:2025A0007E4B4A43D21853689B1B834229D2917BAB7A99421FD805980521049C7B4D017407
:2025C000287B0A2811D0287BE97A401C884203D17049774802F0B1FC287B2C54287B0A2836
:2025E00007D0287B401C287383E7E87A0028EFD0F2E70020F7E701218C46917C0629CED111
:2026000002E0604600282AD03D46009114202A46424362480621161831741038007B0A283A
:20262000624816D0017BC07A491C814203D161A1634802F082FC5D48017B4554017B0A29D2
:202640000BD0017B491C0173B57C0098A842DDD106E0C07A0028EAD0EDE70021F3E7009781
:202660000599022008744D4D607AB84207D1059900988874049860720120A07221E0039869
:20268000062F0FD0062803D14AA14E4802F055FC03981422504340190499817405990098DB
:2026A00088740EE0062803D142A1474802F045FC0398142250434019049981740599062076
:2026C0008874012011B0F0BD70B50D4606463F4900242046891BA04103D236A13C4802F0F2
:2026E0002CFC3C490020491BA04103D231A13A4802F023FC394A70190021821A8C4101D324
:202700003749401870BDF8B5401EC0B21421484322494518687B062813D203007B441B7963
:20272000DB189F44020C0A080604002066E0B42010E073200EE032200CE00A200AE0062076
:2027400008E0FF201BA1E23002F0F7FB697B0020002953D0022140186968002440180C217B
:2027600000026956000A00294ADBF1F79DFA174A06460C27EF570021101AA14103D20DA1EB
:20278000134802F0DAFB13490020C91BA0412CD208A127E0E022010012010020B41C002002
:2027A000FFFF3F00FFFFFF0014070000A41C0020090200007372635C72656D2E6300000060
:2027C000C7030000DF030000E5030000FF7F841EF50300000020A107F60300000080841E6A
:2027E00000807BE1FB4802F0A8FBFB4AF0190021821A8C4101D3F9494018F8BD0421AAE774
:20280000F1F752FA0C21695600224018F449091AA241F2D24042F8BDF0B5064683B0F14883
:202820000190457A029534687068001B0702EE483F0A001B0090062D2DD014202946414398
:20284000EA480122081884464168E74892058646081B904210D3631A93420DD302467046F6
:20286000724503D900984018401C05E073450ED9411A0819401C404200280CDA6046029550
:20288000857C0198C0790028D5D003B0F0BDD849D84802F052FB0298854226D014214843A1
:2028A000D2490123401802908068CF499B058C46011B8646994210D3221A9A420DD3634636
:2028C000614503D900997144491C06E0194662452DD9091A0819401C4142002905DD029809
:2028E000B17A807B814200D37446062D15D0BF491420454368184268121B1202120ABA4203
:202900000BD2B27A837B9A4200D38468857C0198C0790028B9D1062DEAD13068A042B4D0A4
:20292000E0190002000A3460706003B0F0BDB049B04802F002FBD8E7F0B5AF490446486898
:2029400085B0C005C00D1CD0103840B200280CDA0207120F083A920892005118C9698007C2
:20296000C00EC1400806800F09E08108A34A8900891809688007C00EC1400806800F0028D6
:2029800008D000262078002806D0012804D0002005B0F0BD0126F5E72079062813D2030072
:2029A0007B441B79DB189F44020C0A080604002018E0B42010E073200EE032200CE00A20FF
:2029C0000AE0062008E0FF208949E23002F0B5FA21790020002905D002214718814D002E25
:2029E00002D003E00421F8E70020E87102AA6946A068F1F763F9694608228A56E06801A953
:202A00008018C01C01221F2801DA019209E003AAF1F754F96846007B002802D00198401C87
:202A2000019000990198401808300002000A0190C81B0002000A009060796946887200980D
:202A40000390F1F7CAF8009A019B121A181A6C4912020002120A000A8A4216D8884214D844
:202A60006846FFF7D9FE00990398814205D0C8190002000AF1F718F9A0600120E97900297D
:202A800086D0002EB0D005B0F0BD0020F6E7F3B58FB05C480C460B9001F088F85A4A0F999E
:202AA000504E5518203D594F00280BD05848007D002803D057A15A4802F03FFA2078012865
:202AC0007DD05FE1787F0A280CD0787F397F401C884203D14FA1534802F02FFA2078012854
:202AE00004D00CE0387F0028F4D0F7E7E87F002803D048A14C4802F020FA0120E877787F33
:202B00000F991422494D5043401901742078022823D0787F1421484345192079287260790A
:202B200068722A460C322946A068F1F7C7F80C2028560F2804DD1F3828732868401C2860C7
:202B40000C22AA56281DE16802908818C01C1F283FDA029901200860FDE027494868C00565
:202B6000C00D20D0103840B200280CDA0207120F083A920892005118C9698007C00EC140C7
:202B80000806800F09E081081C4A8900891809688007C00EC1400806800F002803D11DA178
:202BA000234802F0CAF9787F1421484345190021E0686A460591117303AA05A900E0D8E0BA
:202BC000F1F77CF86A460C2010560F2832DD012031E0B3E0F60300000080841E00807BE155
:202BE000FF7F841E381D0020FFFFFF00B41C0020B42701001407000000ED00E000E400E0CB
:202C0000FFFF3F00441D0020160100206C1C00208C1C00207372635C72656D2E63000000D6
:202C200017050000F5040000FA040000AC1B00200605000000200599401808900220A872A5
:202C40002079287260796872A068291DC01C03911F2801DA01200AE006AAF1F72FF8684636
:202C6000007E002804D0039803990068401C0860287A062813D203007B441B79DB189F4496
:202C8000020C0A08060400200FE0B4200DE073200BE0322009E00A2007E0062005E0FF2046
:202CA000FD49E23002F049F900202179002943D002214118069168680831401808990590E8
:202CC00008180699401A0C900020F071F0F785FF04462860089820180002000AE860707A6B
:202CE000062825D0707A14214843EC49401840680090059940180002000A0190687A69461E
:202D000088726846FFF788FD0098019A001B121B00021202E24B000A120A0C99984207D84E
:202D20008A4205D80099069808180002000A2860F0790028C8D110E00421BAE704AA0299D6
:202D4000F0F7BCFF6846007C002804D0029802990068401C08602078A872787F0A2806D099
:202D6000787F401C78770B9800F038FF47E00020F8E7E87F002803D0CAA1CD4802F0DDF878
:202D80000120E877CB490F9808742078022803D1C4A1C94802F0D1F8C64D20792872607996
:202DA00068722A460C322946A068F0F787FF0C2028560F2804DD1F3828732868401C28607F
:202DC0000C22AA56281DE16802908818C01C1F2803DA0299012008600CE003AA0299F0F7C6
:202DE0006DFF6846007B002804D0029802990068401C08602078A872AE4901200875797FA2
:202E0000387F814223D0747A062C22D0F0F7E5FE14214C43A1496218117C042917D0032974
:202E200015D0536892681B1A101A1B0200029C491B0A000A082B0AD30A468B4207D8904288
:202E400005D8787F397F884201D0F0F712FF11B0F0BD787F397F8842F7D111B0F0BD10B571
:202E60000020F0F718FE10BD10B50120F0F713FE10BDF1B5009802281FD0904C607A062882
:202E800003D188A18E4802F058F80026A6710125E572607A03211422804F5043C01901747F
:202EA000F0F7ECFE009800280CD001282AD003287CD0B5207BA1C00044E082480078EFF70E
:202EC00051FEF8BD8048007F002803D075A17F4802F033F865717C4D00202E60F0F7EEFD93
:202EE000A968481C04D0012300221846F0F71CFE607A617A401CC0B2142251437A580121A3
:202F00009047F8BD0120F0F7D9FD607900280DD06D488068401C09D0607A617A401CC0B214
:202F2000142251437A5806219047F8BD6648007F01280AD0022812D0032824D0042836D0B5
:202F400058A1634801F0F9FFF8BD2079002803D02671F0F798FEE5705B480677F8BD207AC3
:202F6000002804D1FEF770FAEFF75CFE2572607A617A401CC0B2142251437A580021904707
:202F800051480677F8BD504F0123397B78680022411A1846F0F7C8FD2079002803D026715D
:202FA000F0F771FEE57002203877F8BD1BE0464E217870680123411A00221846F0F7B4FD49
:202FC000207A002804D1FEF73FFAEFF72BFE2572607A617A401CC0B2142251437A58002146
:202FE00090473577F8BD607A617A401CC0B2142251437A5805219047F8BD10B52F4C607AAE
:20300000062803D127A1334801F097FF607A617A401CC0B214225143204A52580421904787
:2030200010BDF0B583B006200290F0F7D6FD234C0090617A28480190062920D0617A142070
:20304000414316480918097C042918D0617A142251430818007C03287BD00198009A03687E
:2030600040689B1A801A1B0200020D491B0A000A082B6ED30A468B426BD8904269D8124874
:203080008068401C03D007A1144801F056FF00206071607A062823E0142C0100B41C0020A2
:2030A000FFFF3F007372635C72656D2E630000001E0500008C1C002024050000381D0020D1
:2030C0005505000010010020181D0020610500009C050000AF050000281D0020EB05000000
:2030E00007D16078002804D0FE48C178417081780170607A062815D0607A1421FA4A4843BF
:203100008018007C04280DD1607A0290617A01201423594389180874617A59438918897C1C
:203120006172A072F14D687F297FF14F884233D0F04E287F142148438019007CC05D0128D0
:20314000287F07D048438019007CC05D02282FD044E001E2142148438019807A01280AD0AE
:20316000287F0221142250438019007CC155287F0A2808D009E0297F0020142251438919C3
:20318000097CC8552AE0002001E0287F401C2877687F297F8842CCD1D74D287D00284CD0DD
:2031A000287CC15D012928D0C05D022830D03AE0287F142148438019807A012803D0CFA164
:2031C000D14801F0BAFE297F00201422514389198872297F51438919097CC855287F1421A3
:2031E00048438219287F48438019017C0098FEF7EBFF287F0A28C8D1C5E7A97A012904D0AB
:203200000221C155002028750DE00021C1550AE0A87A012803D0B9A1BC4801F08EFE002091
:20322000A872297CC855287D002806D0297CB24A0098FEF7C9FF00202875029806281ED0A6
:2032400014214843A8494018017C012917D10721AF4D0174287B0A283CD0287BE97A401CFA
:20326000884203D1A5A1AB4801F067FE297B02986854287B0A2831D0287B401C2873607ADD
:2032800006287DD0A07A00287BD00020A072617A142041439448A04B0A18566891681D465E
:2032A000D2687C35DE67AA6069609C4D697E002916D00226617A14228B4851430818407BB1
:2032C00006281BD203007B441B79DB189F440A1412100E0CE87A0028C4D0C7E70020CDE7AD
:2032E0000426E7E700200FE0B4200DE073200BE0322009E00A2007E0062005E0FF207FA1F2
:20330000E23001F01AFE00202873697E022901D0012910D12969009A09188A1A1202120AC8
:203320003A2A08D90320687632390802000A2861322028730AE0322808D2207A00280ED193
:20334000FEF782F8EFF76EFC012007E0207A002805D0FEF798F8EFF78EFC002020726149BE
:203360000822487820700978012901D0032906D101212171297B884201D9421A083201E0E1
:2033800091E0A1E0A378002B00D0921C2179002901D1002B5DD09446614A00990092019A3F
:2033A000176852687F1A511A3F0209023F0A090ABC451BD85A4A974218D8009A914215D86D
:2033C000297B884223D92B69421A9A1A1202120A101880190002000A2A616860002914D082
:2033E000032028770006000E3ED14CE000202071A070297B002925D02869401880190002B5
:20340000000A6860022028772EE00120E9E781420BD92A69511889190902090A69600028C6
:2034200001D00420DDE70220DBE7002B03D133A13C4801F082FD286980190002000A68602A
:20344000002004E0296989190902090A6960287719E0287B00280FD02969081880190002BE
:20346000000A68600220287728690123811900221846F0F759FB09E0286980190002000A90
:203480006860002028770120F0F718FB607A1421484315490C22401882560123002069681F
:2034A000F0F742FB10E00120F0F708FB0020F0F705FBF0F7E9FA207A002805D0FDF7E3FFAF
:2034C000EFF7D9FB00202072A078002804D0F0F7DAFB0020E070A0706078002827D00148F0
:2034E000C17821E012010020B41C00206C1C002015010020AC1B00208C1C00207372635C3E
:2035000072656D2E630000000D06000029060000A41C00203B060000AC1C0020181D002036
:20352000FFFF3F008D0600004170817801702079002806D00020CE49E0700978002900D107
:203540002071CC48017BC07A814203D0CA484078EFF708FB0120E07103B0F0BDF0B5C74C3D
:203560000746607A83B0062804D16F20C4A1000101F0E3FC607A1421C44E48438019007C68
:20358000032803D0BEA1C24801F0D7FCC14DA868401C03D0BAA1C04801F0CFFC607A142185
:2035A000484381190C20085600216A4600911171C01901AA6946F0F781FB6A4604201056A8
:2035C0000F2801DD012000E0002000994018696840180102090AA9606079002804D0012383
:2035E00000221846F0F7A0FA03B0F0BD70B5AC4CAA4A0B1AA34214D3451AA54211D3934269
:2036000003D9101A43185B1C0BE0954204D9511A0818401C434204E099A1A24801F08DFC45
:203620000023184670BD10B50146012300220220F0F77AFA10BD10B50220F0F73FFA10BD6C
:2036400010B5F0F7CAFA10BDF0B58C4D0446E87A83B0002803D18AA1934801F06EFC642CE3
:203660004DD3924A00210846121B884147D39048417F007F814242D18E48007D00283ED158
:20368000687A1421814F4843824EC519306801AA00196946F0F712FB6946042008560028B2
:2036A00002DD0098401C0090A96800986B680A18D21A1202804B120A9A4220D8AA7C062AF8
:2036C00008D014235A43D2195268511A0902090A814214D3B068401C05D00120F0F7EEF92E
:2036E0000020C043B060306800193060A868009940180002000A7061012003B0F0BD0020D7
:2037000003B0F0BDF8B50646401EC4B214205F4960434518287C002804D1772058A100016E
:2037200001F00BFC6248017F407F81420CD0634A14234B439B181B7CB3420CD00A290CD06D
:20374000491CC9B28142F3D15A48017D002961D0007CB0425ED10020F8BD0021F1E70529EF
:2037600003D0062901D0072928D101212974C17A0023027B8A4221D00246565CA64201D142
:20378000012301E0002B04D00A2911D04E1C965D56540A290ED0491C167BC9B28E42ECD1FB
:2037A000002B0BD0117B002906D0117B491E04E00026ECE70021EFE70A211173697C0029F4
:2037C0002AD06F74C17A0023027B8A4224D0425CA24201D1012301E0002B04D00A2912D004
:2037E0004A1C825C42540A290FD0491C027BC9B28A42ECD1002B0FD0027B0146002A06D029
:203800000A7B521E04E00022EBE70021EEE70A220A7301E017480027297C01299FD16A7CB0
:20382000002A9CD10120F8BD70B505461420174A0521684380180F4C0174207B0A2811D02F
:20384000207BE17A401C884203D10DA11C4801F074FB207B2554207B0A2807D0207B401C57
:20386000207370BDE07A0028EFD0F2E70020F7E712010020A41C002010010020381D0020B7
:203880007372635C72656D2E63000000B41C0020F1060000181D0020F2060000FF7F841E5B
:2038A0000020A1071407000033070000FF1FA1076C1C00208C1C0020FFFF3F00AC1B002091
:2038C0000902000010B501462022094801F099F907490020C877084610BD064901204861D8
:2038E0000548064A0168914201D1002101607047481D0020000500401C010020BEBAFECA9D
:20390000064A10705170704704481C2201784171427001707047704770477047200100206A
:2039200030B50346002002460DE09C5C2546303D0A2D02D30020C04330BD0A2568433038D6
:203940002018521CD2B28A42EFD330BD70B50D46144608E00A2101F0CEF92A193031203A27
:20396000641ED177E4B2002CF4D170BD10B5002310E0040A00020443A0B2CC5C4440200676
:20398000000F60400407240C44402006C00C60405B1C9BB29342ECD310BD10B520380C4693
:2039A000030001F0BBFB33E0DBE41B1F23272C31373C41474D5054585C606D716569747812
:2039C0007C8084888C9094989C9FA2A6AAAEB2B8BCC0C5CACFE9F0F3D3D7F800206800F092
:2039E000DDF8D6E0206800F0E1F8D2E0206800F0F5F8CEE0207840B200F092FAC9E02078DF
:203A000040B200F0B0FAC4E02078616840B200F0C3FABEE0207840B200F0D3FAB9E0207860
:203A200040B200F0DEFAB4E02078217940B200F0E9FAAEE02078616840B200F013FBA8E0DA
:203A400000F01FFBA5E0206800F023FBA1E0207800F038FB9DE02068FDF7F5FD99E0206819
:203A6000FDF7F5FD95E021792068FDF7F7FD90E02068FDF73FFC8CE02068FDF740FC88E02E
:203A80002078FDF740FC84E0FDF74EFC81E02078FDF750FC7DE02078FDF762FC79E020685B
:203AA000FDF77BFC75E02068FDF77DFC71E02068FDF77FFC6DE02068FDF780FC69E02068F3
:203AC000FDF782FC65E02068FDF784FC61E02068FDF785FC5DE00846EDF738FB59E0EFF734
:203AE000B4F856E0EFF7E1F853E02068EFF7E9F84FE0206800F080F84BE0206800F082F867
:203B000047E0206800F083F843E02078A268616800F082F83DE0207800F089F839E02078BC
:203B200000F091F835E02078616800F098F830E02078616800F09FF82BE02179207800F0F1
:203B4000D5FB26E02068FDF778FE22E02068FEF74DF91EE02068FEF731F91AE0204607C804
:203B600000F0B9FC15E0206800F00CFD11E06168206800F037FD0CE0206800F029FF08E050
:203B800009E003E0FFE700F03BFF02E0206800F073FF206010BD0120086010BD0021017048
:203BA000084670470146002008707047EFF31081C907C90F72B60278012A01D0012200E0AE
:203BC000002201230370002900D162B6002A01D000207047012040037047E7E7EFF31081EC
:203BE000C907C90F72B600220270002900D162B600207047F2E7000038490968C9B20160D1
:203C0000002070473549C0B24860002070473349C0B2886000207047082801D3304870477E
:203C2000C3002E4818180161426100207047022802D32B48401C70472A4A0121C0008018CC
:203C4000016000207047022802D32548401C7047244A0121C0008018416000207047022823
:203C600002D31F48401C70471F4A8000C9B28018016000207047022802D31948401C70474E
:203C8000194A800080180068C0B208600020704710B5FF20114AC043906008200021C30052
:203CA0009B1819615961401C1028F8D300200E4A05E0022803D383009B18196004E083004B
:203CC0009B181C68E4B21C60401C0428F1D310BDFF200249C04388607047000000F5014040
:203CE0000820000000F0014000F8014010B572B600F0DEF800280BD0EDF7D2FAFEF783F95B
:203D000000F0BBFA6F490020C86288626E49086062B6002010BDF3B5002501200007C06ACF
:203D200081B0C0430006000E04D168480068401C00D1012572B600F0BBF8002801D062B61F
:203D400087E0EDF719FAEDF7AFFA614C614A00212368CB40DB071FD00346CB40DB0718D179
:203D60004BB2002B07DA1E07360F083EB608B600B618F66904E09E08574FB600F619366856
:203D80009B07DB0EDE4033069B0F012B04D0032B02D062B65148FEBD491C2029D8D3019C35
:203DA00001204F49230001F0B9F9142224242424242424240B0D1012142016181A1C1E2F0F
:203DC000002400E00124C86314E00224FBE70324F9E70424F7E70824F5E70924F3E70A2449
:203DE000F1E70B24EFE70C24EDE70524EBE7072400E00624D06901210002000AC907084330
:203E0000D061002D04D009E062B601200003FEBD2C4D3448E862EDF747FAA8622A49324835
:203E20000860324902980860EDF73EFA214600F00BFAFEF7AEF800F00DFC00F087FA019887
:203E4000EDF7FCF9040062B603D0FFF74FFF2046FEBD0020FEBD10B5044600F029F8002812
:203E600000D001202070002010BD214908600020704710B50C46102808D011280BD01228B6
:203E80000CD013280ED00120086010BD61682068FFF741FF0AE0FFF729FF07E02068FFF7E3
:203EA000DAFF03E01249206808600020206010BD05480D490068884201D1012070470020EF
:203EC00070470000000500401C0100200010001000E100E000ED00E000E400E00110000026
:203EE0004000004000200000BEBAFECA28010020040000208107C90E002808DA0007000FF6
:203F000008388008814A80008018C06904E080087F4A800080180068C8400006800F7047C4
:203F200010B5044600F0DBF8002813D02046FFF7E1FFC0B200F0E1F800280DD07549E20682
:203F40000B78D20E01209040002B08D04A681043486006E0704810BD6F48401C10BD6F495A
:203F60000860002010BD10B5044600F0B8F800280BD06849E2060B78D20E01209040002B22
:203F800005D04A6882434A6004E0634810BD634980310860002010BD70B50D46044600F06B
:203FA0009EF800280BD05E480068E206D20E01219140084000D001202860002070BD5648F3
:203FC00070BD10B5044600F08AF8002807D0E106C90E0120884052490860002010BD4E4807
:203FE00010BD10B5044600F07AF8002808D0E106C90E012088404A4980310860002010BD43
:20400000454810BD70B50D46044600F068F8002819D0284600F071F8002816D0A007C20ED7
:20402000FF209040A907090E9140002C10DA2207120F083A9308354A9B009B18DA698243E7
:204040000A43DA610CE0344870BD3348401C70BDA3082F4A9B009B181A6882430A431A60BF
:20406000002070BD70B50C46054600F038F8002805D02846FFF73EFF2070002070BD264828
:2040800070BDBFF34F8F21492648C860BFF34F8FFEE770B51F4C05462178012000290ED151
:2040A000207072B600F0F8F81C4E803631688143616000F0F1F8C043306062B600202870EE
:2040C000002070BD13490A78002A06D0002804D1124A48681060002008700020704710B508
:2040E0000446202805DA00F0D7F80121A140084201D0002010BD012010BD012803D0032870
:2041000001D00020704701207047000000ED00E000E400E02C0100200120000000E100E05F
:2041200000E200E00400FA05F8B50446800700250126002804DA5A48C563C663022084430E
:20414000E00404D55748C563C66380148443600003D55548456080058443E00504D5534838
:20416000C563C66380158443A00404D55048C563C6634014844360042704C00FF90F8842E1
:2041800003D04CA1612000F0D8FEB80F0AD04E49CD634E48C563C563CE63C663C663032024
:2041A0008003844320050AD5494FFD632F20ECF7FBFFFE632F20ECF7F7FFF8148443002C05
:2041C00003DAFFF765FD640064084248044203D038A1902000F0B1FEF8BDF0B500210A4644
:2041E000FF230446CC40E4072AD04CB2E606F60E0125B540384E3560384E3560002C11DA0C
:2042000025072D0F083DAE08354DB6007619F569A407E70E1C46BC40A5431446BC40254372
:20422000F5610DE0A6082F4DB60076193568A407E70E1C46BC40A5431446BC4025433560F6
:20424000491C2029CDD3F0BD70B5274C0D462060FFF76AFF2068FFF7C0FF2846EEF7BEFD4E
:20426000FDF7D6FAFDF782F9FFF712FDFDF7D5F8EEF742FC00F06AF870BD10B51A4C2068F0
:20428000FFF752FF2068FFF7A8FFFFF701FDEEF72AFE0020206010BD1348006870470000CA
:2042A000C01F0040C0CF004000E50140C08F0040C0DF00407372635C736F635F636F6E668E
:2042C00069672E6300000000C0EF0040C0FF0040C0BF0040FEFF0FFC80E100E080E200E045
:2042E00000ED00E000E400E03401002070B5002402460D4620462146002A1ED0012A04D010
:20430000022A04D0032A1ED103E0012002E0022013E003202B0000F001FF07160507090B0B
:204320000D0F1600012108E0022106E0032104E0042102E0052100E00621FDF7D9FE002809
:2043400001D0204670BD0724FBE70000B148002101708170704770B5AF4D01236B60AF4BAF
:204360001C68002CFCD0002407E00E6806601E68002EFCD0001D091D641C9442F5D30020D9
:20438000686018680028FCD070BD70B5A14C0D466178884203D0A2A16C2000F0CEFD2B0024
:2043A00000F0BCFE094F0625254F4F4F4F464F002078022803D09AA1702000F0BEFD0320AC
:2043C0002070A078022802D0012804D008E0A06800F0CEFB04E02269E168A068FFF7BBFF23
:2043E0000020A070FDF724FE0420207070BDFDF7D4FE01466068FFF7F9F8054620780228CD
:2044000003D087A1842000F098FD894A89498A48954206D8401BC86086496078FEF737FBFB
:2044200070BD854202D802224A71F3E7032003E0A0780028FAD10220FDF704FD00F0E0F805
:2044400070BD77A1AD2000F078FD70BD70B50546FDF7A3FE6F4C60602078012803D070A193
:20446000B42000F06AFD73490220087000220A718D6003224A71704ACA6020706078FEF710
:2044800006FB70BD10B5634CA078002802D12078002801D0112010BD6848FDF710FE607056
:2044A0006078002803D001202070002010BD032010BD10B50124020B64040121604BA0428D
:2044C00002D29140186802E0203A58689140084000D0012010BDF8B50E46910005464F199F
:2044E00014463F1F009100F054FB009980028919091FB14201D2012200E00022002C03D065
:20450000FF2101318C4201D90920F8BD4D498D4219D3AF4217D3854205D2874203D22846ED
:204520003043800701D01020F8BD8E420BD3002A09D12846FFF7BDFF002804D13846FFF788
:20454000B8FF002801D00F20F8BD3F483F490068884205D0224631462846FFF7FCFE0FE085
:20456000FFF790FF0028EFD12A480121C6608560046181702046312148431430FFF766FFF7
:204580000020F8BD10B504462E48800A84420BD300F0FFFAA04201D8102010BDA002044606
:2045A000FFF787FF002801D00F2010BD264827490068884203D0204600F0DAFA0AE0FFF79D
:2045C00061FF0028F1D113480221846081702048FFF73CFF002010BD1A48010B0120884061
:2045E000401E704700B50B460246FFF7F5FF104201D00F2000BD124802604360002000BD23
:2046000010B5044C6078FDF7AEFD00202070A07010BD00003801002000E5014000E40140DD
:204620007372635C736F635F666C6173682E630030750000681D0020D0FB01008B430100AE
:2046400000060040006001001C010020BEBAFECA10540000F7480521817000210170417039
:20466000C1708160704710B5F3490A78022A07D0CA681018C860C8689638FEF76FFF10BD3B
:204680008A68101888608868F6E70378EB49EC4A002B02D0012B10D014E00379002B01D0F1
:2046A000012B0FD14379002B01D0012B0AD18368643B8B4206D2C06810E00379002B03D06E
:2046C000012B01D0002070474379002B01D0012BF8D1C368643B8B42F4D280689042F1D879
:2046E00001207047F8B504460226FEF7BDFB0068002803D0D3A1BE2000F01FFC0127CD4D14
:20470000002C08D02078002817D0012805D0022811D0032813D02F710DE06068C82808D3B7
:20472000FEF792FF002804D06068FFF79CFF012603E0002601E000F0F9F93046F8BD2878E0
:204740000028F8D16068FFF7A0FF0028E3D060680078002826D0A878042803D0B9A1F82041
:2047600000F0EBFBB44F0020387060680079012800D00020387160684079002837D00320C2
:20478000787160688168E868FDF79EFFB8606068C0689630F8600320A870A749E878FEF7F8
:2047A00076F9C8E7A4480221017061680979012919D00021017161684979002915D00321AD
:2047C000417161688968963181606168C968C160C068984C14346060FDF7DFFC20606F7068
:2047E0000220A870A7E70321E4E70221E8E70220C6E7F8B58F4C0D46E178884204D0FF2050
:2048000090A11A3000F099FB28468A4F002501261437030000F082FC090612375A7C8D97F8
:20482000C4A0C400A078032807D0A078022804D0FF2084A11E3000F080FBF8BDA07803282B
:2048400007D0A078022804D0FF207EA1223000F074FB0420A07025712078002810D1FFF71B
:2048600002FFE078FDF74FFFE0607D49886A7D4A024022617B4AD24310408862002050E0B5
:2048800000F054F9F8BDA078032807D0A078022804D0FF206BA1453000F04FFB207800285C
:2048A00002D000F04FF9F8BDA07803281FD104202AE0091A6048C1600146E078FEF7E7F879
:2048C000F8BD0420FDF7BEFAA570F8BDA078032807D0A078022804D0FF205AA1663000F0B9
:2048E0002CFB20780028DCD1A07803280BD0FDF754FC01463868FEF779FE0028E1DB7968AA
:204900008142DEDBD5E70520FDF79CFAA670F8BDA078042804D0FF204AA1873000F00DFB14
:204920000220A1688847FFF7DDFEFF260546C03642E0A078042804D0FF2042A18C3000F05E
:20494000FCFA0120EDE7A078042899D0FF203DA1913000F0F2FA93E7A07804280AD06078B5
:20496000002802D0A078022804D0FF2035A1963000F0E3FA2078002893D12079002804D0E6
:204980000620FDF75FFA2571C0E76078002805D02949E078FEF77BF86570F8BD0720B3E715
:2049A000FF2028A1B13046E7002D0AD0012D06D024A1304600F0C1FA022DF5D1F8BD042042
:2049C00000E00320A1688847FFF78CFE0546F3E770B5050005D0174CA078052803D01120AC
:2049E00070BD102070BD2048FDF769FBE070E078002803D0A5600020A07070BD032070BD18
:204A000010B50C480178002901D0112010BD817805292BD0817801292AD08178002927D0B4
:204A2000012101708178012922D0807800281FD020E000004C010020781D00203D860100D9
:204A4000FF1FA1077372635C736F635F726164696F5F74696D65736C6F742E6300000000D8
:204A60000005004002810080F34701000F2010BD00F068F8002010BDF8B5394E0446B078D4
:204A8000002801D001280DD1002C0DD02046FFF7FCFD00280AD02078324D002808D0B07877
:204AA000012823D00F20F8BD1020F8BD0720F8BD02272F702079012814D000202871607935
:204AC000002811D003206871A0689630A860E068E860E868224C14346060FDF75EFB2060D8
:204AE000B77019E00320E9E70220ECE7002028702079012816D0002028716079002813D0B1
:204B000003206871A168F068FDF7DEFDA860E0689630E8600320B0701249F078FDF7B7FF5B
:204B20000020F8BD0320E7E70220EAE710B50E48816A0E4A11400A4A126911438162FDF713
:204B400077FA10BD10B5064CE078FDF70CFB0820FDF778F90520A07000202070607010BD9E
:204B60004C010020781D002000050040FD7EFF7F0A4A022151600A490B68002BFCD0906000
:204B800008680028FCD00020506008680028FCD070470120000740697047000000E5014018
:204BA00000E4014070477047034610B50B439B070FD1042A0DD308C810C9121FA342F8D0EF
:204BC00018BA21BA884201D9012010BD0020C04310BD002A03D0D30703D0521C07E0002087
:204BE00010BD03780C78401C491C1B1B07D103780C78401C491C1B1B01D1921EF1D1184682
:204C000010BDF8B5042A2CD3830712D00B78491C0370401C521E83070BD00B78491C03709A
:204C2000401C521E830704D00B78491C0370401C521E8B079B0F05D0C91ADF002023DE1B14
:204C400008C90AE0ECF7C0FAF8BD1D4608C9FD401C46B4402C4310C0121F042AF5D2F30820
:204C6000C91A521EF0D40B78491C0370401C521EEAD40B78491C0370401C521EE4D40978D8
:204C80000170F8BD01E004C0091F0429FBD28B0701D50280801CC90700D0027070470029AF
:204CA0000BD0C30702D00270401C491E022904D3830702D50280801C891EE3E70022EEE75F
:204CC0000022DFE70378C2781946437812061B0219438378C0781B04194311430902090A6C
:204CE000000608437047020A08704A70020C8A70020ECA707047002203098B4273D3030A17
:204D00008B4258D3030B8B423CD3030C8B4221D312E003460B437FD4002243088B4274D384
:204D200003098B425FD3030A8B4244D3030B8B4228D3030C8B420DD3FF22090212BA030CDE
:204D40008B4202D31212090265D0030B8B4219D300E0090AC30B8B4201D3CB03C01A5241E9
:204D6000830B8B4201D38B03C01A5241430B8B4201D34B03C01A5241030B8B4201D30B03A2
:204D8000C01A5241C30A8B4201D3CB02C01A5241830A8B4201D38B02C01A5241430A8B42BC
:204DA00001D34B02C01A5241030A8B4201D30B02C01A5241CDD2C3098B4201D3CB01C01A8B
:204DC000524183098B4201D38B01C01A524143098B4201D34B01C01A524103098B4201D3C7
:204DE0000B01C01A5241C3088B4201D3CB00C01A524183088B4201D38B00C01A5241430827
:204E00008B4201D34B00C01A5241411A00D201465241104670475DE0CA0F00D049420310A1
:204E200000D34042534000229C4603098B422DD3030A8B4212D3FC22890112BA030A8B42A0
:204E40000CD3890192118B4208D3890192118B4204D389013AD0921100E08909C3098B428B
:204E600001D3CB01C01A524183098B4201D38B01C01A524143098B4201D34B01C01A524159
:204E800003098B4201D30B01C01A5241C3088B4201D3CB00C01A524183088B4201D38B0091
:204EA000C01A5241D9D243088B4201D34B00C01A5241411A00D20146634652415B101046C5
:204EC00001D34042002B00D54942704763465B1000D3404201B50020C046C04602BD704779
:204EE0007047704710B500F059F810BD30B58C180278401C13071B0F01D10378401C12090A
:204F000006D10278401C03E00578401C0D70491C5B1EF9D101E00B70491C521EFBD1A14223
:204F2000E6D3002030BD000001231B68134B1860134B1960134B1A607047134A134B13609A
:204F40007246053AF0E7114A0F4B1B689A420ED10D4B0020186001980D4B04B598470CBC4F
:204F60009E460246029800990A4B1B68184706980599094B1B68DB68184700007001002055
:204F8000740100207801002068010020EFBEADDEC538010028010020040000201D481E49EB
:204FA0007047FFF7FBFFECF7C9F800BD01200007C06AC0B2FF2804D118481949096888422C
:204FC00002D0184818490160184819490968884203D1184A13605B68184700BD20BFFDE795
:204FE00012481349096888420ED1134B18680B498842F3D080F308881049884204DD1048C3
:20500000026802210A4302600E4880470E4880470E480047881D0020881D0020FFFFFFFFF7
:20502000001000102C050040080000000010000000000020040000200060010000200020E2
:2050400024050040DB380100AD4F0100294F01001348704502D1EFF3098101E0EFF30881C2
:20506000886902380078102814DB202810DB23280BDB0C4A12680C4B9A4203D1602804DBC4
:205080000A4A1047022008607047094A10470000084A1047084A12682C32126810470000D6
:2050A000FDFFFFFF1C010020BEBAFECAAD1200009B390100733E0100040000200D4B0E4960
:2050C00008470E4B0C4908470D4B0B4908470D4B094908470C4B084908470C4B06490847A4
:2050E0000B4B054908470B4B034908470A4B024908470000FD2D00008D3D0000B52F000005
:20510000333C0000E13B000095390000B912000063170000F53C0000A32B000030B4744654
